:020000040800F2
:103000000080002055FD0008B7160108210C0108BA
:1030100000000000000000000000000000000000B0
:10302000000000000000000000000000BB160108C6
:103030000000000000000000BF160108C1CE00081B
:1030400089FD00088BFD00088DFD00088FFD00083C
:1030500091FD000893FD000895FD0008C3160108C6
:1030600099FD00082DCF00089DFD00089FFD000878
:10307000A1FD0008A3FD0008A5FD0008A7FD0008AC
:10308000A9FD0008ABFD0008ADFD0008AFFD00087C
:10309000B1FD000855CF0008B5FD0008B7FD0008D8
:1030A000B9FD0008BBFD0008BDFD000841CF0008C8
:1030B000C1FD0008C3FD0008C5FD0008C7FD0008EC
:1030C000EDAF16204A62304029BD56B31544E9BF22
:1030D00077900D9CFE0B88C07E2615FA8380734086
:0830E0000FCE674B80D541C003
:1030E80000000000000024400000000000005940DB
:1030F800000000000088C3400000000084D797410A
:103108000080E03779C34143176E05B5B5B89346DB
:10311800F5F93FE9034F384D321D30F94877825AA7
:083128003CBF737FDD4F1575FC
:1031300001000000000000000A0000000000000084
:103140006400000000000000E80300000000000030
:103150001027000000000000A08601000000000011
:1031600040420F0000000000809698000000000020
:1031700000E1F5050000000000CA9A3B00000000D5
:1031800000E40B540200000000E87648170000003D
:103190000010A5D4E800000000A0724E180900003D
:1031A00000407A10F35A00000080C6A47E8D030010
:1031B0000000C16FF286230000008A5D784563013C
:1031C000000064A7B3B6E00D0000E8890423C78AB5
:1031D00000B583B06B46073300221A700C4B1A6897
:1031E0000B4B802149000A431A60012000F012F8BD
:1031F000031E04D06B46073301221A7001E009F068
:103200003FFE6B4607331B78180003B000BDC04675
:043210000020024058
:1032140010B584B001900F236B4400221A701D4B2B
:103224001B68002B2BD01C4B1C681A4B1B68190005
:10323400FA2398000BF07AFC0300190020000BF02D
:1032440075FC030018000DF043FA031E12D1019B14
:10325400032B0AD8019901235B42002218000DF0C8
:1032640040FF0E4B019A1A600DE00F236B440122BC
:103274001A7008E00F236B4401221A7003E00F2335
:103284006B4401221A700F236B441B78180004B09E
:1032940010BDC0469C000020AC0000209800002017
:1032A400044B1A68044B1B68D218024B1A60C046C0
:0C32B4007047C046A40B00209C000020C6
:0C32C000014B1B6818007047A40B002095
:1032CC0000B585B00190FFF7F5FF03000293019B59
:1032DC000393039B013304D0084B1B68039AD31848
:1032EC000393C046FFF7E6FF0200029BD31A039A32
:1032FC009A42F7D8C046C04605B000BD9C000020DD
:10330C0082B001900091019B1B68044A1A40009BFB
:10331C001A43019B1A60C04602B07047FFFF3FFE84
:10332C0084B0039002910192039B5B69029A120292
:10333C00D2431A40029B1B0201990B4003490B40DC
:10334C001A43039B5A61C04604B0704700FFFF0745
:10335C0082B00190019B9B68044A13408022520565
:10336C001A43019B9A60C04602B07047E8FFFF6F9A
:10337C0082B00190019B9B68044A134001221A43BE
:10338C00019B9A60C04602B07047C046E8FFFF7FC1
:10339C0082B00190019B9B68044A134002221A439D
:1033AC00019B9A60C04602B07047C046E8FFFF7FA1
:1033BC0082B00190019B9B68044A134004221A437B
:1033CC00019B9A60C04602B07047C046E8FFFF7F81
:1033DC0000B589B001901F236B4400221A700023A2
:1033EC0006930023059300230293019B002B01D12C
:1033FC000123A8E1019B9B6D002B0AD1019B1800B6
:10340C0005F0DEFE019B0022DA65019B54220021AF
:10341C009954019B1B6818000DF015F9031E14D16B
:10342C00019B1B681800FFF793FFC84B1B68C8492A
:10343C0018000BF077FB03005B00029302E0029B89
:10344C00013B0293029B002BF9D1019B1B681800D6
:10345C000DF0F9F8031E0FD1019B9B6D10221A433E
:10346C00019B9A65019BDB6D01221A43019BDA6576
:10347C001F236B4401221A70019B1B6818000DF06E
:10348C00AAFD03000393019B9B6D1022134000D0F7
:10349C004CE1039B002B00D048E1019B9B6DAD4A96
:1034AC00134002221A43019B9A65019B1B6818006A
:1034BC000DF075FD031E37D1019B1B68DB681822CC
:1034CC0093431900019B9A68019B1B680A43DA60BD
:1034DC00019B1B681B699B009908019B5B689B0FF8
:1034EC009A07019B1B680A431A61019B5A68C02307
:1034FC001B069A4218D0019B5A688023DB059A421E
:10350C0012D0019B5A6880231B069A420CD0924B16
:10351C001B68924A13401900019B5A68F0239B03C5
:10352C001A408D4B0A431A60019B1B7E9A03019B28
:10353C005B7EDB031A43019B9B7E5B031A43019B5F
:10354C001B6B002B02D080235B0100E000231A438D
:10355C00019BDB681A43019B1B69002B04DA019B5E
:10356C001B695B005B0801E080239B031A43019BF2
:10357C002C215B5C5B001343069A13430693019B5F
:10358C0020229B5C012B15D1019B9B7E002B05D12E
:10359C00069B80225202134306930BE0019B9B6D0A
:1035AC0020221A43019B9A65019BDB6D01221A4371
:1035BC00019BDA65019B5B6A002B0AD0019B5A6A5E
:1035CC00E0235B001A40019B9B6A1343069A13434A
:1035DC000693019B1A6C019B5B6C1A43019B9B6CC1
:1035EC001A43019BDB6C1343059A13430593019B10
:1035FC003C229B5C012B03D1059B012213430593B9
:10360C00019B1B68DB68564A13401900019B1B6821
:10361C00069A0A43DA60019B1B681B69514A1340E6
:10362C001900019B1B68059A0A431A61019B1868D3
:10363C00019B5B6B1A0000210DF07BFC019B186851
:10364C00019B9B6B48491A000DF073FC019B1B6995
:10365C00002B09D1019B1B689A6A019B1B681021E6
:10366C0049420A439A623AE0019B1A6980239B0300
:10367C009A4234D1002304930CE0019B1A6E049BF4
:10368C009B00DA4013000F2213400F2B06D0049B33
:10369C0001330493049B072BEFD900E0C046049B35
:1036AC00012B09D1019B1B689A6A019B1B68102195
:1036BC0049420A439A6212E0019B1B689B6A019B78
:1036CC00DB69013B9B001C221340102252429A40A2
:1036DC001100019B1A6E019B1B680A439A62019BA5
:1036EC001B68DB68214A1340069A9A420BD1019B56
:1036FC000022DA65019B9B6D0322934301221A433E
:10370C00019B9A651CE0019B9B6D12229343102236
:10371C001A43019B9A65019BDB6D01221A43019BA5
:10372C00DA651F236B4401221A7009E0019B9B6D23
:10373C0010221A43019B9A651F236B4401221A70B5
:10374C001F236B441B78180009B000BDAC0000208F
:10375C00400D0300FDFEFFFF08270140FFFFC3FFE4
:10376C001902FEFF02FCFFDF04FFFF07E7FF3F83A8
:10377C0010B586B0039002910192039B1B68180050
:10378C000DF029FC031E6DD1039B54229B5C012B75
:10379C0001D102236DE0039B542201219954039B18
:1037AC001B68DB680122134013D1039B1B681800B4
:1037BC000DF0F5FB031E04D0039B1B681800FFF7EC
:1037CC00E7FD039B1B68DA68039B1B6801210A4316
:1037DC00DA6017246C44039B180000F025FA0300F0
:1037EC00237017236B441B78002B3FD1039B9B6DDD
:1037FC00214A1340802252001A43039B9A65039B73
:10380C000022DA65039B1B6D1C4ADA62039B1B6D5D
:10381C001B4A1A63039B1B6D1A4A5A63039B1B6852
:10382C001C221A60039B542200219954039B1B6891
:10383C005A68039B1B6810210A435A60039B186D3E
:10384C00039B1B6840331900029A17246C44019B9C
:10385C000CF045FF03002370039B1B681800FFF757
:10386C00A7FD03E017236B4402221A7017236B4445
:10387C001B78180006B010BDFEF0FFFFE93C0008F5
:08388C0089060108A3060108EA
:1038940000B587B00190009117236B4400221A7081
:1038A40000230393019B54229B5C012B01D102232F
:1038B400BBE1019B542201219954019B1B68180010
:1038C4000DF08DFB031E00D09EE1009B5B68022B74
:1038D40000D13EE1019B1A6980231B069A4204D061
:1038E400019B1B69BE4A934208D1019B1A68009B45
:1038F4001B68190010000DF048FBC9E0019B1A6E0B
:10390400009B5B681F210B400F2199400B00DB4398
:1039140013401900009B1B685B035B0B05D1009BE4
:103924001B689B0E1F22134098E0009B1B6801221A
:10393400134000D091E0009B1B680222134000D08A
:1039440089E0009B1B680422134000D081E0009BA7
:103954001B680822134000D079E0009B1B681022EA
:10396400134000D071E0009B1B682022134000D05C
:1039740069E0009B1B684022134000D061E0009B7B
:103984001B688022134000D059E0009B1A688023F2
:103994005B00134051D1009B1A6880239B001340A5
:1039A40049D1009B1A688023DB00134041D1009B5E
:1039B4001A6880231B01134039D1009B1A688023A5
:1039C4005B01134031D1009B1A6880239B01134093
:1039D40029D1009B1A688023DB01134021D1009B6D
:1039E4001A6880231B02134019D1009B1A68802394
:1039F4005B02134011D1009B1A6880239B02134081
:103A040009D1009B1A688023DB02134001D01223E2
:103A140024E0002322E0112320E010231EE00F23E2
:103A24001CE00E231AE00D2318E00C2316E00B23F0
:103A340014E00A2312E0092310E008230EE0072310
:103A44000CE006230AE0052308E0042306E0032330
:103A540004E0022302E0012300E00023009A5268FC
:103A64001F20024093400A001A43019B1A66009BE0
:103A74005B689B085A1C019BDB699A4208D8019B2E
:103A84001868009B5968009B1B681A000CF087FBA0
:103A9400019B1868009B1968009B9B681A00FFF73C
:103AA40043FC009B1B68002B00DBB7E04D4B180068
:103AB4000DF039FA03000493009B1B684A4A9342B1
:103AC4001DD1049A80231B04134018D1049B802227
:103AD40012041343434A19001000FFF715FC434B2B
:103AE4001B68434918000BF021F80300039302E01C
:103AF400039B013B0393039B002BF9D18EE0009BB6
:103B04001B683C4A93420ED1049A80235B04134001
:103B140009D1049B802252041343324A1900100035
:103B2400FFF7F2FB7AE0009B1B68334A934200D014
:103B340074E0049A8023DB03134000D06EE0049BFE
:103B44008022D2031343274A19001000FFF7DCFB3D
:103B540064E0019B1A6980231B069A4204D0019BEE
:103B64001B691F4A934207D1019B1A68009B1B687B
:103B7400190010000CF037FB009B1B68002B4DDA7A
:103B8400184B18000DF0CFF903000493009B1B6839
:103B9400154A934208D1049B184A1340114A19004C
:103BA4001000FFF7B1FB39E0009B1B68114A9342F8
:103BB40008D1049B124A13400A4A19001000FFF767
:103BC400A3FB2BE0009B1B680B4A934226D1049B6A
:103BD4000C4A1340034A19001000FFF795FB1DE03F
:103BE4000400008008270140001000B0AC00002051
:103BF400400D0300004000B8002000B4FFFF7FFF29
:103C0400FFFFFFFEFFFFBFFF019B9B6D20221A43B6
:103C1400019B9A6517236B4401221A70019B54225D
:103C24000021995417236B441B78180007B000BD7A
:103C340000B585B00190019B1B6818000DF0B3F925
:103C4400031E49D1019B1B689B68254A13400DD074
:103C5400019B9B6D10221A43019B9A65019BDB6DAE
:103C640001221A43019BDA65012336E0019B1B689C
:103C74001800FFF781FB019B5B7E012B2CD0FFF723
:103C84001DFB0300039320E0019B1B6818000DF04B
:103C94008AF9031E04D1019B1B681800FFF76CFB13
:103CA400FFF70CFB0200039BD31A022B0DD9019BD7
:103CB4009B6D10221A43019B9A65019BDB6D0122C7
:103CC4001A43019BDA65012307E0019B1B681B680B
:103CD40001221340012BD7D10023180005B000BDE9
:043CE4001700008045
:103CE80000B585B00190019B9B6A0393039B9B6D74
:103CF8005022134041D1039B9B6D802292001A43AE
:103D0800039B9A65039B1B6818000DF02EF9031E90
:103D18002ED0039B9B7E002B2AD1039B1B681B681C
:103D280008221340082B23D1039B1B6818000DF0B1
:103D380054F9031E10D1039B1B685A68039B1B6828
:103D48000C218A435A60039B9B6D154A134001223C
:103D58001A43039B9A650BE0039B9B6D20221A4331
:103D6800039B9A65039BDB6D01221A43039BDA656B
:103D7800039B180008F00AFA0FE0039B9B6D1022C2
:103D8800134004D0039B18000CF075FC05E0039B5E
:103D98001B6D5B6B019A10009847C04605B000BDCB
:043DA800FEFEFFFF1D
:103DAC0010B586B0019000230393019B54229B5CB9
:103DBC00012B01D102236CE0019B54220121995467
:103DCC0017246C44019B18000DF013F903002370A9
:103DDC00019B1B6818000DF062F9031E4CD1019B6E
:103DEC009B6D2D4A134002221A43019B9A65019B3D
:103DFC001B68DB68032213400493019B1B68DA6881
:103E0C00019B1B6803218A43DA60019B1B689A683B
:103E1C00019B1B68802109060A439A6014E0039BEE
:103E2C0001330393039B1D4A93420DD9019B9B6D58
:103E3C001222934310221A43019B9A65019B542230
:103E4C0000219954012324E0019B1B6818000DF0FC
:103E5C0034F9031EE3D1019B1B68D968019B1B68D5
:103E6C00049A0A43DA60019B9B6D0322934301225F
:103E7C001A43019B9A6505E0019B9B6D10221A4326
:103E8C00019B9A65019B54220021995417236B4482
:103E9C001B78180006B010BDFDFEFFFFFFF10200FD
:103EAC0082B002006B4607331A706B4607331B78DF
:103EBC001A001F231A40044B012191400A001A607A
:0C3ECC00C04602B07047C04600E100E0B4
:103ED80082B002006B4607331A706B4607331B78B3
:103EE8001A001F231340044901229A40130080221C
:0C3EF8008B50C04602B0704700E100E0B3
:103F040010B582B0020000916B4607331A706B46FD
:103F140007331B787F2B36D9324A6B4607331B781D
:103F240019000F230B40083B9B0806339B00D31852
:103F340004331B686A4607321278110003220A40D0
:103F4400D200FF2191400A00D2431A401100009B85
:103F54009B01FF221A406B4607331B78180003238A
:103F64000340DB009A401F486B4607331B781C0054
:103F74000F232340083B9B080A4306339B00C318C6
:103F840004331A602BE0184A6B4607331B785BB284
:103F94009B08C0339B009B586A4607321278110075
:103FA40003220A40D200FF2191400A00D2431A4062
:103FB4001100009B9B01FF221A406B4607331B78BC
:103FC400180003230340DB009A4007486B4607337D
:103FD4001B785BB29B080A43C0339B001A50C0464F
:0C3FE40002B010BD00ED00E000E100E0C4
:103FF00000B583B00190019B5A1E80235B049A4256
:1040000001D3012310E00A4B019A013A5A600123BF
:104010005B4203211800FFF775FF054B00229A60F1
:10402000034B07221A600023180003B000BDC046EE
:0440300010E000E0BC
:1040340000B583B00190019B002B01D1012377E0EF
:10404400019B1B683C4A94466344142118000AF0FF
:104054006DFD03009A00019B1A64019B2522022135
:104064009954019B1B681A68019B1B6833490A40D9
:104074001A60019B1B681968019B9A68019BDB68A5
:104084001A43019B1B691A43019B5B691A43019BF9
:104094009B691A43019BDB691A43019B1B6A1A4300
:1040A400019B1B680A431A60019B180000F034F955
:1040B400019B9A688023DB019A4202D1019B002272
:1040C4005A60019B5A68019B5B6CFF210A401A608D
:1040D400019B9B6C019AD26C5A60019B5B68002B1C
:1040E40011D0019B5B68042B0DD8019B180000F0D4
:1040F4003DF9019B1B6D00221A60019B5B6D019AC7
:10410400926D5A6008E0019B00221A65019B00220F
:104114005A65019B00229A65019B0022DA63019B88
:10412400252201219954019B242200219954002322
:10413400180003B000BDC046F8FFFDBF0F80FFFFAD
:1041440000B585B00190554B1B680393019B1B6818
:104154001B680293019B1B6C1C22134004229A408F
:104164001300039A134027D0029B0422134023D048
:10417400019B1B681B682022134007D1019B1B680D
:104184001A68019B1B6804218A431A60434B5968CF
:10419400019B1B6C1C22134004229A403F4B0A4390
:1041A4005A60019B1B6B002B00D173E0019B1B6BBE
:1041B400019A100098476DE0019B1B6C1C22134070
:1041C40002229A401300039A13402ED0029B02222B
:1041D40013402AD0019B1B681B68202213400BD17B
:1041E400019B1B681A68019B1B680A218A431A6099
:1041F400019B252201219954284B5968019B1B6C72
:104204001C22134002229A40244B0A435A60019B09
:10421400242200219954019BDB6A002B3AD0019B94
:10422400DB6A019A1000984734E0019B1B6C1C2246
:10423400134008229A401300039A13402BD0029B88
:104244000822134027D0019B1B681A68019B1B6836
:104254000E218A431A60114B5968019B1B6C1C2266
:10426400134001229A400D4B0A435A60019B0122DC
:10427400DA63019B252201219954019B2422002108
:104284009954019B5B6B002B05D0019B5B6B019ADE
:1042940010009847C046C04605B000BD000002406B
:1042A40084B00390029101920093039B9B6C039A48
:1042B400D26C5A60039B1B6D002B04D0039B5B6D77
:1042C400039A926D5A60134B5968039B1B6C1C2212
:1042D400134001229A400F4B0A435A60039B1B6808
:1042E400009A5A60039B9B68102B08D1039B1B68A0
:1042F400019A9A60039B1B68029ADA6007E0039BA9
:104304001B68029A9A60039B1B68019ADA60C04694
:0843140004B0704700000240F4
:10431C0000B585B00190019B1B681A00FF23134068
:10432C00083B142118000AF0FDFB03000393019BCA
:10433C001B6C9B08094A944663449B001A00019B22
:10434C005A64019B064A9A64039B1C221340012267
:10435C009A40019BDA64C04605B000BD0082001093
:04436C008008024083
:1043700084B00190019B5B68FF2213400393039B71
:104380000A4A944663449B001A00019B1A65019BEC
:10439000074A5A65039B013B0322134001229A40BE
:1043A000019B9A65C04604B07047C0463F8200102A
:0443B000400902407E
:1043B40010B586B00390029100920193204B1B78B4
:1043C400012B01D1022337E01D4B01221A701C4B33
:1043D40000225A6017246C441A4B180000F0C4F8E9
:1043E4000300237017236B441B78002B1ED1039BFF
:1043F400012B06D1009A019B0299080000F01CF9D8
:1044040005E0009A029B1100180000F01FF8172421
:104414006C440C4B180000F0A7F8030023700A4BFF
:104424005A69039BD943084B0A405A61044B002242
:104434001A7017236B441B78180006B010BDC046D1
:10444400800B0020881300000020024008B4024BB7
:0C4454009C4608BC6047C04601000020E8
:1044600082B06B46073300221A700C4B5B69002B3D
:104470000DDA0A4B0A4A9A60084B0A4A9A60074BBF
:104480005B69002B03DA6B46073301221A706B4617
:1044900007331B78180002B07047C0460020024066
:0844A00023016745AB89EFCD54
:1044A80082B06B46073301221A700A4B5A69094BCE
:1044B800802109060A435A61064B5B69002B03DA1F
:1044C8006B46073300221A706B4607331B781800B7
:0844D80002B070470020024011
:1044E00082B06B46073301221A700E4B5A69802343
:1044F000DB0513400FD00B4B0B4ADA60094B0B4A1C
:10450000DA60084B5A698023DB05134003D16B4600
:10451000073300221A706B4607331B78180002B06D
:104520007047C046002002403B2A19087F6E5D4C50
:1045300082B06B46073301221A700B4B5A690A4B43
:104540008021C9050A435A61074B5A698023DB055C
:10455000134003D06B46073300221A706B460733B3
:0C4560001B78180002B0704700200240D9
:10456C0000B585B00190FEF7A5FE0200019B9B18DB
:10457C00039307E0FEF79EFE0200039B934201D8D3
:10458C0003234BE0274B1A6980235B021A408023DC
:10459C005B029A42EED0234B1B69234A13400293D1
:1045AC00204B9A698023DB051340029A1343029334
:1045BC00029B9B0F9B0707D01A4B9969029B9B0F81
:1045CC009A07184B0A439A61029B9B009B0804D0E4
:1045DC00144B029A920092081A61029B002B04D091
:1045EC00124B029A5A60012318E0FEF763FE020098
:1045FC00019B9B18039307E0FEF75CFE0200039BF4
:10460C00934201D8032309E0064B1A698023DB028D
:10461C001A408023DB029A42EED00023180005B02A
:10462C0000BDC04600200240FA830000800B002031
:10463C0030B585B00390009201930B4B5A690A4B2D
:10464C0001210A435A61039B009A1A60BFF36F8FD2
:10465C00C046019B1C0000231D00039B0433220059
:0C466C001A60C04605B030BD00200240BE
:1046780010B584B0019000912F4B1B78012B01D10C
:10468800022355E02C4B01221A702B4B00225A6052
:104698000F246C44294B1800FFF764FF03002370B4
:1046A8000F236B441B78002B3CD1019B1B68042B08
:1046B8000AD100F0EBF80F246C44204B1800FFF7E8
:1046C80051FF030023702DE0009B012252421A6023
:1046D800019B5B68029317E0029B180000F0E2F868
:1046E8000F246C44154B1800FFF73CFF03002370A0
:1046F8000F236B441B78002B03D0009B029A1A608F
:104708000AE0029B01330293019B5A68019B9B6854
:10471800D318029A9A42DFD3094B5A69084B0221EF
:104728008A435A61044B00221A700F236B441B788A
:10473800180004B010BDC046800B0020881300008C
:04474800002002400B
:10474C0010B584B001903B4B1B78012B01D1022397
:10475C006DE0384B01221A70364B00225A60019BD7
:10476C001B680122134008D0019B5868019B996873
:10477C00019BDB681A0000F0ABF8019B1B6806225A
:10478C001340062B09D1019B5869019B9969019B28
:10479C001B691A0000F0B6F821E0019B1B6802228D
:1047AC0013400BD000F006F903000293019B1A6929
:1047BC000299029B180000F0A5F810E0019B1B6801
:1047CC00042213400BD000F0E1F803000293019B8C
:1047DC005869019B9B69029A190000F093F80F2409
:1047EC006C44154B1800FFF7BBFE030023700F231E
:1047FC006B441B78002B14D1104B5A690F4B802142
:10480C0089020A435A610F246C440B4B1800FFF7C2
:10481C00A7FE03002370094B5A69084B08490A404C
:10482C005A61044B00221A700F236B441B7818003A
:10483C0004B010BD800B0020881300000020024043
:04484C00FFFFFDFF6E
:1048500000B583B00190019B07221A60019B586844
:10486000019B08331900019B0C331A0000F06CF80F
:1048700000F092F80200019B1A6100F0A1F802001A
:10488000019B9A61019B024A5A61C04603B000BD78
:0448900000604F076E
:10489400034B5A69024B03490A435A61C0467047A5
:0848A4000020024004000100A5
:1048AC0084B00190074B5B69074A13400393019B4B
:1048BC00DA00039B1A43034B04490A435A61C0466E
:1048CC0004B070470020024007FEFFFF0200010009
:1048DC0084B0039002910192039B012B06D0019BA3
:1048EC001904074B029A0A431A6305E0019B190449
:1048FC00034B029A0A43DA62C04604B07047C046C2
:04490C000020024045
:1049100086B00390029101920A4B1B6A0593039B98
:10492000FF221343DA43059B13400593059A029B2C
:104930001A431100034B019A0A431A62C04606B09B
:084940007047C0460020024050
:1049480084B0039002910192039B012B0DD10F4B70
:10495800DB6A3F221A40029B1A600C4BDB6A1B0C75
:104968003F221A40019B1A600CE0084B1B6B3F2248
:104978001A40029B1A60054B1B6B1B0C3F221A4006
:10498800019B1A60C04604B07047C0460020024030
:1049980082B0084B1B6AFF2213400193019BAA2B8C
:1049A80004D0019BCC2B01D0BB2300E0019B180055
:0849B80002B07047002002402C
:1049C00082B0044B1B6A044A13400193019B1800F8
:0C49D00002B070470020024000604F075A
:1049DC0000B587B0019000910023059347E1009B3F
:1049EC001B680121059A91400A0013400393039B15
:1049FC00002B00D138E1009B5B68022B03D0009B9D
:104A0C005B68122B23D1059BDA08019B08329200BC
:104A1C00D3580493059B072213409B000F229A4006
:104A2C001300DA43049B13400493009B1A69059B03
:104A3C0007210B409B009A401300049A13430493E4
:104A4C00059BDA08019B083292000499D150019B16
:104A5C001B680493059B5B0003229A401300DA4306
:104A6C00049B13400493009B5B6803221A40059B34
:104A7C005B009A401300049A13430493019B049A1D
:104A8C001A60009B5B68012B0BD0009B5B68022BB0
:104A9C0007D0009B5B68112B03D0009B5B68122B2B
:104AAC0030D1019B9B680493059B5B0003229A40C9
:104ABC001300DA43049B13400493009BDA68059BB4
:104ACC005B009A401300049A13430493019B049ACD
:104ADC009A60019B5B6804930122059B9A4013002A
:104AEC00DA43049B13400493009B5B681B0901226F
:104AFC001A40059B9A401300049A13430493019B9C
:104B0C00049A5A60019BDB680493059B5B000322AB
:104B1C009A401300DA43049B13400493009B9A6859
:104B2C00059B5B009A401300049A13430493019B6A
:104B3C00049ADA60009B5A6880235B05134000D10D
:104B4C0092E0504A059B9B0818339B009B5804939A
:104B5C00059B03221340DB000F229A401300DA431B
:104B6C00049B13400493019AA023DB059A4213D0B3
:104B7C00019B454A93420DD0019B444A934207D076
:104B8C00019B434A934201D1032306E0052304E031
:104B9C00022302E0012300E00023059A03210A40CE
:104BAC00D2009340049A134304933649059B9B0807
:104BBC0018339B00049A5A50324A8023D3580493DA
:104BCC00039BDA43049B13400493009B5A68802395
:104BDC005B02134003D0049A039B134304932949AB
:104BEC008022049B8B50274A8423D3580493039B25
:104BFC00DA43049B13400493009B5A6880239B0266
:104C0C00134003D0049A039B134304931D4984223D
:104C1C00049B8B501B4B1B680493039BDA43049B34
:104C2C0013400493009B5A6880235B03134003D00A
:104C3C00049A039B13430493124B049A1A60114B6E
:104C4C005B680493039BDA43049B13400493009B1F
:104C5C005A6880239B03134003D0049A039B13438D
:104C6C000493084B049A5A60059B01330593009BEF
:104C7C001A68059BDA40131E00D0B0E6C046C04649
:104C8C0007B000BD0018024000040050000800509E
:044C9C00000C0050B8
:104CA00000B583B002006B4606331A80134BDB68F5
:104CB0006A460632128813400AD0104B6A46063202
:104CC0001288DA606B4606331B8818000CF05BFA1A
:104CD0000A4B1B696A460632128813400AD0074BFA
:104CE0006A46063212881A616B4606331B88180022
:104CF0000CF0CDFCC04603B000BDC0460018024019
:104D0000044B1A68034B802149000A431A60C046CD
:084D10007047C046007000402E
:104D1800034B1A68024B03490A401A60C0467047A1
:084D280000700040FFFEFFFFD8
:104D300000B585B00190194B1B68194A1340190042
:104D4000164B019A0A431A60019A80239B009A42EB
:104D50001FD1144B1A6813005B009B185B001249AB
:104D6000180009F0E5FE03000133039308E0039BFC
:104D7000002B03D0039B013B039301E0032309E0D5
:104D8000064B5A698023DB001A408023DB009A42DD
:104D9000EDD00023180005B000BDC04600700040F3
:0C4DA000FFF9FFFFAC00002040420F00B4
:104DAC00034B9A68E023DB01134018007047C046A0
:044DBC0000100240A1
:104DC00000B589B00190019B002B01D10123FAE2CB
:104DD000019B1B680122134000D17CE0C34B9B6800
:104DE000382213400693C14BDB680322134005931E
:104DF000069B102B02D1059B032B02D0069B082B90
:104E00000BD1BA4B1A6880239B02134062D0019BDE
:104E10005B68002B5ED10123D5E2019B5A68802399
:104E20005B029A4207D1B14B1A68B04B802149020C
:104E30000A431A6020E0019B5A68A023DB029A42D1
:104E40000ED1AA4B1A68A94B8021C9020A431A60E5
:104E5000A64B1A68A54B802149020A431A600BE051
:104E6000A24B1A68A14BA2490A401A609F4B1A68CC
:104E70009E4BA0490A401A60019B5B68002B14D02E
:104E8000FEF71EFA0300049308E0FEF719FA020089
:104E9000049BD31A642B01D9032394E2934B1A6821
:104EA00080239B021340F0D015E0FEF709FA0300BF
:104EB000049308E0FEF704FA0200049BD31A642B63
:104EC00001D903237FE2894B1A6880239B02134098
:104ED000F0D100E0C046019B1B680222134000D1C4
:104EE00099E0824B9B683822134006937F4BDB6826
:104EF000032213400593069B102B02D1059B022B26
:104F000002D0069B002B35D1784B1A688023DB003A
:104F1000134005D0019BDB68002B01D1012352E235
:104F2000724B5B68744A13401900019B5B691A025B
:104F30006E4B0A435A60069B002B12D16B4B1B68C9
:104F40006E4A13401900019B1A69684B0A431A60A4
:104F5000664B1B68DB0A07221340694ADA40694B3B
:104F60001A60694B1B681800FEF754F9031E51D0F4
:104F7000012328E2019BDB68002B30D05B4B1B68D0
:104F80005E4A13401900019B1A69584B0A431A6084
:104F9000564B1A68554B802149000A431A60FEF7A8
:104FA0008FF90300049308E0FEF78AF90200049BDE
:104FB000D31A022B01D9032305E24C4B1A68802334
:104FC000DB001340F0D0494B5B684B4A134019009B
:104FD000019B5B691A02454B0A435A601BE0434B35
:104FE0001A68424B49490A401A60FEF769F9030002
:104FF000049308E0FEF764F90200049BD31A022B25
:1050000001D90323DFE1394B1A688023DB00134009
:10501000F0D100E0C046019B1B680822134047D036
:10502000324B9B6838221340182B0AD12F4B1B6E32
:10503000022213403CD0019B9B69002B38D10123F5
:10504000C1E1019B9B69002B19D0284B1A6E274B9D
:1050500001210A431A66FEF733F90300049308E0BE
:10506000FEF72EF90200049BD31A022B01D9032369
:10507000A9E11E4B1B6E02221340F1D018E01B4B1E
:105080001A6E1A4B01218A431A66FEF719F90300BA
:10509000049308E0FEF714F90200049BD31A022BD4
:1050A00001D903238FE1114B1B6E02221340F1D172
:1050B000019B1B680422134000D1C7E01F236B44EF
:1050C00000221A70094B9B6838221340202B1FD1F5
:1050D000064BDB6D0222134000D1B7E0019B9B68B9
:1050E000002B00D0B2E001236DE1C0460010024069
:1050F000FFFFFEFFFFFFFBFFFF80FFFFFFC7FFFF7C
:105100000024F400AC00002098000020FFFEFFFF08
:10511000AE4BDA6B80235B05134001D1012300E025
:105120000023002B11D0A94BDA6BA84B8021490535
:105130000A43DA63A54BDA6B80235B0513400393C4
:10514000039B1F236B4401221A70A14B1A68802312
:105150005B0013401AD19E4B1A689D4B8021490079
:105160000A431A60FEF7ACF80300049308E0FEF768
:10517000A7F80200049BD31A022B01D9032322E1D2
:10518000934B1A6880235B001340F0D0019B9B680F
:10519000012B06D18D4BDA6D8C4B01210A43DA6568
:1051A0001CE0019B9B68052B0CD1884BDA6D874B6B
:1051B00004210A43DA65854BDA6D844B01210A43E9
:1051C000DA650BE0814BDA6D804B01218A43DA65A9
:1051D0007E4BDA6D7D4B04218A43DA65019B9B6827
:1051E000002B14D0FEF76CF80300049309E0FEF7DF
:1051F00067F80200049BD31A764A934201D903232D
:10520000E1E0724BDB6D02221340F0D013E0FEF7B9
:1052100057F80300049309E0FEF752F80200049BDC
:10522000D31A6C4A934201D90323CCE0674BDB6D60
:1052300002221340F0D11F236B441B78012B05D1B0
:10524000624BDA6B614B64490A40DA63019BDB69AC
:10525000002B00D1B6E05D4B9B6838221340102B29
:1052600000D17EE0019BDB69022B53D1574B1A68BA
:10527000564B5A490A401A60FEF722F8030004937D
:1052800008E0FEF71DF80200049BD31A022B01D997
:10529000032398E04D4B1A6880239B041340F0D100
:1052A0004A4BDB684E4A13401900019B1A6A019B66
:1052B0005B6A1A43019B9B6A1B021A43019BDB6AD0
:1052C0001A43019B1B6B1A43404B0A43DA603F4B66
:1052D0001A683E4B802149040A431A603B4BDA6846
:1052E0003A4B802149050A43DA60FDF7E9FF0300E4
:1052F000049308E0FDF7E4FF0200049BD31A022B9D
:1053000001D903235FE0314B1A6880239B041340CB
:10531000F0D057E02D4B1A682C4B30490A401A60E8
:105320002A4BDA68294B03218A43DA60274BDA6873
:10533000264B2C490A40DA60FDF7C2FF03000493B4
:1053400008E0FDF7BDFF0200049BD31A022B01D930
:10535000032338E01D4B1A6880239B041340F0D1CF
:1053600030E0019BDB69012B01D101232BE0174BBE
:10537000DB680593059B03221A40019B1B6A9A4236
:105380001ED1059B70221A40019B5B6A9A4217D17D
:10539000059AFE23DB011A40019B9B6A1B029A427D
:1053A0000ED1059AF8239B031A40019BDB6A9A42AF
:1053B00006D1059B5B0F5A07019B1B6B9A4201D0DC
:1053C000012300E00023180009B000BD00100240D6
:1053D0000070004088130000FFFFFFEFFFFFFFFE9B
:0853E0008C80C11FFFFFFEEFEE
:1053E80000B585B001900091019B002B01D10123EC
:1053F800E9E0764B1B6807221340009A9A421ED9AF
:10540800724B1B68072293431900704B009A0A439A
:105418001A60FDF751FF0300039309E0FDF74CFF05
:105428000200039BD31A6A4A934201D90323CAE0B4
:10543800664B1B6807221340009A9A42EED1019BE3
:105448001B680222134015D0019B1B6804221340DD
:1054580006D0604B9A685F4BE021C9010A439A6005
:105468005C4B9B685C4A13401900019B9A68594B36
:105478000A439A60019B1B680122134057D0019B85
:105488005B68012B07D1534B1A6880239B0213409A
:105498002BD1012397E0019B5B68022B07D14D4B71
:1054A8001A6880239B0413401FD101238BE0019BC2
:1054B8005B68002B07D1474B1A688023DB00134039
:1054C80013D101237FE0019B5B68032B06D1414B7D
:1054D8001B6E0222134008D1012374E03D4BDB6DA3
:1054E8000222134001D101236DE03A4B9B68072249
:1054F80093431900019B5A68364B0A439A60FDF79B
:10550800DBFE0300039309E0FDF7D6FE0200039BD0
:10551800D31A2F4A934201D9032354E02D4B9B6899
:1055280038221A40019B5B68DB009A42ECD1274B7A
:105538001B6807221340009A9A421ED2234B1B680D
:10554800072293431900214B009A0A431A60FDF77A
:10555800B3FE0300039309E0FDF7AEFE0200039BD0
:10556800D31A1B4A934201D903232CE0174B1B681B
:1055780007221340009A9A42EED1019B1B6804222D
:10558800134009D0134B9B68144A13401900019B20
:10559800DA68104B0A439A6000F028F801000D4BB6
:1055A8009B681B0A0F221A400D4B9200D3581F22EA
:1055B80013400A00DA400B4B1A600B4B1B681800AB
:1055C800FDF724FE0300180005B000BD00200240CE
:1055D8008813000000100240FFF0FFFFFF8FFFFF5D
:0C55E8005CFC0008AC00002098000020D3
:1055F40000B587B03B4B9B68382213400FD1394B21
:105604001B68DB0A0722134001229A40130000930F
:105614000099354809F08AFA030004935DE0314BA0
:105624009B6838221340082B02D1304B049354E07A
:105634002C4B9B6838221340102B38D1294BDB6844
:10564400032213400393274BDB681B0907221340F3
:1056540001330293039B032B0DD10299234809F0D4
:1056640065FA030019001F4BDB681B0A7F221340F5
:105674004B4305930DE002991B4809F057FA0300C8
:105684001900184BDB681B0A7F2213404B43059318
:10569400C046144BDB685B0F0722134001330193B0
:1056A4000199059809F042FA0300049315E00D4BA3
:1056B4009B6838221340202B03D180231B020493C0
:1056C4000BE0084B9B6838221340182B03D1FA23B4
:1056D400DB01049301E000230493049B180007B04A
:1056E40000BDC046001002400024F40000127A00FD
:0C56F400014B1B6818007047AC00002040
:1057000010B5FFF7F7FF0400FFF750FB03001A0B7B
:10571000044B9200D3581F221340DC402300180092
:0857200010BDC0469CFC00080E
:1057280000B587B0019013236B4400221A7012232E
:105738006B4400221A70019B1A6880239B02134055
:1057480000D1A4E011236B4400221A70864BDA6B57
:1057580080235B05134011D1834BDA6B824B802188
:1057680049050A43DA63804BDA6B80235B051340F3
:105778000293029B11236B4401221A707B4B1A6817
:105788007A4B802149000A431A60FDF795FD030012
:1057980003930BE0FDF790FD0200039BD31A022B45
:1057A80004D913236B4403221A7005E06F4B1A685F
:1057B80080235B001340EDD013236B441B78002B30
:1057C80054D1694BDA6DC0239B0013400593059BA8
:1057D800002B19D0019B9B69059A9A4214D0624B01
:1057E800DB6D634A134005935F4BDA6D5E4B802196
:1057F80049020A43DA655C4BDA6D5B4B5D490A4046
:10580800DA65594B059ADA65059B0122134016D0D3
:10581800FDF752FD030003930CE0FDF74DFD020078
:10582800039BD31A544A934204D913236B4403228B
:105838001A7004E04C4BDB6D02221340EDD01323A9
:105848006B441B78002B0AD1474BDB6D484A134049
:105858001900019B9A69444B0A43DA650CE012234C
:105868006B4413226A4412781A7005E012236B44C1
:1058780013226A4412781A7011236B441B78012B87
:1058880005D1394BDA6B384B3C490A40DA63019B46
:105898001B680122134009D0334B5B6D03229343ED
:1058A8001900019B5A68304B0A435A65019B1B68D3
:1058B8000222134009D02C4B5B6D0C229343190034
:1058C800019B9A68284B0A435A65019B1B68402232
:1058D800134009D0244B5B6D294A13401900019BE2
:1058E800DA68214B0A435A65019B1A688023DB0159
:1058F800134015D01C4B5B6D9B009908019B5A699E
:10590800194B0A435A65019B5A698023DB059A4261
:1059180006D1154BDA68144B802149020A43DA6034
:10592800019B1A6880231B01134016D00E4B5B6D38
:10593800144A13401900019B1A690B4B0A435A6514
:10594800019B1A698023DB019A4206D1064BDA686B
:10595800054B802149020A43DA6012236B441B7805
:10596800180007B000BDC04600100240007000409B
:10597800FFFCFFFFFFFFFEFF88130000FFFFFFEFA4
:08598800FFCFFFFFFF3FFFFF0F
:1059900010B584B001900F236B4401221A70019B53
:1059A000002B00D181E0019B29229B5CDBB2002B04
:1059B0000BD1019B282200219954019B88221202BD
:1059C0005A60019B180007F069F8019B2922022107
:1059D0009954019B1B68CA225A62019B1B6853227F
:1059E0005A620F246C44019B18000BF0D4FB030097
:1059F00023700F236B441B78002B49D1019B1B683C
:105A00009A69019B1B682C490A409A61019B1B689B
:105A10009969019B9A68019B5B691A43019BDB6949
:105A20001A43019B1B680A439A61019B1B68019AF8
:105A300012691A61019B1B681969019BDB681A04D2
:105A4000019B1B680A431A610F246C44019B1800D8
:105A500000F06EF9030023700F236B441B78002BBA
:105A600016D1019B1B689A69019B1B68D200D20862
:105A70009A61019B1B689969019B5A6A019B1B6A89
:105A80001A43019B9B691A43019B1B680A439A6155
:105A9000019B1B68FF225A620F236B441B78002B6B
:105AA00003D1019B2922012199540F236B441B78B8
:0C5AB000180004B010BDC046BFFF8FFB03
:105ABC0010B586B0039002910192039B28229B5C47
:105ACC00012B01D1022393E0039B2822012199543D
:105ADC00039B292202219954039B1B68CA225A62F8
:105AEC00039B1B6853225A6213246C44039B1800BB
:105AFC000BF04BFB0300237013236B441B78002B20
:105B0C0062D1019B002B25D1039B1B689B69402212
:105B1C00134002D1029B0022DA70029B1B78180002
:105B2C000AF0C1FE03001C04029B5B7818000AF00B
:105B3C00BAFE03001B021C43029B9B7818000AF060
:105B4C00B2FE030022001A43029BDB789B05134331
:105B5C00059317E0039B1B689B694022134002D1FD
:105B6C00029B0022DA70029B1B781A04029B5B7862
:105B7C001B021343029A92781A43029BDB789B0513
:105B8C0013430593039B1B68059A1B490A401A6033
:105B9C00039B1B689A69039B1B6818490A409A610E
:105BAC00039B1B689969029BDA68029B1B691A4369
:105BBC00039B1B680A439A6113246C44039B1800D3
:105BCC0000F0B0F803002370039B1B68FF225A629D
:105BDC0013236B441B78002B03D1039B2922012137
:105BEC009954039B28220021995413236B441B784E
:105BFC00180006B010BDC0467F7F7F00FFFFFBFF83
:105C0C0010B586B0039002910192039B28229B5CF5
:105C1C00012B01D102237FE0039B282201219954FF
:105C2C00039B292202219954019B002B0ED1029B2C
:105C3C005B781A001023134008D0029B5B7810226B
:105C4C009343DBB20A33DAB2029B5A70019B002BEE
:105C5C001CD1029BDB7818000AF025FE03001C0403
:105C6C00029B5B7818000AF01EFE03001B021C430B
:105C7C00029B9B7818000AF016FE030022001A43C0
:105C8C00029B1B785B03134305930EE0029BDB78AE
:105C9C001A04029B5B781B021343029A92781A43F4
:105CAC00029B1B785B0313430593039B1B68CA225F
:105CBC005A62039B1B6853225A6213246C44039B45
:105CCC0018000BF062FA0300237013236B441B784B
:105CDC00002B0DD1039B1B68059A11490A405A6091
:105CEC0013246C44039B180000F01CF80300237071
:105CFC00039B1B68FF225A6213236B441B78002BF7
:105D0C0003D1039B292201219954039B28220021B2
:105D1C00995413236B441B78180006B010BDC04671
:045D2C003FFFFF0036
:105D300000B585B001900F236B4400221A701D4BF3
:105D4000DA681C4B80218A43DA601A4B9B69202257
:105D500013400ED1019B18000AF086FD031E22D0CD
:105D6000019B2922032199540F236B4403221A70AB
:105D700019E0104B9A690F4B20218A439A61019BCD
:105D800018000AF071FD031E07D0019B2922032190
:105D900099540F236B4403221A70064B9A69054BE2
:105DA00020210A439A610F236B441B78180005B029
:085DB00000BDC04600280040C0
:105DB80000B585B00190019B002B01D101238AE039
:105DC800019B00229A62019B5D229B5CDBB2002B47
:105DD80007D1019B5C2200219954019B180007F010
:105DE80005F8019B5D2202219954019B1B681A68E2
:105DF800019B1B6840218A431A60019BDA68E023F3
:105E0800DB009A4202D90023039302E080235B015E
:105E18000393019BDA68F0231B019A4208D0019B87
:105E2800DA68E023DB009A4202D0019B00229A62E2
:105E3800019B1B6B002B0CD1019BDA68E023DB0074
:105E48009A4203D9019B02221A6302E0019B0122B4
:105E58001A63019B5A68019B9B681A43019B1B6943
:105E68001A43019B5B691A43019B996980239B0034
:105E78000B401A43019BDB691A43019B1B6A1A43B7
:105E88001100019B9A6A019B1B680A431A60019BD7
:105E98009B691B0C04221A40019B5B6A1A43019BF5
:105EA8005B6B1A43019BDB681A431100019B1B685B
:105EB800039A0A435A60019B1B68DA69019B1B68B5
:105EC80006490A40DA61019B00221A66019B5D229D
:105ED800012199540023180005B000BDFFF7FFFF0A
:105EE80000B58BB00390029101921A006B46023301
:105EF8001A800123099323236B4400221A70039B01
:105F08005C229B5C012B01D1022325E2039B5C22CE
:105F180001219954FDF7D0F9030007931B236B4423
:105F2800039A5D21525C1A70039B5B6805931223E8
:105F38006B446A46023212881A8004AB6A460232FF
:105F480012881A801B236B441B78012B12D0059AE8
:105F580082235B009A4208D1039B9B68002B04D1E3
:105F68001B236B441B78042B04D023236B4402228D
:105F78001A70E6E1029B002B07D0019B002B04D08E
:105F88006B4602331B88002B04D123236B44012268
:105F98001A70D6E1039B5D229B5CDBB2042B03D015
:105FA800039B5D2205219954039B00221A66039BDB
:105FB800019A1A64039B6A460232462112885A5291
:105FC800039B6A460232442112885A52039B029A62
:105FD8009A63039B6A4602321288DA87039B6A46F1
:105FE800023212889A87039B0022DA64039B0022FC
:105FF8001A65039BDA68E023DB009A4203D804ABF6
:106008001B88012B08D9039B1B685A68039B1B68D4
:10601800CA490A405A6008E0039B1B685A68039BF8
:106028001B68802149010A435A60039B1B681B684F
:1060380040221340402B07D0039B1B681A68039B20
:106048001B6840210A431A60039BDA68E023DB00DF
:106058009A4200D87FE0039B5B68002B05D012238F
:106068006B441B88012B00D069E0039B9B6B1A884B
:10607800039B1B68DA60039B9B6B9A1C039B9A63C8
:10608800039BDB8F9BB2013B9AB2039BDA8756E0F6
:10609800039B1B689B6802221340022B1BD1039BA6
:1060A800DB8F9BB2002B16D0099B012B13D1039BCE
:1060B8009B6B1A88039B1B68DA60039B9B6B9A1C7B
:1060C800039B9A63039BDB8F9BB2013B9AB2039BB2
:1060D800DA8700230993039B1B689B6801221340FE
:1060E800012B1CD1039B46229B5A9BB2002B16D036
:1060F800039B1B68DA68039B1B6C92B21A80039B94
:106108001B6C9A1C039B1A64039B46229B5A9BB2E6
:10611800013B99B2039B4622995201230993FDF74B
:10612800CBF80200079BD31A0C9A9A4207D80C9B0B
:10613800013304D023236B4403221A7001E1039B2B
:10614800DB8F9BB2002BA3D1039B46229B5A9BB2A9
:10615800002B9DD1E2E0039B5B68002B05D0122346
:106168006B441B88012B00D0CBE0039BDB8F9BB2D9
:10617800012B12D9039B9B6B1A88039B1B68DA605F
:10618800039B9B6B9A1C039B9A63039BDB8F9BB2BD
:10619800023B9AB2039BDA87B3E0039B9A6B039B9B
:1061A8001B680C3312781A70039B9B6B5A1C039B59
:1061B8009A63039BDB8F9BB2013B9AB2039BDA87FE
:1061C8009FE0039B1B689B6802221340022B34D17B
:1061D800039BDB8F9BB2002B2FD0099B012B2CD16B
:1061E800039BDB8F9BB2012B12D9039B9B6B1A88F5
:1061F800039B1B68DA60039B9B6B9A1C039B9A6347
:10620800039BDB8F9BB2023B9AB2039BDA8712E0B7
:10621800039B9A6B039B1B680C3312781A70039BC1
:106228009B6B5A1C039B9A63039BDB8F9BB2013BBE
:106238009AB2039BDA8700230993039B1B689B6828
:1062480001221340012B49D1039B46229B5A9BB242
:10625800002B43D0039B46229B5A9BB2012B24D987
:10626800039B1B68DA68039B1B6C92B21A80039B22
:106278001B6C9A1C039B1A64039B46229B5A9BB275
:10628800023B99B2039B46229952039B46229B5A92
:106298009BB2012B20D8039B1B685A68039B1B6881
:1062A800802149010A435A6016E0039B1B680C339E
:1062B8001A00039B1B6C1278D2B21A70039B1B6CDA
:1062C8005A1C039B1A64039B46229B5A9BB2013BB0
:1062D80099B2039B4622995201230993FCF7ECFFDC
:1062E8000200079BD31A0C9A9A4202D80C9B0133DE
:1062F80002D10C9B002B04D123236B4403221A7078
:106308001FE0039BDB8F9BB2002B00D059E7039B58
:1063180046229B5A9BB2002B00D052E7079A0C9951
:10632800039B18000AF075FF031E09D023236B4452
:1063380001221A70039B20221A6602E0FFEFFFFF7A
:10634800C046039B5D2201219954039B5C220021D6
:10635800995423236B441B7818000BB000BDC0462A
:1063680000B585B00390029100936B4607331A700D
:1063780050E0009B01334DD0FCF79EFF0200069BC6
:10638800D31A009A9A4202D9009B002B42D1039B50
:106398001B685A68039B1B68E0218A435A60039B69
:1063A8005A6882235B009A4213D1039B9A68802320
:1063B8001B029A4205D0039B9A688023DB009A420D
:1063C80007D1039B1B681A68039B1B6840218A43FB
:1063D8001A60039B9A6A80239B019A4210D1039BFF
:1063E8001B681A68039B1B6814490A401A60039BC0
:1063F8001B681A68039B1B68802189010A431A607D
:10640800039B5D2201219954039B5C22002199542E
:10641800032310E0039B1B689B68029A1340029AAF
:10642800D31A5A425341DBB21A006B4607331B7822
:106438009A429ED10023180005B000BDFFDFFFFF80
:1064480000B585B003900291019200935CE0029A36
:10645800C023DB009A4206D1019B002B03D1039B8A
:106468001B680C331B78009B01334DD0FCF724FFCD
:106478000200069BD31A009A9A4202D9009B002B6D
:1064880042D1039B1B685A68039B1B68E0218A431F
:106498005A60039B5A6882235B009A4213D1039B7C
:1064A8009A6880231B029A4205D0039B9A6880232E
:1064B800DB009A4207D1039B1B681A68039B1B6881
:1064C80040218A431A60039B9A6A80239B019A425F
:1064D80010D1039B1B681A68039B1B6810490A406C
:1064E8001A60039B1B681A68039B1B68802189013B
:1064F8000A431A60039B5D2201219954039B5C2285
:1065080000219954032308E0039B1B689B68029AA7
:106518001340019A9A429AD10023180005B000BD91
:04652800FFDFFFFF93
:10652C0000B583B00190019B3D2202219954019B3F
:10653C001B681B6A104A13400DD1019B1B681B6A18
:10654C000E4A134007D1019B1B681A68019B1B68FC
:10655C0001218A431A60019B18000AF0D2F9019BB1
:10656C003D2200219954019B3C2200219954002387
:10657C00180003B000BDC046111100004404000017
:10658C0000B585B001900091009B0C2B2AD0009B8C
:10659C000C2B30D8009B082B1BD0009B082B2AD827
:1065AC00009B002B03D0009B042B09D023E0019B04
:1065BC001B68DA68019B1B6802210A43DA601BE046
:1065CC00019B1B68DA68019B1B6804210A43DA6093
:1065DC0012E0019B1B68DA68019B1B6808210A43C7
:1065EC00DA6009E0019B1B68DA68019B1B681021CB
:1065FC000A43DA6000E0C046019B1B680099012247
:10660C0018000AF072FE019B1B689B680B4A134032
:10661C000393039B062B0CD0039A80235B029A42B4
:10662C0007D0019B1B681A68019B1B6801210A4358
:10663C001A600023180005B000BDC0460700010019
:10664C0000B583B001900091009B0C2B2AD0009BCD
:10665C000C2B30D8009B082B1BD0009B082B2AD866
:10666C00009B002B03D0009B042B09D023E0019B43
:10667C001B68DA68019B1B6802218A43DA601BE005
:10668C00019B1B68DA68019B1B6804218A43DA6052
:10669C0012E0019B1B68DA68019B1B6808218A4386
:1066AC00DA6009E0019B1B68DA68019B1B6810210A
:1066BC008A43DA6000E0C046019B1B680099002207
:1066CC0018000AF012FE019B1B681B6A0A4A134051
:1066DC000DD1019B1B681B6A084A134007D1019B13
:1066EC001B681A68019B1B6801218A431A600023EE
:1066FC00180003B000BDC046111100004404000096
:10670C0000B583B00190019B1B681B6902221340EA
:10671C00022B24D1019B1B68DB6802221340022B45
:10672C001DD1019B1B68032252421A61019B01225D
:10673C001A77019B1B689B690322134004D0019BB1
:10674C00180001F0E3FE07E0019B18000AF014F9B1
:10675C00019B18000AF015F9019B00221A77019B86
:10676C001B681B6904221340042B25D1019B1B6859
:10677C00DB6804221340042B1ED1019B1B680522ED
:10678C0052421A61019B02221A77019B1B689A697B
:10679C00C0239B00134004D0019B180001F0B6FEEF
:1067AC0007E0019B18000AF0E7F8019B18000AF0BB
:1067BC00E8F8019B00221A77019B1B681B690822D1
:1067CC001340082B24D1019B1B68DB680822134063
:1067DC00082B1DD1019B1B68092252421A61019B97
:1067EC0004221A77019B1B68DB690322134004D037
:1067FC00019B180001F08AFE07E0019B18000AF0CB
:10680C00BBF8019B18000AF0BCF8019B00221A7718
:10681C00019B1B681B6910221340102B25D1019B77
:10682C001B68DB6810221340102B1ED1019B1B68C8
:10683C00112252421A61019B08221A77019B1B6894
:10684C00DA69C0239B00134004D0019B180001F0AF
:10685C005DFE07E0019B18000AF08EF8019B180002
:10686C000AF08FF8019B00221A77019B1B681B69A9
:10687C0001221340012B0FD1019B1B68DB68012205
:10688C001340012B08D1019B1B68022252421A6152
:10689C00019B18000AF06BF8019B1B681B69802296
:1068AC001340802B0FD1019B1B68DB6880221340A7
:1068BC00802B08D1019B1B68812252421A61019BDB
:1068CC0018000AF06DF8019B1B681A6980235B00A5
:1068DC001A4080235B009A420ED1019B1B68DB6837
:1068EC0080221340802B07D1019B1B681B4A1A6125
:1068FC00019B18000AF059F8019B1B681B69402288
:10690C001340402B0FD1019B1B68DB6840221340C6
:10691C00402B08D1019B1B68412252421A61019BFA
:10692C0018000AF033F8019B1B681B6920221340E6
:10693C00202B0FD1019B1B68DB6820221340202BDE
:10694C0008D1019B1B68212252421A61019B18003D
:10695C000AF021F8C04603B000BDC046FFFEFFFFA1
:10696C0000B585B0039002910192039B3C229B5C85
:10697C00012B01D102238AE0039B3C220121995473
:10698C00039B3D2202219954019B002B1BD1039B9D
:10699C001868029B1968029B5A68029BDB6800F01E
:1069AC00EFF8039B1B689A69039B1B680C218A43B5
:1069BC009A61039B1B689969029B9A68039B1B68ED
:1069CC000A439A615AE0019B042B1CD1039B186863
:1069DC00029B1968029B5A68029BDB6800F024F941
:1069EC00039B1B689A69039B1B682A490A409A619E
:1069FC00039B1B689969029B9B681A02039B1B688B
:106A0C000A439A613AE0019B082B1BD1039B18683F
:106A1C00029B1968029B5A68029BDB6800F042F9E2
:106A2C00039B1B68DA69039B1B680C218A43DA61A0
:106A3C00039B1B68D969029B9A68039B1B680A43DA
:106A4C00DA611BE0039B1868029B1968029B5A6869
:106A5C00029BDB6800F064F9039B1B68DA69039BFB
:106A6C001B680C490A40DA61039B1B68D969029BBD
:106A7C009B681A02039B1B680A43DA61039B3D2245
:106A8C0001219954039B3C220021995400231800A6
:086A9C0005B000BDFFF3FFFF90
:106AA40084B001900091019B1B680393019B2F4AC2
:106AB400934203D0019B2E4A934208D1039B702238
:106AC40093430393009B5B68039A13430393019BD3
:106AD400264A934213D0019B254A93420FD0019B2F
:106AE400244A93420BD0019B234A934207D0019B33
:106AF400224A934203D0019B214A934208D1039B2B
:106B0400204A13400393009BDB68039A13430393C7
:106B1400039B802293431A00009B5B6913430393F6
:106B2400019B039A1A60009B9A68019BDA62009B9E
:106B34001A68019B9A62019B0C4A93420BD0019BF9
:106B44000D4A934207D0019B0C4A934203D0019B08
:106B54000B4A934203D1009B1A69019B1A63019B60
:106B640001225A61C04604B07047C046002C01405F
:106B74000004004000200040004001400044014067
:086B840000480140FFFCFFFF87
:106B8C0086B00390029101920093039B1B6A012231
:106B9C0093431A00039B1A62039B9B690593039B07
:106BAC001B6A0493039B1D4A934207D0039B1C4A08
:106BBC00934203D0039B1B4A934201D1012300E073
:106BCC000023002B08D0059B032293430593059AC1
:106BDC00019B1343059303E0059B0122134305938B
:106BEC00059BF02293430593009B1B01FF2213404E
:106BFC00059A13430593049B0A2293430493029B27
:106C0C000A221340049A13430493039B059A9A6136
:106C1C00039B049A1A62C04606B07047002C0140D0
:086C2C0000040040004001409B
:106C340086B00390029101920093039B1B6A102279
:106C440093431A00039B1A62039B9B690593039B5E
:106C54001B6A0493059B134A13400593019B1B0273
:106C6400059A13430593059B0F4A13400593009B14
:106C74001B031B041B0C059A13430593049BA022BE
:106C840093430493029B1B01A0221340049A1343D1
:106C94000493039B059A9A61039B049A1A62C04663
:0C6CA40006B07047FFFCFFFFFF0FFFFF72
:106CB00086B00390029101920093039B1B6A194ACC
:106CC0001A40039B1A62039BDB690593039B1B6AB3
:106CD0000493059B032293430593059A019B134359
:106CE0000593059BF02293430593009B1B01FF2214
:106CF0001340059A13430593049B0B4A13400493D6
:106D0000029B1A02A0231B011340049A134304930D
:106D1000039B059ADA61039B049A1A62C04606B087
:0C6D20007047C046FFFEFFFFFFF5FFFFBD
:106D2C0086B00390029101920093039B1B6A194A4F
:106D3C001A40039B1A62039BDB690593039B1B6A36
:106D4C000493059B144A13400593019B1B02059A5F
:106D5C0013430593059B114A13400593009B1B039A
:106D6C001B041B0C059A13430593049B0C4A1340FC
:106D7C000493029B1A03A0231B021340049A13438F
:106D8C000493039B059ADA61039B049A1A62C0462A
:106D9C0006B07047FFEFFFFFFFFCFFFFFF0FFFFF89
:046DAC00FF5FFFFF87
:106DB00086B003900291019217236B4400221A704F
:106DC000039B3C229B5C012B01D102232EE0039B01
:106DD0003C2201219954019B002B03D0019B042BE1
:106DE0000CD017E0039B1B689B6E0F229343190086
:106DF000039B1B68029A0A439A6610E0039B1B6878
:106E00009B6E0C4A13401900039B1B68029A0A43AD
:106E10009A6604E017236B4401221A70C046039B54
:106E20003C220021995417236B441B78180006B0AC
:086E30007047C046FFF0FFFFB0
:106E380084B0039002916B4606331A80039B80222C
:106E48009B58202B00D082E0029B002B04D06B467D
:106E580006331B88002B01D1012379E0039B9A6834
:106E680080235B019A4209D1039B1B69002B05D142
:106E7800029B0122134001D0012369E0039B7C227D
:106E88009B5C012B01D1022362E0039B7C22012140
:106E98009954039B029A1A65039B6A460632542149
:106EA80012885A52039B6A460632562112885A5251
:106EB800039B00221A67039B882200219950039B99
:106EC800802221219950039B5A6E80239B059A4268
:106ED8001ED1039B9A6880235B019A4207D1039BCA
:106EE8001B69002B03D1039B1B4A1A6702E0039B13
:106EF8001A4A1A67039B7C2200219954039B1B683A
:106F08009A68039B1B68802109040A439A601CE065
:106F1800039B9A6880235B019A4207D1039B1B69F4
:106F2800002B03D1039B0E4A1A6702E0039B0D4A0C
:106F38001A67039B7C2200219954039B1B681A68DB
:106F4800039B1B6880210A431A60002300E0022388
:106F5800180004B07047C0463D7D0008997C0008C1
:086F680037130108D5090108E7
:106F700084B0039002916B4606331A80039B8422EF
:106F80009B58202B00D0DAE0029B002B04D06B46EC
:106F900006331B88002B01D10123D1E0039B9A68A3
:106FA00080235B019A4209D1039B1B69002B05D109
:106FB000029B0122134001D00123C1E0039B7C22EC
:106FC0009B5C012B01D10223BAE0039B7C220121AF
:106FD0009954039B029A9A65039B6A4606325C2188
:106FE00012885A52039B6A4606325E2112885A5210
:106FF000039B0022DA66039B9A6880235B019A4216
:107000000DD1039B1B69002B04D1039B60224E49C9
:1070100099522EE0039B6022FF21995229E0039BA5
:107020009B68002B0DD1039B1B69002B04D1039B94
:107030006022FF2199521CE0039B60227F2199521C
:1070400017E0039B9A6880235B059A420DD1039B4E
:107050001B69002B04D1039B60227F21995208E019
:10706000039B60223F21995203E0039B6022002191
:107070009952039B882200219950039B842222214C
:107080009950039B1B689A68039B1B6801210A4364
:107090009A60039B5A6E80239B059A422FD1039BD3
:1070A00068229B5A6A46063212889A4227D3039B6B
:1070B0009A6880235B019A4207D1039B1B69002BCE
:1070C00003D1039B214ADA6602E0039B204ADA6679
:1070D000039B7C2200219954039B1B681A68039B25
:1070E0001B68802149000A431A60039B1B689A6849
:1070F000039B1B68802149050A439A601DE0039B9E
:107100009A6880235B019A4207D1039B1B69002B7D
:1071100003D1039B0F4ADA6602E0039B0E4ADA664C
:10712000039B7C2200219954039B1B681A68039BD4
:107130001B68902149000A431A60002300E00223E3
:10714000180004B07047C046FF0100008D800008A1
:0C715000597F0008A17E0008E97D0008BE
:10715C0000B589B001900023039313236B440022E4
:10716C001A7000230593019B9A68019B1B691A43B3
:10717C00019B5B691A43019BDB6913430693019BDB
:10718C005B6E069A13430693019B1B681B68B44AFB
:10719C0013401900019B1B68069A0A431A60019B55
:1071AC001B685B68AF4A13401900019BDA68019BAE
:1071BC001B680A435A60019B9B690693019B1B6ADF
:1071CC00069A13430693019B1B689B68A64A1340BF
:1071DC001900019B1B68069A0A439A60019B1B6865
:1071EC00DB6A0F2293431900019B5A6A019B1B68AF
:1071FC000A43DA62019B1B689C4A934227D19C4B41
:10720C005B6D03221340032B17D01BD8022B0AD023
:10721C0018D8002B02D0012B0AD013E01F236B448B
:10722C0000221A7058E01F236B4402221A7053E09C
:10723C001F236B4404221A704EE01F236B44082258
:10724C001A7049E01F236B4410221A7044E0019B12
:10725C001B68884A934227D1854B5B6D0C221340E7
:10726C000C2B17D01BD8082B0AD018D8002B02D007
:10727C00042B0AD013E01F236B4400221A702BE05E
:10728C001F236B4402221A7026E01F236B44042236
:10729C001A7021E01F236B4408221A701CE01F2374
:1072AC006B4410221A7017E0019B1B68724A9342C0
:1072BC0004D11F236B4400221A700DE0019B1B6844
:1072CC006E4A934204D11F236B4400221A7003E0D0
:1072DC001F236B4410221A70019BDA6980231B0256
:1072EC009A4200D0CEE11F236B441B78082B00D1AF
:1072FC003CE100DD99E1042B00D1D6E000DD94E106
:10730C00002B03D0022B00D161E08EE1FEF7F2F9E5
:10731C000200019B5B6A002B44D0019B5B6A012B32
:10732C003ED0019B5B6A022B38D0019B5B6A032B1E
:10733C0032D0019B5B6A042B2CD0019B5B6A052B22
:10734C0026D0019B5B6A062B20D0019B5B6A072B26
:10735C001AD0019B5B6A082B14D0019B5B6A092B2A
:10736C000ED0019B5B6A0A2B08D0019B5B6A0B2B2E
:10737C0002D180235B0016E0012314E0802312E08D
:10738C00402310E020230EE010230CE00C230AE035
:10739C000A2308E0082306E0062304E0042302E0A5
:1073AC00022300E001231900100007F0BBFB0300CF
:1073BC005A00019B5B685B08D218019B5B68190043
:1073CC00100007F0AFFB03009BB2039332E1019B6B
:1073DC005B6A002B54D0019B5B6A012B3ED0019B56
:1073EC005B6A022B38D0019B5B6A032B32D0019B6A
:1073FC005B6A042B2CD0019B5B6A052B26D0019B6E
:10740C005B6A062B20D0019B5B6A072B1AD0019B71
:10741C005B6A082B14D0019B5B6A092B0ED0019B75
:10742C005B6A0A2B08D0019B5B6A0B2B02D1802371
:10743C005B0026E0012324E0802322E0402320E0AF
:10744C0020231EE010231CE00C231AE00A2318E072
:10745C00082316E0062314E0042312E0022310E0B4
:10746C00F369FFCFFFCFFFFFFFF4FF11003801409E
:10747C00001002400044004000480040004C004016
:10748C0001231900B94807F04DFB03005A00019B7A
:10749C005B685B08D218019B5B681900100007F051
:1074AC0041FB03009BB20393C4E0FEF79DF802007E
:1074BC00019B5B6A002B44D0019B5B6A012B3ED085
:1074CC00019B5B6A022B38D0019B5B6A032B32D089
:1074DC00019B5B6A042B2CD0019B5B6A052B26D08D
:1074EC00019B5B6A062B20D0019B5B6A072B1AD091
:1074FC00019B5B6A082B14D0019B5B6A092B0ED095
:10750C00019B5B6A0A2B08D0019B5B6A0B2B02D197
:10751C0080235B0016E0012314E0802312E040235B
:10752C0010E020230EE010230CE00C230AE00A23C9
:10753C0008E0082306E0062304E0042302E002230B
:10754C0000E001231900100007F0ECFA03005A00C8
:10755C00019B5B685B08D218019B5B6819001000EB
:10756C0007F0E0FA03009BB2039363E0019B5B6AB4
:10757C00002B44D0019B5B6A012B3ED0019B5B6AC4
:10758C00022B38D0019B5B6A032B32D0019B5B6AC8
:10759C00042B2CD0019B5B6A052B26D0019B5B6ACC
:1075AC00062B20D0019B5B6A072B1AD0019B5B6AD0
:1075BC00082B14D0019B5B6A092B0ED0019B5B6AD4
:1075CC000A2B08D0019B5B6A0B2B02D180235B003A
:1075DC0016E0012314E0802312E0402310E0202366
:1075EC000EE010230CE00C230AE00A2308E0082329
:1075FC0006E0062304E0042302E0022300E001235A
:10760C0019008023180207F08DFA03005A00019B21
:10761C005B685B08D218019B5B681900100007F0CF
:10762C0081FA03009BB2039304E013236B44012201
:10763C001A70C046039B0F2B1FD9039A80235B0241
:10764C009A421AD2039B9AB20A236B440F218A43A3
:10765C001A80039B5B089BB20722134099B20A2342
:10766C006B440A226A4412880A431A80019B1B68E5
:10767C000A226A441288DA60AEE113236B440122B9
:10768C001A70A9E11F236B441B78082B00D12EE143
:10769C0000DD8BE1042B00D1C8E000DD86E1002B7E
:1076AC0003D0022B00D163E080E1FEF723F8020047
:1076BC00019B5B6A002B44D0019B5B6A012B3ED083
:1076CC00019B5B6A022B38D0019B5B6A032B32D087
:1076DC00019B5B6A042B2CD0019B5B6A052B26D08B
:1076EC00019B5B6A062B20D0019B5B6A072B1AD08F
:1076FC00019B5B6A082B14D0019B5B6A092B0ED093
:10770C00019B5B6A0A2B08D0019B5B6A0B2B02D195
:10771C0080235B0016E0012314E0802312E0402359
:10772C0010E020230EE010230CE00C230AE00A23C7
:10773C0008E0082306E0062304E0042302E0022309
:10774C0000E001231900100007F0ECF903001A0007
:10775C00019B5B685B08D218019B5B6819001000E9
:10776C0007F0E0F903009BB2039324E10024F4003A
:10777C00019B5B6A002B44D0019B5B6A012B3ED0C2
:10778C00019B5B6A022B38D0019B5B6A032B32D0C6
:10779C00019B5B6A042B2CD0019B5B6A052B26D0CA
:1077AC00019B5B6A062B20D0019B5B6A072B1AD0CE
:1077BC00019B5B6A082B14D0019B5B6A092B0ED0D2
:1077CC00019B5B6A0A2B08D0019B5B6A0B2B02D1D5
:1077DC0080235B0016E0012314E0802312E0402399
:1077EC0010E020230EE010230CE00C230AE00A2307
:1077FC0008E0082306E0062304E0042302E0022349
:10780C0000E0012319007E4807F08CF903001A00F0
:10781C00019B5B685B08D218019B5B681900100028
:10782C0007F080F903009BB20393C4E0FDF7DCFE84
:10783C000200019B5B6A002B44D0019B5B6A012B0D
:10784C003ED0019B5B6A022B38D0019B5B6A032BF9
:10785C0032D0019B5B6A042B2CD0019B5B6A052BFD
:10786C0026D0019B5B6A062B20D0019B5B6A072B01
:10787C001AD0019B5B6A082B14D0019B5B6A092B05
:10788C000ED0019B5B6A0A2B08D0019B5B6A0B2B09
:10789C0002D180235B0016E0012314E0802312E068
:1078AC00402310E020230EE010230CE00C230AE010
:1078BC000A2308E0082306E0062304E0042302E080
:1078CC00022300E001231900100007F02BF903003C
:1078DC001A00019B5B685B08D218019B5B6819005E
:1078EC00100007F01FF903009BB2039363E0019BA8
:1078FC005B6A002B44D0019B5B6A012B3ED0019B41
:10790C005B6A022B38D0019B5B6A032B32D0019B44
:10791C005B6A042B2CD0019B5B6A052B26D0019B48
:10792C005B6A062B20D0019B5B6A072B1AD0019B4C
:10793C005B6A082B14D0019B5B6A092B0ED0019B50
:10794C005B6A0A2B08D0019B5B6A0B2B02D180234C
:10795C005B0016E0012314E0802312E0402310E0CA
:10796C0020230EE010230CE00C230AE00A2308E08D
:10797C00082306E0062304E0042302E0022300E0CF
:10798C00012319008023180207F0CCF803001A0019
:10799C00019B5B685B08D218019B5B6819001000A7
:1079AC0007F0C0F803009BB2039304E013236B446D
:1079BC0001221A70C046039B0F2B09D9039A80230E
:1079CC005B029A4204D2019B1B68039ADA6003E0C3
:1079DC0013236B4401221A70019B6A2201219952D4
:1079EC00019B682201219952019B0022DA66019BBE
:1079FC0000221A6713236B441B78180009B000BDD2
:047A0C000024F4005E
:107A100082B00190019B9B6A012213400BD0019B15
:107A20001B685B684A4A13401900019BDA6A019B94
:107A30001B680A435A60019B9B6A022213400BD0C9
:107A4000019B1B685B68434A13401900019B1A6B3A
:107A5000019B1B680A435A60019B9B6A04221340E6
:107A60000BD0019B1B685B683B4A13401900019BCC
:107A70005A6B019B1B680A435A60019B9B6A082250
:107A800013400BD0019B1B685B68344A13401900FC
:107A9000019B9A6B019B1B680A435A60019B9B6A7E
:107AA000102213400BD0019B1B689B682C4A13408B
:107AB0001900019BDA6B019B1B680A439A60019BCA
:107AC0009B6A202213400BD0019B1B689B68254AB0
:107AD00013401900019B1A6C019B1B680A439A60B2
:107AE000019B9B6A402213401DD0019B1B685B6871
:107AF0001D4A13401900019B5A6C019B1B680A43E5
:107B00005A60019B5A6C80235B039A420BD1019B04
:107B10001B685B68154A13401900019B9A6C019B16
:107B20001B680A435A60019B9B6A802213400BD05A
:107B3000019B1B685B680E4A13401900019BDA6CBD
:107B4000019B1B680A435A60C04602B07047C0469A
:107B5000FFFFFDFFFFFFFEFFFFFFFBFFFF7FFFFFBC
:107B6000FFEFFFFFFFDFFFFFFFFFEFFFFFFF9FFFC5
:047B7000FFFFF7FF1D
:107B740000B587B00390039B882200219950FBF73E
:107B84009DFB03000593039B1B681B68082213409D
:107B9400082B0CD1059B802291030398164A00926E
:107BA400002200F02BF8031E01D0032320E0039BE6
:107BB4001B681B6804221340042B0CD1059B8022F4
:107BC400D10303980C4A0092002200F017F8031E18
:107BD40001D003230CE0039B802220219950039BB6
:107BE400842220219950039B7C2200219954002354
:0C7BF400180007B000BDC046FFFFFF01F5
:107C000000B585B00390029100936B4607331A705C
:107C10002BE0069B013328D0FBF752FB0200009BB0
:107C2000D31A069A9A4202D3069B002B1DD1039BBE
:107C30001B681A68039B1B6816490A401A60039B5D
:107C40001B689A68039B1B6801218A439A60039B07
:107C5000802220219950039B842220219950039B4C
:107C60007C2200219954032310E0039B1B68DB69ED
:107C7000029A1340029AD31A5A425341DBB21A00B5
:107C80006B4607331B789A42C3D00023180005B017
:087C900000BDC0465FFEFFFFCE
:107C980084B00190019B80229B58212B44D10E2354
:107CA8006B44019A6A21525A1A8038E0019B562285
:107CB8009B5A9BB2002B11D1019B1B689A68019BB0
:107CC8001B681B490A409A60019B1B681A68019B44
:107CD8001B6840210A431A60C04625E0019B1B68C7
:107CE800DB698022134013D0019B1B6D1A78019B1E
:107CF8001B689A62019B1B6D5A1C019B1A65019BAC
:107D080056229B5A9BB2013B99B2019B562299522B
:107D18000E236B441A880E236B44013A1A800E23F3
:107D28006B441B88002BC1D1C04604B07047C046C5
:047D3800FFFF7FFFCB
:107D3C0084B00190019B80229B58212B49D10E23AA
:107D4C006B44019A6A21525A1A803DE0019B5622DB
:107D5C009B5A9BB2002B11D1019B1B689A68019B0B
:107D6C001B681D490A409A60019B1B681A68019B9D
:107D7C001B6840210A431A60C0462AE0019B1B681D
:107D8C00DB698022134018D0019B1B6D0293029B70
:107D9C001B881A00019B1B68D205D20D9A62019BAD
:107DAC001B6D9A1C019B1A65019B56229B5A9BB218
:107DBC00013B99B2019B562299520E236B441A88AF
:107DCC000E236B44013A1A800E236B441B88002B44
:0C7DDC00BCD1C04604B07047FFFF7FFF21
:107DE80000B585B001900E236B44019A6021525A68
:107DF8001A80019B84229B58222B40D1019B1B682F
:107E08005A6A03AB1A8003AB1B88DAB20E236B44A1
:107E18001B88D9B2019B9B6D0A40D2B21A70019B94
:107E28009B6D5A1C019B9A65019B5E229B5A9BB2D3
:107E3800013B99B2019B5E229952019B5E229B5A9B
:107E48009BB2002B23D1019B1B681A68019B1B68FE
:107E580010490A401A60019B1B689A68019B1B68BD
:107E680001218A439A60019B842220219950019B19
:107E78000022DA66019B180008F0A3FD07E0019BC9
:107E88001B689A69019B1B6808210A439A61C046CE
:087E980005B000BDDFFEFFFF95
:107EA00000B585B001900E236B44019A6021525AAF
:107EB0001A80019B84229B58222B40D1019B1B6876
:107EC0005A6A03AB1A80019B9B6D029303AB0E228F
:107ED0006A441B88128813409AB2029B1A80019B45
:107EE0009B6D9A1C019B9A65019B5E229B5A9BB2DB
:107EF000013B99B2019B5E229952019B5E229B5AE3
:107F00009BB2002B23D1019B1B681A68019B1B6845
:107F100010490A401A60019B1B689A68019B1B6804
:107F200001218A439A60019B842220219950019B60
:107F30000022DA66019B180008F047FD07E0019B6C
:107F40001B689A69019B1B6808210A439A61C04615
:087F500005B000BDDFFEFFFFDC
:107F580000B585B0019003AB019A6021525A1A808E
:107F6800019B84229B58222B00D078E00E236B447F
:107F7800019A6821525A1A8045E0019B1B685A6A87
:107F880002AB1A8002AB1B88DAB203AB1B88D9B2EA
:107F9800019B9B6D0A40D2B21A70019B9B6D5A1CC3
:107FA800019B9A65019B5E229B5A9BB2013B99B249
:107FB800019B5E229952019B5E229B5A9BB2002B29
:107FC8001AD1019B1B681A68019B1B6829490A4042
:107FD8001A60019B1B689A68019B1B6826490A4026
:107FE8009A60019B842220219950019B0022DA6625
:107FF800019B180008F0E5FC0E236B441A880E2339
:108008006B44013A1A800E236B441B88002BB4D1B1
:108018000A236B44019A5E21525A1A800A236B4440
:108028001B88002B23D0019B68229B5A0A226A4492
:1080380012889A421BD2019B1B689A68019B1B6895
:108048000E490A409A60019B0D4ADA66019B1B683B
:108058001A68019B1B6820210A431A6007E0019BEC
:108068001B689A69019B1B6808210A439A61C046EC
:1080780005B000BDFFFEFFFFFEFFFFEFFFFFFFEFB4
:04808800E97D000886
:10808C0000B587B0019005AB019A6021525A1A8055
:10809C00019B84229B58222B00D078E016236B4442
:1080AC00019A6821525A1A8045E0019B1B685A6A52
:1080BC0004AB1A80019B9B6D039304AB05AA1B8830
:1080CC00128813409AB2039B1A80019B9B6D9A1CD9
:1080DC00019B9A65019B5E229B5A9BB2013B99B214
:1080EC00019B5E229952019B5E229B5A9BB2002BF4
:1080FC001AD1019B1B681A68019B1B6829490A400D
:10810C001A60019B1B689A68019B1B6826490A40F0
:10811C009A60019B842220219950019B0022DA66EF
:10812C00019B180008F04BFC16236B441A8816238D
:10813C006B44013A1A8016236B441B88002BB4D174
:10814C0012236B44019A5E21525A1A8012236B44FB
:10815C001B88002B23D0019B68229B5A12226A4455
:10816C0012889A421BD2019B1B689A68019B1B6860
:10817C000E490A409A60019B0D4ADA66019B1B6806
:10818C001A68019B1B6820210A431A6007E0019BB7
:10819C001B689A69019B1B6808210A439A61C046B7
:1081AC0007B000BDFFFEFFFFFEFFFFEFFFFFFFEF7D
:0481BC00A17E000898
:1081C00084B00190019B7C229B5C012B01D1022396
:1081D00027E0019B7C2201219954019B80222421CC
:1081E0009950019B1B681B680393019B1B681A68CD
:1081F000019B1B6801218A431A60039B0A4A1340B2
:108200000393019B00225A66019B1B68039A1A6024
:10821000019B802220219950019B7C2200219954AE
:0C8220000023180004B07047FFFFFFDFD0
:10822C0000B587B0002302930023059333E0294B5C
:10823C00059A9200D35801930023039300230493CF
:10824C000CE0244B049A9200D358019A9A4202DD16
:10825C00039B01330393049B01330493049B7F2BF7
:10826C00EFD9059BD9B21C4A039BD3180A1C1A7070
:10827C00194A039BD3181B78002B09D1029B012BA5
:10828C0004D1164B180006F019FDFEE701230293EA
:10829C00059B01330593059B7F2BC8D9104B4022BE
:1082AC001A70002305930EE00B4A059BD3181A781D
:1082BC000B4B1B789A4203D1059BDAB2084B1A7010
:1082CC00059B01330593059B7F2BEDD9C046C0461A
:1082DC0007B000BD7C050020B0080020E8000108B4
:0482EC00441000201A
:1082F00000B587B00023049300F0A8F8802303930F
:108300001D4B5B681B0A7F221340029300230493DA
:1083100021E0194B5B68194A13401900049B1A02AB
:10832000154B0A435A600223059303E000F02AF834
:1083300003000593059B022BF8D000230193019ABB
:10834000059BD318019301990D4B049A9200D150CB
:10835000049B01330493049A039B9A42D9D3064B9E
:108360005B68064A13401900029B1A02024B0A433B
:108370005A60C04607B000BD00100240FF80FFFFFA
:048380007C05002058
:1083840010B582B02B4B1B68042B0CD1294B012256
:108394001A60294B00211800FEF7F6F8152008F0A2
:1083A400B4FE022343E0234B1B68032B01D00223BA
:1083B4003DE0204B1B68032B38D1152008F0B5FE97
:1083C4001D4B00211800FEF73FF91A4B04221A60D6
:1083D4001A4B1B68002B07D0194B1B681A03194B47
:1083E4001B68D218174B1A60144B1B68092B06D84C
:1083F400124B1B685A1C114B1A60022317E000230E
:1084040001930E4B00221A600B4B1B689B6A5C1C89
:108414000C4B1B680A21180006F088FB0300634319
:108424000193084B00221A60019B00E0002318000E
:1084340002B010BD280C0020F40A0020C80B002054
:088444002C0C0020E80B0020C5
:10844C0010B500F007F8024B04221A60C04610BDAC
:04845C00280C0020C8
:1084600000B587B0284B1A6C274B802189020A433C
:108470001A64254B1A6C80239B0213400193019BC5
:10848000224B234A1A60214B1800FEF74FF81F4B6E
:10849000204ADA601D4B00225A601C4B00221A61F0
:1084A0001A4B00229A60194B180008F0FAFE031EBE
:1084B00000D0FEE702AB00221A6002AB01225A6034
:1084C00002AB0C229A6002AB0022DA6002A90F4BC9
:1084D00000221800FEF74AFA031E00D0FEE70B4BFD
:1084E000002202211800FEF763FC031E00D0FEE705
:1084F00000220021152008F0F6FD152008F017FED7
:10850000C04607B000BDC04600100240F40A00207B
:0885100000440140FFFF0000E0
:1085180000B583B00190019B1B7F012B6ED1394BB5
:108528001B68012B0BD1019B0021180008F0F0F902
:108538000200354B1A60334B02221A605EE0314B61
:108548001B68022B5AD1019B0021180008F0E0F9A2
:1085580002002E4B1A60152008F0E5FD2C4B002177
:108568001800FEF76FF8019B1B68032252421A613C
:10857800264B1A68244B1B689A4219D9234B1A6850
:10858800214B1B68D21A234B1A60224B1B681B0312
:10859800214A93422FD8214B180005F091F91D4B21
:1085A8001B681A031E4B1100180006F089FB22E015
:1085B800164B1A68144B1B689A421BD2134B1A6845
:1085C800114B1B68D31A174A9A18124B1A60114B91
:1085D8001B681B03104A93420DD8104B180005F076
:1085E8006FF90C4B1B681A030D4B1100180006F0AD
:1085F80067FB00E0FEE7034B03221A60C04603B0A6
:1086080000BDC046280C0020240C0020200C0020AF
:10861800F40A00202C0C00203F5DC6004801010828
:0886280058010108FFFF0000EA
:1086300010B586B00590049103920293059B049AAD
:108640001A60059B1B684C4A1A60059B1B689622A2
:10865000D2015A60059B1B68802252019A60059BDB
:108660001B680022DA60059B1B688022D2001A6119
:10867000059B1B680C225A61059B1B6800229A61AE
:10868000059B1B680022DA61059B1B6800221A62A9
:10869000059B1B6800225A62059B1B6800229A6298
:1086A000059B1B68039A5A60029B002B0AD1059B0D
:1086B0001B688022D2001A61059B1B688022520130
:1086C0009A6015E0029B012B0AD1059B1B68C02212
:1086D000D2001A61059B1B68802252019A6007E054
:1086E000059B1B6800221A61059B1B6800229A608B
:1086F000089B012B04D1059B1B680022DA6004E073
:10870000059B1B6880229201DA60059B1C68099812
:1087100006F030F90022194B08F0C7FA02000B00EE
:108720001000190006F08AF80300009300230022CD
:108730000021200000F026F8031E01D008F0B9FF48
:10874000059B1B681800FFF73BFD031E01D008F0D6
:10875000B0FF059B1868059B273380225200190043
:10876000FEF706FC031E04D0054B180006F0ACFA19
:10877000FEE7C04606B010BD0038014000000C40C6
:04878000DC0101080F
:1087840000B587B00390029101920093039B002BE4
:1087940001D1012395E0039B80229B58002B07D134
:1087A400039B7C2200219954039B180004F0DCFCF9
:1087B400039B802224219950039B1B681A68039B06
:1087C4001B6801218A431A60039B1800FEF7C4FC4E
:1087D4000300012B01D1012373E0039B9B6A002B4F
:1087E40003D0039B1800FFF711F9039B1B689A68D9
:1087F400039B1B688021C9010A439A60039B1B6881
:108804009B68314A13401900039B1B68029A0A4370
:108814009A60019B5B050593009B1B04059A134317
:108824000593039B1B681B68284A13401900039B8C
:108834001B68059A0A431A60039B1B685A68039BCA
:108844001B68802109040A435A60039B1B681A6849
:10885400039B1B688021C9040A431A60039B5A685E
:108864009623DB019A420AD8039B1B685B691B0EA3
:108874001906039B1B68089A0A435A6114E0039B78
:108884005B68134A53431349180006F04FF9030079
:1088940001330493039B1B685B691B0E1906039B3E
:1088A4001B68049A0A435A61039B1B681A68039B5A
:1088B4001B6801210A431A60039B1800FFF758F94B
:1088C4000300180007B000BDFF7FFFFFFFFF00FC9F
:0888D400D606000040420F002F
:1088DC0000B589B00190019B1B68DB690793019B74
:1088EC001B681B680693019B1B685B680593019BC7
:1088FC001B689B680493079B0F2213400393039BF5
:10890C00002B5DD0049B954A134004D1069A90230A
:10891C005B00134054D0079B0122134010D0069AE1
:10892C0080235B0013400BD0019B1B6801221A6251
:10893C00019B88229B5801221A43019B88215A5083
:10894C00079B022213400FD0049B012213400BD033
:10895C00019B1B6802221A62019B88229B580422ED
:10896C001A43019B88215A50079B042213400FD0B5
:10897C00049B012213400BD0019B1B6804221A623A
:10898C00019B88229B5802221A43019B88215A5032
:10899C00079B0822134013D0069B2022134003D1BF
:1089AC00049B6E4A13400BD0019B1B6808221A6271
:1089BC00019B88229B5808221A43019B88215A50FC
:1089CC00079A80231B0113401DD0069A8023DB04D9
:1089DC00134004D1049A80231B04134013D0019B31
:1089EC001B68802212011A62019B8422202199505B
:1089FC00019B802220219950594B01221A75584B0A
:108A0C00584A01219954079B2022134037D0069BCA
:108A1C002022134004D1049A80235B0513402ED0EE
:108A2C00019B84229B58222B21D14D4A8A239B00E7
:108A3C00D358FF2B1BD8019B1B68596A484A8A23C1
:108A4C009B00D358C8B2464A2721D3185B18021C86
:108A5C001A70434A8A239B00D358591C404A8A23D4
:108A6C009B00D1503E4B3F4A0121995407E0019B9A
:108A7C001B689A69019B1B6808210A439A61079B32
:108A8C008022134012D0069B8022134004D1049AFA
:108A9C0080231B04134009D0314B1B68180008F0CD
:108AAC007EFC2F4A8C239B000121D154079B402232
:108ABC0013400FD0069B402213400BD0284B26228C
:108ACC0000219954019B180008F000F8019B8422A6
:108ADC0022219950019B88229B58002B3BD0019B53
:108AEC00842222219950079B2022134015D0069BEB
:108AFC002022134004D1049A80235B0513400CD030
:108B0C00019B1B689A69019B1B6808210A439A61A7
:108B1C00019B8822002199501DE0079B8022134065
:108B2C0019D0069B8022134004D1049A80231B0485
:108B3C00134010D00A4B262200219954019B180097
:108B4C0007F0C4FF019B842222219950044A8C23F4
:108B5C009B000121D154C04609B000BD010000109A
:088B6C00480300203102000063
:108B740086B00190009116236B44012252421A8060
:108B84000023049334E0019A049BD3181B78190042
:108B940016236B4416226A4412884A401A8008231A
:108BA40003931FE016236B441B88012213400FD04C
:108BB40016236B4416226A44128852081A8016231C
:108BC4006B4416226A4412880E494A401A8006E011
:108BD40016236B4416226A44128852081A80039B97
:108BE400013B0393039B002BDCD1049B01330493CF
:108BF400049A009B9A42C6D316236B441B88180020
:088C040006B0704701A0FFFF5C
:108C0C0000B587B00190019B27330593019A8A2305
:108C1C009B00D3580493059B1B780393049B042B54
:108C2C0005D8019B180007F09DFF002321E0049A52
:108C3C00059B1100180007F062FF0300013305D1FA
:108C4C00019B180007F08EFF002312E0039B002B02
:108C5C0001D102230DE0084B1B8B9BB21A00039B26
:108C6C00934201D1022304E0019B180007F07AFF24
:0C8C7C000023180007B000BDB00000206D
:108C880000B589B00390029101921A006B46033334
:108C98001A706B4603331B789AB23F4B1B8B9BB2FF
:108CA8009A420CD06B4603331B78002B07D0019BEC
:108CB80003980B22062108F05EFC030068E0029B83
:108CC80002331B781B02029A033212789B18069310
:108CD800029B04331B781B02029A053212789B18F8
:108CE8000593059B002B02D0059B7D2B07D9019B83
:108CF80003980322032108F03EFC030048E0069A8B
:108D0800059BD318013BD32B07D9019B039802225B
:108D1800032108F030FC03003AE0039A019BD318C2
:108D280003221A70019B01330193059BD9B2039A60
:108D3800019BD2180B1CDB18DBB21370019B0133AB
:108D48000193069B07931CE0039A019BD3181249D1
:108D5800079A52008A1801321278D2B21A70019B0F
:108D680001330193039A019BD3180B4A07994900D1
:108D78008A5CD2B21A70019B01330193079B0133BD
:108D88000793069A059BD318079A9A42DCD3019B4E
:0C8D9800180009B000BDC046B00000206B
:108DA40000B589B003900291019200934B4B1B8B49
:108DB4009BB21A00009B93420AD0009B002B07D061
:108DC400019B03980B22062108F0D7FB030081E0E6
:108DD400029B02331B781B02029A033212789B18FF
:108DE4000593029B04331B781B02029A0532127806
:108DF4009B18049307230693049B002B02D0049B27
:108E04007B2B07D9019B03980322102108F0B5FBA3
:108E140003005FE0059A049BD318013BD32B07D9C9
:108E2400019B03980222102108F0A7FB030051E0E4
:108E3400059B079319E0029A069BD3181978274AD1
:108E4400079B5B00D31801330A1C1A70069B01337D
:108E5400029AD3181978214B079A5200D154069BD1
:108E640002330693079B01330793059A049BD31897
:108E7400079A9A42DFD3039A019BD31810221A70DF
:108E8400019B01330193059B190A039A019BD31893
:108E9400CAB21A70019B01330193039A019BD31840
:108EA400059AD2B21A70019B01330193049B190AEB
:108EB400039A019BD318CAB21A70019B0133019320
:108EC400039A019BD318049AD2B21A70019B0133FE
:108ED4000193019B180009B000BDC046B0000020FA
:108EE40000B587B00390029101920093324B1B8B23
:108EF4009BB21A00009B93420AD0009B002B07D020
:108F0400019B03980B22062108F037FB030050E075
:108F1400029B02331B781B02029A033212789B18BD
:108F24000593059BD32B07D9019B039802220621A5
:108F340008F023FB03003CE0029B19791E4A059BC1
:108F44005B00D31801330A1C1A70029B59791A4B1F
:108F5400059A5200D154039A019BD31806221A7021
:108F6400019B01330193059B190A039A019BD318B2
:108F7400CAB21A70019B01330193039A019BD3185F
:108F8400059AD2B21A70019B01330193039A019B93
:108F9400D318029A12791A70019B01330193039A30
:108FA400019BD318029A52791A70019B01330193E1
:0C8FB400019B180007B000BDB0000020B9
:108FC00000B585B001AB18000C231A00002106F093
:108FD0001DFE754B754A1A60734BE02252035A60AE
:108FE000714B00229A60704B0022DA606E4B802237
:108FF00092031A616C4B08225A616B4B00221A765D
:10900000694B00225A76684B01229A76664B0A22F7
:10901000DA61654B202200219954634B00225A6289
:10902000614B00229A62604B2C22012199545E4BC5
:10903000802252011A635C4B05225A635A4B052267
:109040009A63594B3C2201219954574B0C221A64C4
:10905000554B00225A64544B00229A64524B002212
:10906000DA64514B1800FAF7B9F9031E01D008F081
:1090700020FB01AB01221A6001AB00225A6001AB58
:1090800007229A6001AA484B11001800FAF702FC67
:10909000031E01D008F00DFB01AB454A1A6001AB7D
:1090A00004225A6001AB07229A6001AA3E4B1100CC
:1090B0001800FAF7EFFB031E01D008F0FAFA01AB33
:1090C0003C4A1A6001AB08225A6001AB07229A6041
:1090D00001AA354B11001800FAF7DCFB031E01D082
:1090E00008F0E7FA01AB344A1A6001AB0C225A606F
:1090F00001AB07229A6001AA2B4B11001800FAF766
:10910000C9FB031E01D008F0D4FA01AB2B4A1A6048
:1091100001AB10225A6001AB07229A6001AA224BD0
:1091200011001800FAF7B6FB031E01D008F0C1FACF
:1091300001AB234A1A6001AB14225A6001AB07222B
:109140009A6001AA184B11001800FAF7A3FB031E3E
:1091500001D008F0AEFA01AB1A4A1A6001AB18222E
:109160005A6001AB07229A6001AA0F4B1100180048
:10917000FAF790FB031E01D008F09BFA01AB124AEC
:109180001A6001AB1C225A6001AB07229A6001AA47
:10919000054B11001800FAF77DFB031E01D008F003
:1091A00088FAC04605B000BD9409002000240140A3
:1091B00002000004040000080800000C1000001069
:0C91C0000001002000040028001000B096
:1091CC0000B58BB0019005AB180014231A000021D8
:1091DC0006F016FD019B1B686E4A934200D0D5E049
:1091EC006D4B1A6C6C4B802149030A431A646A4B11
:1091FC001A6C80235B0313400493049B664B5A6BDD
:10920C00654B01210A435A63634B5B6B012213408C
:10921C000393039B604B5A6B5F4B02210A435A63C7
:10922C005D4B5B6B022213400293029B05AB012248
:10923C001A6005AB03225A6005AB00229A6005AA9E
:10924C00A023DB0511001800FBF7C2FB05AB0222C3
:10925C001A6005AB03225A6005AB00229A6005AA7E
:10926C00A023DB0511001800FBF7B2FB05AB0422B1
:10927C001A6005AB03225A6005AB00229A6005AA5E
:10928C00A023DB0511001800FBF7A2FB05AB0122A4
:10929C001A6005AB03225A6005AB00229A6005AB3D
:1092AC003E4A19001000FBF793FB05AB02221A6033
:1092BC0005AB03225A6005AB00229A6005AB374A16
:1092CC0019001000FBF784FB05AB04221A6005ABF8
:1092DC0003225A6005AB00229A6005AB2F4A190095
:1092EC001000FBF775FB05AB08221A6005AB0322D7
:1092FC005A6005AB00229A6005AAA023DB05110079
:10930C001800FBF765FB05AB10221A6005AB0322B6
:10931C005A6005AB00229A6005AAA023DB05110058
:10932C001800FBF755FB1E4B1E4A1A601C4B0522FE
:10933C005A601B4B00229A60194B0022DA60184BC2
:10934C0080221A61164B802252005A61144B8022E3
:10935C0012019A61124B2022DA61114B00221A621F
:10936C000F4B1800FAF760FE031E01D008F09BF9B2
:10937C00019B0B4A1A650A4B019A9A620022002142
:10938C000C2007F0AAFE0C2007F0BBFEC0460BB069
:10939C0000BDC046002401400010024000040050F3
:0893AC00F8090020080002404E
:1093B40000B587B003900A000B236B441A7005AB09
:1093C40023221A7005AA05A903980A2300930323EC
:1093D400FCF788FD05AB9B785BB2102293435AB22D
:1093E4000B236B441B785BB213435BB2DAB205AB5D
:1093F4005A7005AB43221A7005AA05A903980A23DB
:1094040000930223FCF76EFD05AB23221A7005AA14
:1094140005A903980A2300930323FCF763FD05AB16
:109424009B780B226A4412781340DBB20B226A4405
:1094340012789A4204D0044B180004F043FAFEE771
:0C944400C04607B000BDC046C8FD0008CF
:1094500000B587B003900A000B236B441A7005AB6C
:1094600023221A7005AA05A903980A23009303234F
:10947000FCF73AFD05AB9B785BB2602293435AB28E
:109480000B236B441B785BB213435BB2DAB205ABC0
:109490005A7005AB43221A7005AA05A903980A233E
:1094A00000930223FCF720FD05AB23221A7005AAC6
:1094B00005A903980A2300930323FCF715FD05ABC8
:1094C0009B780B226A4412781340DBB20B226A4469
:1094D00012789A4204D0044B180004F0F5F9FEE724
:0C94E000C04607B000BDC046ECFD00080F
:1094EC0000B587B003900A000B236B441A7005ABD0
:1094FC0022221A7005AA05A903980A2300930323B4
:10950C00FCF7ECFC05AB9B785BB2072213405AB21C
:10951C000B236B441B785BB213435BB2DAB205AB23
:10952C005A7005AB42221A7005AA05A903980A23A2
:10953C0000930223FCF7D2FC05AB22221A7005AA79
:10954C0005A903980A2300930323FCF7C7FC05AB7A
:10955C009B780B226A4412781340DBB20B226A44CC
:10956C0012789A4204D0044B180004F0A7F9FEE7D5
:0C957C00C04607B000BDC04608FE000855
:1095880000B587B003900A000B236B441A7005AB33
:1095980051221A7005AB0B226A4412785A7005AB37
:1095A80000229A7005AA05A903980A2300930223AA
:1095B800FCF796FC05AB31221A7005AA05A9039899
:1095C8000A2300930323FCF78BFC05AB9B780B2243
:1095D8006A4412789A4203D0034B180004F070F9D9
:0C95E800C04607B000BDC04644FE0008AD
:1095F40000B587B0039005AB114A118819809278A1
:109604009A7005AA05A903980A2300930223FCF77C
:1096140069FC05AB26221A7005AA05A903980A233A
:1096240000930323FCF75EFC05AB9B780A2B04D064
:10963400044B180004F046F9FEE7C04607B000BD2D
:089644008CFE000864FE000822
:10964C0000B583B00190019AC4235B00D258019BF2
:10965C009A67019BCE229B5A19B2019B7C2299528C
:10966C00019BCC229B5A19B2019B7E229952019BE1
:10967C00D4229B581900019B80229950034B002146
:10968C00180001F07FFCC04603B000BDB000002004
:10969C0000B587B00190019BD4229B581900019B07
:1096AC0084229950019B84229A58019B80215B58FB
:1096BC00D31A05930D4B1B680493049A13005B019A
:1096CC009B1A9B009B18DB000599180005F002FA09
:1096DC0003000393019B8821039A5A50044B0021E9
:1096EC00180001F04FFCC04607B000BD140C002060
:0496FC00B00000209A
:1097000000B585B0164BCC229B5A19B2144B8C2253
:109710009952134B8C229B5A1BB21900104B7E227C
:109720009B5A1BB2CB1A03930E4B1B680293029AEF
:1097300013005B019B1A9B009B18DB000399180028
:1097400005F0CEF903000193054B9021019A5A5080
:10975000034B0021180001F01BFCC04605B000BD02
:08976000B00000201C0C0020E9
:1097680000B585B001904B4B180005F0A9FA019B94
:109778009C229B58002B04D1474B180004F0A0F8FA
:1097880086E0019B9C229B58180005F0A3F8002254
:10979800424B04F00DFF02000B0010001900404B73
:1097A8001A685B6804F004FF02000B00029203933E
:1097B80000223C4B0298039907F073FA02000B0051
:1097C8001000190004F0D0FF0200019B94215A50A8
:1097D800019BCE229B5A19B2019B98229952019B58
:1097E800CC229B5A19B2019B9A2299522C4B1A6887
:1097F8005B682D49080005F063FA019B9C229B5881
:10980800180005F067F80022244B04F0D1FE02008E
:109818000B002649080005F053FA019B98229B5A31
:109828001BB2180005F056F80022214B04F0C0FEC8
:1098380002000B001F49080005F042FA019B9A221A
:109848009B5A1BB2180005F045F80022184B04F08B
:10985800AFFE02000B001849080005F031FA019B21
:1098680094229B58180005F035F800220D4B07F09C
:1098780018FA02000B001149080005F021FA104BF4
:10988800180005F01DFA0F4B0021180001F07CFBB1
:1098980005B000BD90FE0008A4FE000800408F40FF
:1098A8004003002080842E4100FF000820FF0008AC
:1098B8000000594030FF00083CFF000848FF00083E
:0898C8005CFF0008B000002065
:1098D00000B585B05C4B180005F0F6F95B4BCE2265
:1098E0009B5A19B2594BA0229952584BA0229B5A0D
:1098F0001BB2180004F0F2FF0022554B04F05CFE8E
:1099000002000B005349080005F0DEF94F4BCE2250
:109910009B5A1BB219004D4B98229B5A1BB2CB1A73
:109920000393039804F0DAFF0022494B04F044FE4D
:1099300002000B004849080005F0C6F9474B1A68B9
:109940005B6800920193454B1A685B6844490800C4
:1099500005F0BAF93D4B9C229B58180004F0BEFF5D
:109960000022404B04F028FE02000B003E49080094
:1099700005F0AAF9354B9C229B58180004F0AEFF65
:109980000022384B04F018FE02000B0010001900F2
:10999000009A019B04F010FE02000B00009201935C
:1099A0000022324B0098019904F058FD02000B0090
:1099B00000920193039804F091FF02000B000098BD
:1099C000019904F0F9FD02000B00009201930022BE
:1099D000274B0098019907F068F902000B0010006E
:1099E000190004F0C5FE0200184BA4215A50174B71
:1099F000A4229B58180004F071FF00221C4B04F0B5
:109A0000DBFD02000B00100019000022104B07F0D4
:109A10004CF902000B00100019000022134B04F057
:109A200039FC02000B001349080005F04DF9124BF8
:109A3000180005F049F9054B0021180001F0A8FABB
:109A4000C04605B000BDC04674FF0008B00000204D
:109A5000000059408CFF00089CFF000830030020E4
:109A6000ACFF000800408F40E0FF00080000F03F1E
:0C9A700065CDCD41ECFF0008100001089E
:109A7C0000B591B00190A64B1B68A64A934204D046
:109A8C00A34B1B685A1CA24B1A60A34B1B68002BE0
:109A9C0000DA01335B105B421A009F4B1B68D21833
:109AAC009D4B1A609C4B1A68019BD2189A4B1A60FA
:109ABC00994B1B68002B00DA01335B100F93974A0C
:109ACC00C4235B000F99D150944B9B6F0F9AD21A01
:109ADC00934B1A60914BD4229B5819008F4B8022C8
:109AEC009B58CB1A0E938D4B88229B580E9A53433E
:109AFC00180004F0EDFE00228A4B04F057FD020022
:109B0C000B001000190004F02DFE03000D93834A86
:109B1C00C6235B000D99D150814B1A680D9BD21A4C
:109B2C00814B1A607D4BCC229B5A1BB219007B4B8C
:109B3C007E229B5A1BB2CB1A180004F0C9FE0200FD
:109B4C000B000A920B93754B90229B58180004F053
:109B5C00BFFE0A9A0B9B07F0A2F802000B00100044
:109B6C00190000226F4B04F021FD02000B001000C5
:109B7C00190004F0F7FD030009936B4B1A68099B5D
:109B8C00D21A6A4B1A60694B1B68180004F0A0FECD
:109B9C000022674B07F083F802000B00100019003D
:109BAC000022644B07F07BF802000B001000190038
:109BBC000022614B04F0FAFC02000B005F490A60C2
:109BCC004B60564B94229B58180004F081FE0022E7
:109BDC005B4B04F0EBFC02000B0010001900574B20
:109BEC001A685B6807F05BF802000B0055490A60C5
:109BFC004B604A4BCE229B5A1BB21900474B982202
:109C0C009B5A1BB2CB1A180004F062FE02000B0028
:109C1C0006920793414BA4229B58180004F058FE5F
:109C2C000022494B04F0C2FC02000B000492059385
:109C3C00049A059B0698079907F031F802000B006F
:109C4C00100019000022414B04F01EFB02000B0017
:109C5C00029203933B4B18685968029A039B07F0D6
:109C6C001EF802000B003A490A604B60384B18682A
:109C7C0059680022374B04F035FD031E08D1344BD4
:109C8C00186859680022344B04F04CFD031E07D0B1
:109C9C00224AC8235B00D258204BE4215A5010E0D2
:109CAC002B4B1868596800221E4B06F0F8FF020077
:109CBC000B001000190004F055FD0200174BE421B5
:109CCC005A50134B1B68142B1BDD144BE4229A586F
:109CDC00124BE8215B589A4205DD104BE4229A584E
:109CEC000E4BE8215A500D4BE4229A580B4BEC21A9
:109CFC005B589A4205DA094BE4229A58074BEC213F
:109D0C005A50164B01221A600023180011B000BDE6
:109D1C00BC0B0020FFFFFF7F080C0020B0000020D0
:109D2C00140C002000408F401C0C0020180C00204C
:109D3C000000084000005940000060414003002032
:109D4C0080842E413003002065CDCD410000F03FD2
:109D5C003803002000307140003071C0B00B00207F
:109D6C0000B585B001AB47221A60043306220021EE
:109D7C00180005F045FF344B00221A70802359015E
:109D8C00A023DB050122180006F02EFD9620F9F722
:109D9C0097FA2E4B00221021180006F025FD962074
:109DAC00F9F78EFA294B01221021180006F01CFD40
:109DBC009620F9F785FA254B00222021180006F091
:109DCC0013FD9620F9F77CFA204B01222021180074
:109DDC0006F00AFD9620F9F773FA80235901A023A7
:109DEC00DB050022180006F0FFFC002202210720F0
:109DFC0007F073F9072007F084F9154B1800FFF7EB
:109E0C00F3FB9620F9F75CFA114B20211800FFF7B1
:109E1C0067FB0F4B00211800FFF7C6FA0C4B2021F3
:109E2C001800FFF70FFB0A4B34211800FFF7A6FBB5
:109E3C009620F9F745FA044B03221A7006F0DAFE65
:109E4C00C04605B000BDC0464510002000040050BF
:049E5C0030090020A9
:109E600000B589B003AB12221A6004330622002128
:109E7000180005F0CBFE0023079303AA03A9184896
:109E80000A2300930523FCF72FF806AB0022DA70B3
:109E900003AB9A7806AB9A7003ABDA7806AB5A70CC
:109EA00003AB1A7906AB1A70069A80231B049A42F8
:109EB00007D3069B0B4A944663440693069B07937D
:109EC00006E0069A80231B049A4201D2069B079360
:109ED000079B1800FFF7D2FDC04609B000BDC04681
:089EE00030090020010000FF21
:109EE80000B583B0114BDB6D180000231900E12287
:109EF8001201002304F0D8FD02000B000092019328
:109F08000A4BF83318685968094A002304F0CCFD55
:109F180002000B0010001900009A019B04F028FEB3
:109F280002000B001300180003B000BDB0000020B1
:049F3800A0860100FE
:109F3C00F0B589B04648002104900591454886212A
:109F4C0049004158002907D14249C96D8C46414806
:109F5C0086214900644644503E48B421490041588A
:109F6C00002908DA3B48B4214900415849420A000B
:109F7C00C9170B0001E00022002302920393002278
:109F8C00002306920793334A86235B00D358002B99
:109F9C001DDC049A059B0298039904F083FD0200D2
:109FAC000B00100019002B4BDB6D1E0000231F0053
:109FBC0032003B0004F0DAFD02000B001000190027
:109FCC00049A059B121A8B41069207931EE0049A81
:109FDC00059B0298039904F065FD02000B0010002C
:109FEC0019001C4A86235B00D3580093DB1701939E
:109FFC00009A019B04F0BAFD02000B00100019003E
:10A00C00049A059B121A8B4106920793079A059B9B
:10A01C009A4207DC079A059B9A4208D1069A049B40
:10A02C009A4204D9049A059B069207930CE0079B6D
:10A03C00002B09DC079B002B02D1069B002B03D1C4
:10A04C000022002306920793069B180009B0F0BD6E
:08A05C00A0860100B000002005
:10A06400F0B59FB0002200231C921D930022002310
:10A074001A921B93002200231892199300220023A2
:10A0840016921793002200231492159300220023A2
:10A09400129213930022002310921193884BDB6DCC
:10A0A400180000231900E1221201002304F0FEFC31
:10A0B40002000B000E920F93824B1A685B6811002A
:10A0C40019430BD17E4A96235B00D2587E4B5343EF
:10A0D4001E0000231F007B4B1E605F607B4B1A68D1
:10A0E4005B68110019430DD1754A98235B00D2585F
:10A0F400754B5343009300230193744B0099019AC9
:10A1040019605A606E4BE4229B58002B23DB6C4B86
:10A1140052229B5A9BB2180004F0DEFB00226C4BC7
:10A1240004F048FA02000B0014921593644BE422E5
:10A134009B58180004F0D0FB149A159B06F0B3FD4D
:10A1440002000B001000190004F010FB02005C4B2D
:10A15400F0215A5069E05A4BD86D594A6823D35AB2
:10A164009BB2190004F0E2FC03000D93544BE4226B
:10A174009A580D9B5B429A4251DA514BE4229B5808
:10A18400180004F0A9FB02000B001A921B930D980F
:10A1940004F0A2FB02000B001A981B9904F00AFABF
:10A1A40002000B001C921D931C9B0A931D9A802392
:10A1B4001B0653400B930A9A0B9B1C921D93404B16
:10A1C40050229B5A9BB2180004F086FB0022404B9D
:10A1D40004F0F0F902000B001892199300223D4B91
:10A1E4001898199904F038F902000B001C981D996D
:10A1F40003F0D2FE02000B0016921793169A179BD7
:10A204001A981B9906F04FFD02000B00100019006C
:10A2140004F0ACFA02002A4BF0215A5005E0284B16
:10A22400E4229A58264BF0215A50254B70229B5A0F
:10A234001BB21900224BF0229B585A1A204BF021D2
:10A244005A501F4BE4229B58002B45DA1C4BE42246
:10A254009B585B420293DB1703931A4B1A685B68A3
:10A26400029803998018594102000B0015490A60AD
:10A274004B60144B18685968134A002304F092FC8D
:10A2840002000B0011000E4A96235B00D1500C4AC9
:10A2940096235B00D25813005B019B1A9B009B180A
:10A2A400DB001A00064BDB6D1900100004F03EFCC5
:10A2B400030099B2024A9E235B00D1522CE0C046AF
:10A2C400B00000200003002080EE360010030020C0
:10A2D400000059400000F03FB24BE4229B58049325
:10A2E400DB170593B04B1A685B68049805998018CE
:10A2F400594102000B00AC490A604B60AA4B186834
:10A304005968AA4A002304F04DFC02000B00110016
:10A31400A44A98235B00D150A24BF0229958A14B38
:10A32400F8331A685B680691C9170791069807996C
:10A3340012184B419B49F8310A604B60994BF0224B
:10A344009B580893DB170993994B1A685B68089824
:10A3540009998018594102000B0095490A604B6025
:10A36400934B18685968E1221201002304F002FC9F
:10A3740002000B0011008B4AB4235B00D150894BBF
:10A38400F8331A685B680F99994205DB0F99994273
:10A3940009D10E99914206D2824BF83319000E9AD4
:10A3A4000F9B0A604B60824B1A685B68002B02DCCF
:10A3B40006D1002A04D07E49002200230A604B60A3
:10A3C400784BDB6D774A5421525A92B253431800AA
:10A3D40004F0CEFA0022774B04F0ECF802000B00F4
:10A3E4001000190004F0DCF902000B001092119324
:10A3F4006C4BD8229B586B4A5821525A92B29342C2
:10A4040018DD684BE4229B581C00DB171D00119BD0
:10A41400AB4205DC119BAB420CD1109BA34209D982
:10A42400654B00229B5E9BB201339BB21AB2624B16
:10A434001A8002E0604B00221A805F4B00229B5E70
:10A444001900584B56229B5A9BB2994210DD554B2A
:10A45400F83319000E9A0F9B0A604B60544900228E
:10A4640000230A604B6003F0A5F9544B01221A60E3
:10A474004C4BF83318685968E1221201002304F0A8
:10A4840079FB02000B001100464BF4229950454B16
:10A49400D8229B584349C02252008A5A92B293420E
:10A4A40041DA474B1B8801339AB2454B1A80444B1F
:10A4B4001B88042B3AD9414B1B68012B36D1394BED
:10A4C40056229B5A9AB23E4B1A80364A90235B001E
:10A4D400D258E1231B019A421FD3324A90235B00D6
:10A4E400D358384A934218D82E4AB4235B00D35821
:10A4F400002B04DB2B4AB4235B00D35804E0294A25
:10A50400B4235B00D3585B422649862252008B5009
:10A5140002F0F2FF294B00221A60224A92235B00C8
:10A524000021D15002E0264B00221A801D4B6422E8
:10A534009B5A9BB2042B2CD89A00234BD3181B682C
:10A544009F46FFF7CFFC0100164A80235B00D150E1
:10A5540025E0FFF7F1FC0100124A80235B00D15093
:10A564001DE002F0E5FF01000E4A80235B00D1509C
:10A5740015E003F01BF801000A4A80235B00D15068
:10A584000DE003F099F80100064A80235B00D150E6
:10A5940005E0044A80235B000021D150C046C04638
:10A5A4001FB0F0BDB00000201003002080EE360084
:10A5B4002803002000005940320C0020AC0B00207E
:0CA5C400300C002080FC0A0018FC00088D
:10A5D00000B587B001900091474B1B68474A9342F2
:10A5E00004D0454B1B685A1C434B1A60444B1A68F5
:10A5F000434B1B689B09D21A414B1A60404B1A68A7
:10A60000019BD2183E4B1A603D4B1B689B0905937A
:10A610003C4B1A683B4B1B689B09D21A394B1A609A
:10A62000384B1A68009BD218364B1A60354B1B68A2
:10A630009B090493059A049BD31A180004F03AF975
:10A64000031C0393304BCA229B5A9BB2180004F0A0
:10A6500031F9031C0399181C03F008FF031C181C94
:10A6600004F0A2F90022294B03F0A6FF02000B0020
:10A670001000190004F0BAF9031C0393039804F0C6
:10A6800093F9234A234B03F0E9FE02000B0010006C
:10A6900019000022204B06F008FB02000B001000FE
:10A6A000190004F065F80200174BD8215A50124BDC
:10A6B0001A68A0239B009A421BDD134BD8229A589C
:10A6C000114BDC215B589A4205DD0F4BD8229A587A
:10A6D0000D4BDC215A500C4BD8229A580A4BE021E2
:10A6E0005B589A4205DA084BD8229A58064BE0216B
:10A6F0005A50C04607B000BDC00B0020FFFFFF7FCF
:10A70000F80B0020000C0020B00000200000F040FA
:0CA71000DA9E4A94EEBF903F00004540E6
:10A71C0000B585B01F4B0393039B1B88180004F0F6
:10A72C0013F9031C02938B21C905029803F0F4FE64
:10A73C00031C02931849029803F092FE031C181C88
:10A74C0004F064F80200154B1A60154B0393039B3D
:10A75C001B88180004F0F8F8031C01938B21C90521
:10A76C00019803F0D9FE031C01930B49019803F0E7
:10A77C0077FE031C181C04F049F80200094B1A6000
:10A78C00084B1A68054B1B68D21A074B1A60C04657
:10A79C0005B000BDA875FF1F00803B45F00B0020E5
:0CA7AC00CA75FF1FF40B0020EC0B00200E
:10A7B80000B585B00190019B144A53431B0C0393C9
:10A7C800039A134B1B68D31A0393039B114A5343F1
:10A7D8000393114B1B681900039804F07DF90300DB
:10A7E8000393039B0D4A944663440393039B0A21F6
:10A7F800180004F071F9030019B2094BCC229952E0
:10A8080000F010F8C04605B000BDC046E40C0000DA
:10A81800F00B0020A0860100EC0B00203075000032
:04A82800B00000205C
:10A82C0030B585B0254B5A229B5A99B2234AC02386
:10A83C005B00D152214BCC229B5A1AB21F4B6A217E
:10A84C005B5A1BB29A4235DA0E236B441B4ACC215D
:10A85C00525A1A80194BCC229B5A1AB2174B6C21A4
:10A86C005B5A1BB29A4205DC0E236B44134A6C21D3
:10A87C00525A1A80114B6C229B5A18B20F4B6E22F3
:10A88C009B5A9BB219B20D4B6A229B5A1AB20B4BB4
:10A89C005A241B5B9BB21CB20E236B4400255B5FDE
:10A8AC000093230006F083FE030099B2034AC023F1
:10A8BC005B00D152C04605B030BDC046B000002090
:10A8CC0000B583B00B4B9A6B0A4B01210A439A6378
:10A8DC00084B9B6B012213400193019B0022012129
:10A8EC00092006F0FAFB092006F00BFCC04603B069
:08A8FC0000BDC046001002403F
:10A9040086B0039002910192039A019BD218124BD4
:10A914001B689902FF239B020B40802109058C468A
:10A9240063449A4201D9012313E0002305930BE009
:10A93400039A059BD3181900029A059BD3180A7829
:10A944001A70059B01330593059A019B9A42EFD334
:0CA954000023180006B07047E075FF1FDC
:10A9600000B583B0184B1B689A02FF239B0213406B
:10A97000164A944663446A46D11D01221800FFF727
:10A98000C1FF031E01D003231AE06B4607331B7877
:10A99000FF2B05D10E4B180002F096FF00230FE0AD
:10A9A0006B4607331B78362B05D10A4B180002F093
:10A9B0008BFF012304E0084B180002F085FF0223FF
:10A9C000180003B000BDC046E075FF1F00F8FF0788
:0CA9D0002C000108440001086C00010884
:10A9DC0000B587B00190964B180002F06FFF954BB5
:10A9EC0003939623DA01039B5A610022039B1A837B
:10A9FC000122039B5A830122039B9A830022039B0F
:10AA0C00DA840022039B1A850022039B5A850022BC
:10AA1C00039B9A850022039BDA850022039B1A86EE
:10AA2C000022039B5A860022039B5A630022039B3D
:10AA3C009A630022039BDA630022039B1A647E4A0A
:10AA4C00039B5A640022039B9A640022039BDA64E2
:10AA5C000022039B1A65794A039B5A656321039B69
:10AA6C00582299526921039B5A229952744A039B8A
:10AA7C00DA65744A039B1A660A21039B6422995275
:10AA8C000221039B662299526F49039B68229952BB
:10AA9C006E49039B6A2299520021039B6C229954A4
:10AAAC000221039B6E229952AF239901039B7022C2
:10AABC0099526749039B722299526649039B7422EF
:10AACC0099526549039B76229952FA235942039B6A
:10AADC0078229952FA21039B7A2299525F49039B5F
:10AAEC007C2299525E49039B7E2299525D49039BBD
:10AAFC00802299525C49039B822299525749039BAD
:10AB0C00842299525649039B862299525549039B9C
:10AB1C00882299525449039B8A2299523221039BD1
:10AB2C008C229952C8235942039B8E2299524F4929
:10AB3C00039B902299520721039B92229952002148
:10AB4C00039B942299500021039B982299505A21DF
:10AB5C00039B9C2299520021039BA0229950039B9A
:10AB6C009B685A1C039B9A60039BA4229A80039BAC
:10AB7C000022DA80039B36221A70F9F76BFCFA2359
:10AB8C009B001800F9F7ECFC394B5B690122134070
:10AB9C0005D0374B5A69364B01218A435A61354BE4
:10ABAC0002221A60334B3F225A60324B01229A60C8
:10ABBC0002AA304B11001800F9F758FD031E00D003
:10ABCC00FEE72D4B1B689A02FF239B0213402B4A76
:10ABDC009446634405930023049313E0154A049BA5
:10ABEC00DB00D3181A685B6805990120F9F7DCFBC8
:10ABFC00031E06D1059B08330593049B0133049374
:10AC0C0000E0FEE71C4B1B689A02FF239B021340DB
:10AC1C001B4A94466344059A9A42DFD3F9F73EFCEB
:10AC2C00019B180000F096FB0300180007B000BD54
:10AC3C00900001085802002090D0030040420F0001
:10AC4C00A086010080482800B0360000302C00009F
:10AC5C00E02E000060EA0000C0DA00004C1D00008D
:10AC6C00581B000054F2FFFF48F4FFFF10270000B0
:10AC7C0000200240980B0020E075FF1F00F8FF0732
:04AC8C00A4F8FF0722
:10AC900000B587B00190AB4B180002F015FEAA4B2F
:10ACA0000393019B180000F05BFB019B9A6F039BD1
:10ACB0001A65019B7C229B5A1AB2039BDA84019B82
:10ACC0007E229B5A1AB2039B1A85019B80229A58B6
:10ACD000039B5A63019B84229A58039B9A63019BAE
:10ACE00088229A58039BDA63019B8C229B5A1AB2E2
:10ACF000039BDA85019B90229A58039B1A64019B5F
:10AD000094229B581A00039B5A65019B98229B5AD8
:10AD10001AB2039B5A85019B9A229B5A1AB2039B33
:10AD20009A85019B9C229A58039B5A64019BA022FE
:10AD30009B5A1AB2039B1A86019BA4229A58039B22
:10AD40009A64019BA8229B5A1AB2039B5A86019BC4
:10AD5000AC229A58039BDA649623DA01039B5A616A
:10AD60000022039B1A830122039B5A830122039B27
:10AD70009A830022039BDA830022039B1A84002219
:10AD8000039B5A840022039B9A846321039B5822CD
:10AD900099526E4A039BDA656D4A039B1A660A2133
:10ADA000039B642299526921039B5A2299520221E2
:10ADB000039B662299526749039B68229952664910
:10ADC000039B6A2299520021039B6C229954022111
:10ADD000039B6E229952AF239901039B70229952D3
:10ADE0005E49039B722299525D49039B74229952DA
:10ADF0005C49039B76229952FA235942039B78229D
:10AE00009952FA21039B7A2299525749039B7C223B
:10AE100099525649039B7E2299525549039B8022A1
:10AE200099525449039B822299524F49039B842291
:10AE300099524E49039B862299524D49039B882281
:10AE400099524C49039B8A2299523221039B8C22AE
:10AE50009952C8235942039B8E2299524649039B1B
:10AE6000902299520721039B922299520021039B21
:10AE7000942299500021039B982299505A21039BB8
:10AE80009C2299520021039BA0229950F9F7E8FADD
:10AE9000FA239B001800F9F769FB384B5B69012224
:10AEA000134005D0354B5A69344B01218A435A610E
:10AEB000334B02221A60324B3F225A60304B012240
:10AEC0009A6002AA2E4B11001800F9F7D5FB031E59
:10AED00000D0FEE72B4B1B689A02FF239B02134016
:10AEE000294A9446634405930023049313E0164AC9
:10AEF000049BDB00D3181A685B6805990120F9F7F9
:10AF000059FA031E06D1059B08330593049B0133B0
:10AF1000049300E0FEE71B4B1B689A02FF239B0291
:10AF200013401A4A94466344059A9A42DFD3F9F7CC
:10AF3000BBFA019B180000F013FA0300180007B0D9
:10AF400000BDC046A800010858020020A0860100EC
:10AF500080482800B0360000302C0000E02E0000B1
:10AF600060EA0000C0DA00004C1D0000581B000021
:10AF700054F2FFFF48F4FFFF1027000000200240BA
:10AF8000980B0020E075FF1F00F8FF07A4F8FF07EB
:10AF900000B587B001900A006B4603331A70DC4B92
:10AFA000180002F091FCDB4B0393019B1A69039B91
:10AFB0005A61019B9B8A9AB2039B1A83019BDB8A8D
:10AFC0009AB2039B5A83019B1B8B9AB2039B9A8371
:10AFD000019B9B8B9AB2039BDA83019BDB8B9AB21A
:10AFE000039B1A84019B1B8C9AB2039B5A84019B7E
:10AFF0005B8C9AB2039B9A84019B7E229B5A1AB265
:10B00000039B1A85019B7C229B5A1AB2039BDA840C
:10B01000019B98229B5A1AB2039B5A85019B9A2244
:10B020009B5A1AB2039B9A85019B8C229B5A1AB297
:10B03000039BDA85019BA0229B5A1AB2039B1A86B6
:10B04000019BA8229B5A1AB2039B5A86019B80221D
:10B050009A58039B5A63019B84229A58039B9A63D4
:10B06000019B88229A58039BDA63019B90229A588D
:10B07000039B1A64019B9C229A58039B5A64019B70
:10B08000A4229A58039B9A64019BAC229A58039B72
:10B09000DA64019B9A6F039B1A65019B94229B586B
:10B0A0001A00039B5A65019B52229B5A99B2039B3B
:10B0B00058229952019B50229B5A99B2039B5A22C3
:10B0C0009952019BDA6D039BDA65019B1A6E039B13
:10B0D0001A66019B54229B5A99B2039B642299528F
:10B0E000019B56229B5A99B2039B66229952019B5F
:10B0F00058229B5A99B2039B68229952019B5A226B
:10B100009B5A99B2039B6A229952019B64229B5AD3
:10B110009BB2D9B2039B6C229954019B68229B5A23
:10B1200099B2039B6E229952019B9B8E99B2039B0D
:10B1300070229952019BDB8E99B2039B7222995225
:10B14000019B1B8F99B2039B74229952019B5B8FC9
:10B1500099B2039B76229952019B9B8F19B2039B54
:10B1600078229952019BDB8F19B2039B7A22995264
:10B17000019B40229B5A19B2039B7C229952019B4E
:10B1800042229B5A19B2039B7E229952019B442270
:10B190009B5A19B2039B80229952019B46229B5ACB
:10B1A00019B2039B82229952019B48229B5A19B2E1
:10B1B000039B84229952019B4A229B5A19B2039BFA
:10B1C00086229952019B4C229B5A19B2039B8822DA
:10B1D0009952019B4E229B5A19B2039B8A22995283
:10B1E000019B6A229B5A19B2039B8C229952019BA4
:10B1F0006C229B5A19B2039B8E229952019B6E229C
:10B200009B5A99B2039B90229952019B70229B5AA0
:10B2100019B2039B92229952019A96235B00D2584D
:10B22000039B94215A50019A98235B00D258039BA8
:10B2300098215A50019B72229B5A99B2039B9C22DF
:10B240009952039B9B68591C039A9160019994221F
:10B2500052008B50039AA0215350039BA4229A8042
:10B26000039B0022DA80039B36221A706B4603335D
:10B270001B78002B07D0284B180002F025FB019B00
:10B280005A68039BDA60F9F7EBF8FA239B00180081
:10B29000F9F76CF9214B5B690122134005D01F4B74
:10B2A0005A691E4B01218A435A611D4B02221A60C2
:10B2B0001B4B3F225A601A4B01229A6002AA184B7C
:10B2C00011001800F9F7D8F9031E00D0FEE7154B5E
:10B2D0001B689A02FF239B021340134A944663445F
:10B2E00005930023049321E00A4A049BDB00D31852
:10B2F0001A685B6805990120F9F75CF8031E06D10E
:10B30000059B08330593049B013304930EE0FEE78D
:10B31000C000010858020020D800010800200240A7
:10B32000980B0020E075FF1F00F8FF070A4B1B6811
:10B330009A02FF239B021340084A94466344059AED
:10B340009A42D1D3F9F7B0F8019B180000F008F841
:10B350000300180007B000BDE075FF1FA4F8FF0749
:10B3600000B585B00190B14B1B689A02FF239B0288
:10B370001340AF4A94466344AE49A8221800FFF731
:10B38000C1FA031E01D001234CE1AA4B0393039B96
:10B390005A69019B1A61039B1A8B019B9A82039B3A
:10B3A0005A8B019BDA82039B9A8B019B1A83039B26
:10B3B000DA8B019B9A83039B1A8C019BDA83039B94
:10B3C0005A8C019B1A84039B9A8C019B5A84039B81
:10B3D0002621595E019B7C229952039B2821595EAC
:10B3E000019B7E229952039B2A21595E019B982240
:10B3F0009952039B2C21595E019B9A229952039BDF
:10B400002E21595E019B8C229952039B3021595E5B
:10B41000019BA0229952039B3221595E019BA822D5
:10B420009952039B5A6B019B80215A50039B9A6B44
:10B43000019B84215A50039BDA6B019B88215A504F
:10B44000039B1A6C019B90215A50039B5A6C019BE1
:10B450009C215A50039B9A6C019BA4215A50039B38
:10B46000DA6C019BAC215A50039B1A6D019B9A67C1
:10B47000039B5B6D1900019B94229950039B5822FA
:10B48000995A019B52229952039B5A22995A019B25
:10B4900050229952039BDA6D019BDA65039B1A6E69
:10B4A000019B1A66039B6422995A019B542299526C
:10B4B000039B6622995A019B56229952039B68224C
:10B4C000995A019B58229952039B6A22995A019BCF
:10B4D0005A229952039B6C229B5C1900019B6422A7
:10B4E0009952039B6E22995A019B68229952039BA1
:10B4F00070229A5A019B9A86039B72229A5A019B48
:10B50000DA86039B74229A5A019B1A87039B762240
:10B510009A5A019B5A87039B78229A5E019B9A87CD
:10B52000039B7A229A5E019BDA87039B7C22995EB9
:10B53000019B40229952039B7E22995E019B4222ED
:10B540009952039B8022995E019B44229952039B4E
:10B550008222995E019B46229952039B8422995E26
:10B56000019B48229952039B8622995E019B4A22A5
:10B570009952039B8822995E019B4C229952039B0E
:10B580008A22995E019B4E229952039B8C22995EDE
:10B59000019B6A229952039B8E22995E019B6C2229
:10B5A0009952039B9022995A019B6E229952039BB8
:10B5B0009222995E019B70229952039B9422995882
:10B5C000019A96235B00D150039B98229958019AC7
:10B5D00098235B00D150039B9C22995A019B7222B5
:10B5E0009952039BDB68019A5360039AA021535040
:10B5F000039BA0229958019A94235B00D150039B8E
:10B600009B88A42B01D001230CE0039BDB88002B3B
:10B6100001D0012306E0039B1B78362B01D00123C8
:10B6200000E00023180005B000BDC046E075FF1F14
:08B6300000F8FF07580200209A
:10B6380030B591B09D4A94235B00D3589AB29C4B85
:10B648001B689BB2D31A99B2984ACB235B00D1529C
:10B6580013230F9314E00F9B5A1E964B9200D15858
:10B66800944B0F9A9200D1500F9B5A1E924B920006
:10B67800D158914B0F9A9200D1500F9B013B0F93D9
:10B688000F9B002BE7DC894BE4229A58894B1A6000
:10B69800864BD8229A58884B1A60884B0E93002301
:10B6A8000D93864B0C9300230B9301235B42089365
:10B6B80001235B42079301235B42069301235B420C
:10B6C800059300230F9352E07A4B0F9A9200D358B8
:10B6D800DA179B1853400C9A9A4209DD754B0F9A5A
:10B6E8009200D358DA179B1853400C930F9B08937A
:10B6F800704B0F9A9200D358DA179B1853400B9A45
:10B708009A4209DC6B4B0F9A9200D358DA179B18B0
:10B7180053400B930F9B0793674B0F9A9200D35894
:10B72800DA179B1853400E9A9A4209DD624B0F9A1A
:10B738009200D358DA179B1853400E930F9B069329
:10B748005D4B0F9A9200D358DA179B1853400D9A05
:10B758009A4209DA584B0F9A9200D358DA179B1875
:10B7680053400D930F9B05930F9B01330F930F9B32
:10B77800132BA9DD0B9A0C9BD31ADA179B1853408D
:10B7880004930D9A0E9BD31ADA179B185340039310
:10B79800464BDA6D454B68215B5A9BB21900100085
:10B7A80003F0C2F903000293029B1421180003F06E
:10B7B80093F90300029305230193049A029B9A428A
:10B7C80002DA01235B426EE0039A019B9A4202DA95
:10B7D80002235B4267E001235B420A9301235B4239
:10B7E800009301235B42099300230F9318E00F9BFA
:10B7F8005A1C304B9200D2582E4B0F998900CB58C7
:10B80800D31ADA179B1853400093009A0A9B9A425E
:10B8180003DD009B0A930F9B09930F9B01330F9342
:10B828000F9B122BE3DD099B0A2B3BD1039803F0F6
:10B8380051F804000D00049803F04CF802000B00C6
:10B848002000290002F0B4FE02000B0010001900CD
:10B8580000221B4B05F025FA02000B00100019000E
:10B8680002F082FF030019B2104A8E235B00D15206
:10B878000E4A94235B00D3581A000D4B1A6000231C
:10B888000F9302E00F9B01330F930F9B132BF9DDEE
:10B89800064A8E235B00D35A1BB2039A04990948BF
:10B8A80003F00EFA0023180011B030BDB0000020DC
:10B8B800DC0B0020A40A0020540A0020FFFFFF7FB1
:08B8C8000088C34008020108DA
:10B8D00000B587B001900091354B1B68354A934203
:10B8E00004D0334B1B685A1C314B1A60324B1A6818
:10B8F000314B1B689B09D21A2F4B1A602E4B1A68CA
:10B90000019BD2182C4B1A602B4B1B689B0905938B
:10B910002A4B1A68294B1B689B09D21A274B1A60BD
:10B92000264B1A68009BD218244B1A60234B1B68C5
:10B930009B090493059A049BD31A180002F0CEFFCA
:10B9400002000B00029203931D4BCA229B5A9BB22A
:10B95000180002F0C3FF029A039B05F0A6F902004B
:10B960000B00100019000022164B02F025FE020009
:10B970000B00029203930022134B0298039902F0EA
:10B980001BFE02000B0010001900104A104B02F0C1
:10B9900013FE02000B001000190002F0E9FE010086
:10B9A000074AC8235B00D150C04607B000BDC0465F
:10B9B000C40B0020FFFFFF7FFC0B0020040C0020C5
:10B9C000B00000200000F04000004440FCA9F1D28B
:04B9D0004D62203F65
:10B9D40000B58BB005AB180014231A00002104F045
:10B9E40013F9594B5A6B584B02210A435A63564B6D
:10B9F4005B6B022213400493049B534B5A6B524BD0
:10BA040004210A435A63504B5B6B04221340039393
:10BA1400039B4D4B5A6B4C4B20210A435A634A4BB0
:10BA24005B6B202213400293029B474B5A6B464B9D
:10BA340001210A435A63444B5B6B01221340019377
:10BA4400019BF9235901A023DB050022180004F00F
:10BA5400CFFE3E4B00221021180004F0C9FE8023C3
:10BA64005B003A480022190004F0C2FE05AB8022B4
:10BA740092001A6005AB364A5A6005AB01229A60FF
:10BA840005AB324A19001000F8F7A6FF05ABF922FE
:10BA940052011A6005AB01225A6005AB00229A607C
:10BAA40005AB0022DA6005AAA023DB05110018000B
:10BAB400F8F792FF05AB40221A6005AB00225A60EA
:10BAC40005AB01229A6005AB224A19001000F8F771
:10BAD40083FF05AB802252001A6005AB01225A6035
:10BAE40005AB00229A6005AB0022DA6005AB174A69
:10BAF40019001000F8F770FF05AB10221A6005ABAF
:10BB040001225A6005AB01229A6005AB0022DA607B
:10BB140005AB0E4A19001000F8F75EFF05AB2022B2
:10BB24001A6005AB01225A6005AB01229A6005AB8D
:10BB34000022DA6005AB054A19001000F8F74CFF43
:10BB4400C0460BB000BDC0460010024000040050C7
:08BB5400000021100008005060
:10BB5C00BFF34F8FC046044B044ADA60BFF34F8FDC
:10BB6C00C046C046C046FCE700ED00E00400FA0504
:10BB7C00F0B5C64600B58EB000230D930023069396
:10BB8C0000230C9300230B930023059300230A93AB
:10BB9C000023099313236B4400221A7023236B4454
:10BBAC0000221A7000F02CFCF7F70CFB00F058FA8E
:10BBBC00DB4B180001F082FEFCF742FCFCF792FB19
:10BBCC00FCF72EFBFFF700FFFEF77AFE01F0D0F832
:10BBDC00FDF7F0F900F0F2FE12236B449846FEF7E5
:10BBEC00B9FE03004246137012236B441B789AB2C1
:10BBFC00CC4B5A8012236B441B78032B17D01BDCC5
:10BC0C00022B0FD018DC002B02D0012B05D013E037
:10BC1C00C44B1800FEF7DCFE0EE0C24B1800FFF719
:10BC2C0099FB09E0BF4B1800FFF72CF804E0BD4B63
:10BC3C001800FFF78FFBC046BB4B180001F03EFE0F
:10BC4C00B84B1800FFF786FB01F088F9B74B402181
:10BC5C00180005F076FA031E11D13220F7F730FBED
:10BC6C00B24B4021180005F06CFA031E07D1B04B03
:10BC7C00180001F023FEAB4B1800FFF703F8A94B9B
:10BC8C001969A84B9B8A9BB29C46A64BDB8A9AB23D
:10BC9C00A848A94B00931300624604F0CAFEFEF7B5
:10BCAC0037FDA64B1800F8F77BF8A549A34B0822E3
:10BCBC001800F7F75DFD00F071FA6420F7F700FB50
:10BCCC00FEF74EF89F4B180001F0F8FD00F0DCFB7E
:10BCDC00002307931CE080231901A023DB0501221C
:10BCEC00180004F081FDAF235B001800F7F7E8FAA9
:10BCFC0080231901A023DB050022180004F074FD39
:10BD0C00AF235B001800F7F7DBFA079B01330793AF
:10BD1C00844B1B8B9BB21A00079B9342DBDB8A4B39
:10BD2C001B68012B48D1884B00221A60844B5B693D
:10BD3C00180000F00BFE824B1B68180000F0E4FFAB
:10BD4C007F4BDB691800FEF731FD7D4B9B691800BA
:10BD5C0000F08CFF7A4B5A68794B9B6819001000E5
:10BD6C00FEF730FC764BDA68754B1B691900100036
:10BD7C00FFF7A8FD6B4BD8229B581C00DB171D004E
:10BD8C00684BE4229B581E00DB171F0032003B005F
:10BD9C002000290002F086FE02000B0010001900A2
:10BDAC00FA229200002302F0E1FE02000B001100C7
:10BDBC005C4A84235B00D150644B1B68012B04D17B
:10BDCC00FFF734FC614B00221A60F7F773FA03009B
:10BDDC000693069A0D9BD31A0393069B0D930C9A0C
:10BDEC00039BD3180C930B9A039BD3180B93099BAF
:10BDFC00002B05DD039B002B02D0099B013B099313
:10BE0C00534B1B681B68DAB213236B440F210A4097
:10BE1C001A704F4B1B685B68029323226A441323EE
:10BE2C006B4412781B789A422BD023236B44132239
:10BE3C006A4412781A703B4A94235B00D358591CFD
:10BE4C00384A94235B00D1500A9B002B07D18023E6
:10BE5C00DA00A023DB051100180004F0E4FCFEF767
:10BE6C00FBF801F0F7F900F01FFB00F045FC00F0C7
:10BE7C0069F900F031FE030019002A4ACC235B005B
:10BE8C00D152284B5B8B9BB2002B00D19AE0294BF3
:10BE9C0026229B5C002B00D094E0224B5B8B9BB248
:10BEAC002C4A93425ED02B4A934200DD83E0FD2264
:10BEBC009200934200D17BE0FD229200934200DD80
:10BECC0079E0254A934200D16EE0FD229200934224
:10BEDC0000DB70E00B2B09DC002B00DC6BE00B2B88
:10BEEC0069D89A001D4BD3181B689F461C4A934275
:10BEFC0056D060E00B4B00211800FFF743F85EE0D2
:10BF0C00084B1800FEF764FD59E0064B1800FEF7CD
:10BF1C00B9FE54E0034B1800FFF71CFA4FE0C04683
:10BF2C007C020108B00000209002010800080050BB
:10BF3C00A0020108480300202408002094090020D6
:10BF4C00600B0020B4020108B40B0020B00B0020E1
:10BF5C00340B0020D2040000F30300002CFC00087A
:10BF6C00F2030000394B01211800FFF70BF826E013
:10BF7C00FFF7EEFD23E0354B1800FDF761FB1EE0EB
:10BF8C00324B1800FDF784FB19E0FDF7B3FB16E00C
:10BF9C002E4B1800FDF7E2FB11E0FDF793FC0EE0D1
:10BFAC00002000F007F90AE0012000F003F906E098
:10BFBC0000F0C4F903E0264B180001F07FFC234B82
:10BFCC0000225A83234B4021180005F0BAF8031EB7
:10BFDC001FD1099B002B1CD10A20F7F771F91D4BBF
:10BFEC004021180005F0ADF8031E12D1FA235B00B6
:10BFFC0009930A9B002B0AD101230A938023D900B1
:10C00C00A023DB050122180004F0EEFB01E0002365
:10C01C000A93114B180005F05CFA031E00D17EE662
:10C02C000D4B1800FCF7ECFD0300022B08D10A9B0A
:10C03C00002B00D073E6084B180004F0A0FD6EE650
:10C04C00064B84222221995069E6C046B00000209C
:10C05C00C4020108000800504803002024080020F6
:10C06C0000B599B00BAB180034231A00002103F073
:10C07C00C7FD07AB180010231A00002103F0C0FD08
:10C08C006B4618001C231A00002103F0B9FD802315
:10C09C009B001800F8F746FEF8F72CFE274BDA6DDC
:10C0AC00264B18210A43DA65F8F730FE0BAB062253
:10C0BC001A600BAB01229A600BAB80225200DA6043
:10C0CC000BAB00221A610BAB40225A610BAB002266
:10C0DC00DA610BAB1800F8F76DFE031E01D005F00A
:10C0EC00E2FA07AB07221A6007AB00225A6007ABD3
:10C0FC0000229A6007AB0022DA6007AB002118001F
:10C10C00F9F76CF9031E01D005F0CDFA6B460C4A19
:10C11C001A606B4600225A606B4600225A616B46CD
:10C12C00802252009A616B461800F9F7F7FA031E49
:10C13C0001D005F0B8FAC04619B000BD001002409D
:04C14C0001400200AC
:10C1500000B583B00C4A94235B00D3580B491800F8
:10C1600002F0E6FC03000193094B1B68019A9A4216
:10C1700007D0074B019A1A60034B00211800FEF705
:10C1800007FFC04603B000BDB00000208051010091
:04C19000E00B0020A0
:10C1940082B00190024B01221A60C04602B070477F
:04C1A400B40B0020B8
:10C1A80010B580235B0003480122190004F01EFB30
:08C1B800C04610BD0004005058
:10C1C00000B58BB002006B4607331A7003AB180042
:10C1D0001C231A00002103F019FD03AB1800F8F727
:10C1E00037FB6B4607331B78002B45D0484B1800B4
:10C1F00001F06AFB03AB1B69AA2B38D103AB022207
:10C200001A6003ABBB221A61F8F72AF9031E03D0A8
:10C21000404B180001F058FBF8F762F9031E03D0F9
:10C220003D4B180001F050FB3C4B180001F04CFB5B
:10C2300003AB1800F8F78AFA031E07D0384B180032
:10C2400001F042FBF8F774F900235EE0F8F770F9AB
:10C25000344B180001F038FBF8F726F9324B180080
:10C2600001F032FB314B180001F02EFB4CE0304B5B
:10C27000180001F029FB47E003AB1B69BB2B43D13E
:10C2800003AB02221A6003ABAA221A61F8F7E8F89E
:10C29000031E05D01F4B180001F016FB002334E0ED
:10C2A000244B180001F010FBF8F71AF9031E05D013
:10C2B000194B180001F008FB002326E01E4B180064
:10C2C00001F002FB03AB1800F8F740FA031E07D099
:10C2D000F8F72EF9194B180001F0F6FA002314E0D4
:10C2E000174B180001F0F0FAF8F722F90D4B18007F
:10C2F00001F0EAFAF8F7D8F80B4B180001F0E4FA6D
:10C30000104B180001F0E0FA012318000BB000BD3B
:10C31000D4020108F40201080803010820030108FF
:10C320003003010848030108600301087003010895
:10C3300090030108B0030108C4030108DC030108ED
:08C34000000401081C040108BF
:10C3480000B589B001AB18001C231A00002103F0C6
:10C3580059FC01AB1800F8F777FA01AB06221A600E
:10C3680001AB06221A6001ABBB221A6101ABE022C5
:10C37800D2045A6101ABA022D2049A61F8F76CF892
:10C38800031E03D0184B180001F09AFAF8F7A4F826
:10C39800031E03D0154B180001F092FA144B180035
:10C3A80001F08EFA01AB1800F8F7CCF9031E07D09C
:10C3B800104B180001F084FAF8F7B6F8002310E0E3
:10C3C800F8F7B2F80C4B180001F07AFAF8F768F8A9
:10C3D8000A4B180001F074FA094B180001F070FAC2
:10C3E8000123180009B000BDF40201080803010880
:10C3F800200301083003010848030108600301080D
:04C4080070030108B4
:10C40C0000B589B06B4618001C231A00002103F0FC
:10C41C00F7FB6B461800F8F715FA1F236B44002244
:10C42C001A706B461B69AA2B08D1144B180001F02B
:10C43C0045FA1F236B4400221A7018E06B461B69E7
:10C44C00BB2B08D10E4B180001F038FA1F236B449C
:10C45C0001221A700BE06B461B69CC2B07D1094BE0
:10C46C00180001F02BFA1F236B4402221A701F23B1
:10C47C006B441B78180009B000BDC046400401088D
:08C48C005C04010878040108BA
:10C49400064A83235B0001214942D152034A822385
:10C4A4005B0001214942D152C0467047B0000020D0
:10C4B40010B58C4A83235B00D35A1BB2002B07D0E0
:10C4C400884A83235B00D35A1BB2013300D0A9E00E
:10C4D400844BD8229B58834A928E92B2934211DAAB
:10C4E400814B180001F0EEF97E4A83235B000121A1
:10C4F400D15280239900A023DB050022180004F008
:10C5040077F98FE0774BE4229958764B9B8F1BB2D7
:10C514001A0013005B019B1A9B009B18DB009942D5
:10C5240011DA724B180001F0CDF96E4A83235B00D7
:10C534000221D15280239900A023DB050022180098
:10C5440004F056F96EE0674BCE229B5A1AB2654B43
:10C5540048215B5A1BB29A4211DD654B180001F069
:10C56400B1F9604A83235B000321D15280239900EF
:10C57400A023DB050022180004F03AF952E0594BDD
:10C58400CC229B5A1AB2574B48215B5A1BB29A428F
:10C5940011DD584B180001F095F9524A83235B00D2
:10C5A4000421D15280239900A023DB050022180026
:10C5B40004F01EF936E04B4BCE229B5A1AB2494B7B
:10C5C4004C215B5A1BB29A4211DA4B4B180001F012
:10C5D40079F9444A83235B000521D15280239900D1
:10C5E400A023DB050022180004F002F91AE03D4BF9
:10C5F400CC229B5A1AB23B4B4C215B5A1BB29A4237
:10C6040010DA3C4B180001F05DF9364A83235B00D5
:10C614000621D15280239900A023DB0500221800B3
:10C6240004F0E6F82F4A83235B00D35A1BB2002B95
:10C6340056D02C4BD8229B582A4AD28E92B293427F
:10C644004EDD284BE4229958264B9B8F1BB21A00CF
:10C6540013005B019B1A9B009B18DB0099423FDD92
:10C66400204BCE229B5A1AB21E4B4A215B5A1BB254
:10C674009A4235DA1B4BCC229B5A1AB2194B4A21E7
:10C684005B5A1BB29A422BDA164BCE229B5A1AB231
:10C69400144B4E215B5A1BB29A4221DD114BCC2222
:10C6A4009B5A1AB20F4B4E215B5A1BB29A4217DDAA
:10C6B4000C4A83235B00D35A1BB2022B10D00F4BBE
:10C6C400180001F0FFF8074A83235B000021D152D0
:10C6D40080239900A023DB050122180004F088F8C8
:10C6E400C04610BDB0000020C4040108E8040108DD
:10C6F4000005010824050108480501086C05010826
:10C7040010B58C4A82235B00D35A1BB2002B07D08E
:10C71400884A82235B00D35A1BB2013300D0A9E0BC
:10C72400844BD8229B58834A128F92B2934211DDD4
:10C73400814B180001F0C6F87E4A82235B00012178
:10C74400D15280235900A023DB050022180004F0F5
:10C754004FF88FE0774BE4229958764BDB8F1BB26E
:10C764001A0013005B019B1A9B009B18DB00994283
:10C7740011DD724B180001F0A5F86E4A82235B00AC
:10C784000221D15280235900A023DB050022180086
:10C7940004F02EF86EE0674BCE229B5A1AB2654B1A
:10C7A40040215B5A1BB29A4211DD654B180001F01F
:10C7B40089F8604A82235B000321D1528023590007
:10C7C400A023DB050022180004F012F852E0594BB4
:10C7D400CC229B5A1AB2574B40215B5A1BB29A4245
:10C7E40011DD584B180001F06DF8524A82235B00AA
:10C7F4000421D15280235900A023DB050022180014
:10C8040003F0F6FF36E04B4BCE229B5A1AB2494B4B
:10C8140044215B5A1BB29A4211DA4B4B180001F0C7
:10C8240051F8444A82235B000521D15280235900E8
:10C83400A023DB050022180003F0DAFF1AE03D4BC9
:10C84400CC229B5A1AB23B4B44215B5A1BB29A42EC
:10C8540010DA3E4B180001F035F8364A82235B00AB
:10C864000621D15280235900A023DB0500221800A1
:10C8740003F0BEFF2F4A82235B00D35A1BB2002B66
:10C8840056D02C4BD8229B582A4A528F92B29342AC
:10C894004EDA284BE4229958264BDB8F1BB21A0040
:10C8A40013005B019B1A9B009B18DB0099423FDA43
:10C8B400204BCE229B5A1AB21E4B42215B5A1BB20A
:10C8C4009A4235DA1B4BCC229B5A1AB2194B42219D
:10C8D4005B5A1BB29A422BDA164BCE229B5A1AB2DF
:10C8E400144B46215B5A1BB29A4221DD114BCC22D8
:10C8F4009B5A1AB20F4B46215B5A1BB29A4217DD60
:10C904000C4A82235B00D35A1BB2022B10D0104B6B
:10C91400180000F0D7FF074A82235B000021D152A0
:10C9240080235900A023DB050122180003F060FFD7
:10C93400C04610BDB00000207C0501089C0501081C
:10C94400B4050108D8050108FC0501082006010802
:04C95400440601088C
:10C9580000B585B00190154B1A68144B1B689B09EC
:10C96800D21A124B1A60114B1A68019BD2180F4B3E
:10C978001A600E4B1B689B090393039B0C4A534395
:10C988000C49180002F0D0F8030099B20A4BC822EB
:10C9980099520399094802F0C7F8030099B2064B67
:10C9A800CA229952C04605B000BDC0460C0C0020F2
:10C9B800E40C0000FFFF0000B000002048F4B70BB3
:10C9C80000B587B001AB180014231A00002103F04A
:10C9D80019F96B4600221A602C4B2D4A1A602B4B12
:10C9E80000229A60294B7F22DA60284BFF221A61C5
:10C9F800264B00225A61254B00229A61234B0022C4
:10CA0800DA61224B8022D2051A62204B00225A6238
:10CA18001E4B1800F8F7B8FF031E01D004F045FEBE
:10CA280001AB02221A7001AB00225A7001AB00223E
:10CA38009A7001AB00225A6001AB0022DA6001ABA8
:10CA480000221A6101A9114B01221800F9F732F8E6
:10CA5800031E01D004F029FE6B4601221A706B46B2
:10CA680004225A706B4616229A706B461822DA70A6
:10CA78006946064B01221800F9F7C4F8031E01D0D5
:10CA880004F013FEC04607B000BDC046340B0020BA
:04CA98000028004032
:10CA9C0084B00190019B1B680D4A934214D10D4B3D
:10CAAC00DA6B0C4B8021C9000A43DA63094BDA6B51
:10CABC008023DB0013400393039B064BDA6D054B7D
:10CACC00802109020A43DA65C04604B07047C046AB
:08CADC00002800400010024098
:10CAE40030B58BB05C4A5D4B0892099300225C4BD5
:10CAF400069207935B4B58229B5A9BB2180001F095
:10CB0400EBFE04000D000022574B0898099901F030
:10CB1400BFFB02000B002000290004F0C4F802004F
:10CB24000B001000190001F021FE030005934D4B8A
:10CB340058229B5A9BB2180001F0CEFE04000D004F
:10CB4400089A099B0020484901F086FC02000B006A
:10CB54002000290004F0A7F802000B0010001900BF
:10CB640001F004FE03000493404B1B6899B23D4A54
:10CB7400CD235B00D1523B4BD8229B580393039A9D
:10CB8400059B9A4205DD3A4B00221A6001235B4261
:10CB94005EE0039A049B9A4205DA354B00221A6040
:10CBA40001235B4254E0324B1B68002B02D1304B13
:10CBB400039A1A602E4B1B68180001F08DFE069A2A
:10CBC400079B01F065FB02000B001000190001F047
:10CBD400CDFD03000293264B1B68180001F07CFE78
:10CBE400069A079B01F038FC02000B0010001900A4
:10CBF40001F0BCFD03000193039A029B9A4208DDF5
:10CC04001B4B00221A60194B00221A6002235B425C
:10CC14001EE0039A019B9A4208DA154B00221A601F
:10CC2400124B00221A6002235B4211E00F4B1B6877
:10CC34005A1C0E4B1A600D4B1B683C2B07D9094B31
:10CC4400E4229B5819B2074A8C235B00D15200237B
:10CC540018000BB030BDC046B81E85EB51B89E3FDE
:10CC640000001440B00000200000F03FE40B00205E
:04CC7400A80B0020E9
:10CC780000B585B00190019B204A5343002B02DA8E
:10CC88001F4A944663441B140393039B1D4A94460E
:10CC980063440393039B642253430393039B0A2136
:10CCA800180001F019FF030019B2174BCE22995250
:10CCB800154BCE229B5A1AB2134BD0215B5A1BB28A
:10CCC8009A4207DD104BCE229B5A19B20E4BD02246
:10CCD800995210E00C4BCE229B5A1AB20A4BD22121
:10CCE8005B5A1BB29A4206DA074BCE229B5A19B2FC
:10CCF800054BD2229952C04605B000BDE40C000095
:0CCD0800FFFF0000A8FDFFFFB0000020AE
:10CD140000B585B00190154B1A68144B1B689B092C
:10CD2400D21A124B1A60114B1A68019BD2180F4B7E
:10CD34001A600E4B1B689B0903930D4BCA229B5A26
:10CD44009BB21A00039B5A4313005B009B18DA0042
:10CD5400D31A0849180001F0E9FE03001900044B36
:10CD6400D4229950C04605B000BDC046100C002026
:08CD7400B0000020FFFF0000E9
:10CD7C0010B51B4B1B4A1A60194B822252005A6089
:10CD8C00174B00229A60164BE022D200DA60144B4B
:10CD9C0000221A61124B01225A61114B8022D202DD
:10CDAC009A610F4B0822DA610D4B00221A620C4B70
:10CDBC0000225A620A4B00229A62094B0722DA625D
:10CDCC00074B00221A63064B00225A63044B1800CF
:10CDDC00F8F7ECFF031E01D004F065FCC04610BD53
:08CDEC00300900200030014075
:10CDF40000B58BB0019005AB180014231A00002174
:10CE040002F002FF019B1B681A4A93422FD11A4B6E
:10CE14001A6C194B802149010A431A64164B1A6C87
:10CE240080235B0113400493049B134B5A6B124BF6
:10CE340001210A435A63104B5B6B01221340039395
:10CE4400039B05ABF0221A6005AB02225A6005ABC6
:10CE540000229A6005AB0022DA6005AB00221A6159
:10CE640005AAA023DB0511001800F7F7B5FDC0469D
:0CCE74000BB000BD003001400010024077
:10CE800082B00E4B1A6C0D4B01210A431A640B4BF6
:10CE90001B6C012213400193019B084BDA6B074B7B
:10CEA000802149050A43DA63044BDA6B80235B0572
:10CEB00013400093009BC04602B070470010024030
:10CEC00000B583B0F6F7EEF9154B1B685A1C144BEE
:10CED0001A60144B0193124B1A68FA239B009A4272
:10CEE0001AD3F6F7EDF90200019B934214D20E4AD1
:10CEF00092235B00D358591C0B4A92235B00D150FC
:10CF0000094A90235B00D358591C074A90235B00C1
:10CF1000D150034B00221A60C04603B000BDC0468A
:0CCF2000B80B0020204E0000B0000020E4
:10CF2C0010B5034B1800F7F707F9C04610BDC04603
:04CF3C00F8090020D0
:10CF400010B5034B1800FBF7C9FCC04610BDC04626
:04CF50002408002091
:10CF540010B5034B1800F9F7D7FBC04610BDC04607
:04CF6400F40A0020AB
:10CF6800354B364A1A80344A92235B000021D1504F
:10CF7800314A90235B000021D1502F4A8A235B005D
:10CF880001214942D1522C4A86235B0001214942A2
:10CF9800D150294A88235B0001214942D150264AB1
:10CFA8008E235B0001214942D152234A8F235B0023
:10CFB80001214942D152204A8C235B000121494278
:10CFC800D1521D4A8D235B0001214942D1521A4B8F
:10CFD8001B6E5B421900184AB6235B00D150164BF2
:10CFE800DB6D5B421900144AB4235B00D150124B2D
:10CFF80002221A81104B00225A810F4B0F229A816C
:10D008000D4BE821802212065A500B4BEC220C499A
:10D018009950094BD0220B499952074BD2220A4901
:10D028009952054BDC2207499950034BE0220649E7
:10D038009950C0467047C046B0000020FF0100006C
:0CD04800FFFFFF7F0080FFFFFF7F000064
:10D05400024B034A9A60C0467047C04600ED00E0A8
:04D064000030000890
:10D0680000B587B03A4B9B6838221340202B11D06B
:10D0780049D8182B09D046D8082B02D0102B0ED02F
:10D0880041E0344B344A1A604FE0324BFA22D20165
:10D098001A604AE02F4B802212021A6045E02C4B9E
:10D0A800DB68032213400493294BDB681B09072222
:10D0B800134001330393049B032B06D1039926489D
:10D0C80001F032FD0300059305E00399234801F0C0
:10D0D8002BFD030005931E4BDB681B0A7F221A40B9
:10D0E800059B534305931A4BDB685B0F07221340DC
:10D0F800013302930299059801F016FD03001A0006
:10D10800144B1A6011E0124B1B68DB0A072213400C
:10D1180001229A40130001930199104801F004FD7F
:10D1280003001A000B4B1A60C046094B9B681B0A88
:10D138000F221A400A4B9200D3580093054B1A68E5
:10D14800009BDA40034B1A60C04607B000BDC046DA
:10D1580000100240AC00002000127A000024F40005
:04D168005CFC000863
:10D16C0000B58BB0019005AB180014231A000021F8
:10D17C0002F046FD019B1B68334A934260D1334B4E
:10D18C001A6C324B8021C9010A431A642F4B1A6C5A
:10D19C008023DB0113400493049B2C4B5A6B2B4BC9
:10D1AC0002210A435A63294B5B6B022213400393FF
:10D1BC00039B05AB08221A6005AB02225A6005AB33
:10D1CC0000229A6005AB0022DA6005AB04221A61DA
:10D1DC0005AB1F4A19001000F7F7FAFB05AB40220C
:10D1EC001A6005AB02225A6005AB01229A6005ABAE
:10D1FC000022DA6005AB00221A6105AB144A190053
:10D20C001000F7F7E5FB05AB80221A6005AB022294
:10D21C005A6005AB00229A6005AB0022DA6005ABC0
:10D22C0000221A6105AB0A4A19001000F7F7D0FB6F
:10D23C00002200211B2003F050FF1B2003F061FF94
:10D24C00C0460BB000BDC046003801400010024083
:04D25C00000400507A
:10D26000F0B591B0A04B1A685B68110019430DD15D
:10D270009E4A9A235B00D3589D4A53430093002350
:10D280000193994B0099019A19605A60994B1A6859
:10D290005B68110019430DD1944A9C235B00D3585D
:10D2A000934A5343029300230393924B0299039AA8
:10D2B00019605A608D4BE4229B58002B22DB8B4B6C
:10D2C00072229B5A9BB20F93884BE4229B580F9A71
:10D2D00053436421180001F003FC03001900834A42
:10D2E000BE235B00D150814B70229B5A19B27F4AFA
:10D2F000BE235B00D3580A00991A7C4ABE235B0008
:10D30000D15006E0794BF0229958784ABE235B0051
:10D31000D150764ABE235B00D3580C93DB170D9394
:10D32000724BD8229B580A93DB170B930A9A0B9BDC
:10D330000C980D9901F0BCFB02000B0010001900C5
:10D34000FA229200002301F017FC02000B00089261
:10D350000993664B1B6E069300230793E12212018B
:10D3600000230698079901F0A3FB02000B0004922A
:10D3700005935E4AB8235B00D31818685968089A69
:10D38000099B12184B415948B821490041180A60BD
:10D390004B60594B18685968089A099B12184B4101
:10D3A00055490A604B60544B18685968E1221201D4
:10D3B000002301F0E1FB02000B0011004B4AB623F1
:10D3C0005B00D150494AB8235B00D3181A685B68E8
:10D3D0000599994205DB059999420AD10499914230
:10D3E00007D2424AB8235B00D118049A059B0A6011
:10D3F0004B60414B1A685B68002B02DC06D1002AA7
:10D4000004D03D49002200230A604B60374AB8230C
:10D410005B00D31818685968E1221201002301F05B
:10D42000ABFB02000B001100304ABC235B00D15063
:10D430002E4A84235B00D358002B35DA2B4A8423F1
:10D440005B00D3585B421E00DB171F00264B1A6897
:10D450005B6892197B4124490A604B60224B186833
:10D460005968234A002301F09FFB02000B001100C2
:10D470001E4A9A235B00D1501C4A96235B00D25867
:10D4800013005B019B1A9B009B18DB001A00174BD3
:10D49000DB6D1900100001F04BFB030099B2134A39
:10D4A0009E235B00D1521CE0104A84235B00D358BA
:10D4B0001C00DB171D000F4B1A685B6812196B41CB
:10D4C0000C490A604B600B4B18685968084A0023E6
:10D4D00001F06AFB02000B001100044A9C235B0070
:10D4E000D150C04611B0F0BD08030020B0000020AC
:0CD4F00080EE360018030020200300200E
:10D4FC0010B50C4AB6235B00D358002B04DB094A49
:10D50C00B6235B00D35804E0064AB6235B00D3581D
:10D51C005B420449882252008B5000F073F9C046DC
:08D52C0010BDC046B000002054
:10D5340000B587B01B4B1B6E029300230393E122BB
:10D54400120100230298039901F0B0FA02000B00C3
:10D55400009201930022002304920593009B019AF8
:10D56400134316D00F4AB8235B00D31818685968C0
:10D574000D4A002301F09AFA02000B001000190072
:10D58400009A019B01F0F6FA02000B000492059345
:10D5940003E00022002304920593049B180007B0C3
:0CD5A40000BDC046B0000020A0860100C1
:10D5B000F0B587B03F480021029003913E48B62164
:10D5C00049004158002908DA3B48B6214900415832
:10D5D00049420A00C9170B0001E000220023009213
:10D5E00001930022002304920593334A88235B00B1
:10D5F000D358002B1DDC009A019B0298039901F07F
:10D6000057FA02000B00100019002B4B1B6E1E0076
:10D6100000231F0032003B0001F0AEFA02000B00B5
:10D6200010001900029A039B121A8B410492059371
:10D630001EE0009A019B0298039901F039FA02005A
:10D640000B00100019001C4A88235B00D3581C00F3
:10D65000DB171D0022002B0001F08EFA02000B00E8
:10D6600010001900029A039B121A8B410492059331
:10D67000059A039B9A4207DC059A039B9A4208D1BC
:10D68000049A029B9A4204D9029A039B049205933E
:10D690000CE0059B002B09DC059B002B02D1049BB1
:10D6A000002B03D10022002304920593049B180051
:0CD6B00007B0F0BDA0860100B000002013
:10D6BC00F0B58BB03B4A00230492059300230993E9
:10D6CC00394A88235B00D358002B0ADC364BDB6DC0
:10D6DC003549B42252008A589B18069300230793AD
:10D6EC000BE0314A86235B00D2582F49B4235B00F0
:10D6FC00CB58D3180693DB1707932B4BD8229B5888
:10D70C002949C02252008A5A92B29B18002B00DA87
:10D71C0001335B100293DB170393029A039B069869
:10D72C00079901F0BFF902000B0010001900FA2252
:10D73C009200002301F01AFA02000B0000920193F0
:10D74C00009A019B0498059901F0ACF902000B00BA
:10D75C0010001900144A88235B00D3581E00DB17F5
:10D76C001F0032003B0001F001FA02000B00130015
:10D77C000993099B1C00DB171D00059BAB4205DBC5
:10D78C00059BAB4205D1049BA34202D2049B099397
:10D79C0004E0099B002B01DC00230993099B180072
:0CD7AC000BB0F0BDA0860100B000002012
:10D7B80000B585B0124B1B6E029300230393E12240
:10D7C800120100230298039901F06EF902000B0080
:10D7D800009201930A4AB8235B00D118009A019B72
:10D7E8000A604B600749002200230A604B60044A24
:10D7F80090235B000021D150C04605B000BDC04653
:08D80800B00000202003002005
:10D8100030B585B0FA229200002302920393254A84
:10D8200086235B00D358002B06D1224A8A235B0053
:10D8300001214942D15239E01E4A86235B00D35868
:10D8400001931C4BDB6D019A9A4208D3029A039B09
:10D85000131C19B2174A8A235B00D15226E0154BDC
:10D86000DB6D002B06D1134A8A235B00012149425C
:10D87000D1521BE0019B180000231900029A039B60
:10D8800001F016F902000B0010001900094BDB6DC6
:10D890001C0000231D0022002B0001F06DF9020086
:10D8A0000B0011B2034A8A235B00D152C04605B077
:08D8B00030BDC046B0000020AD
:10D8B80080B50249096803F0B0F980BDA0000020D6
:10D8C800B0B5044608480568204602F017F9024634
:10D8D8002846214603F0F8FA401C03D00A20FFF737
:0CD8E800E7FFB0BDC043B0BDA0000020B1
:10D8F400C20F490089184000034A40428A4101D3BB
:0CD9040000207047012070470000E0FF89
:10D910000122D2079143034A4A4010434142484101
:08D920007047C0460000F07FD3
:10D92800074A0A40531E9A41C00F49000818054982
:10D93800884201D3002000E0012010407047C04613
:08D948000000F07F0000E0FF89
:10D9500030B50E4B5D1C0C0D2C4010D0AC420ED0DF
:10D96000A2189A4205DD0120C007014009480918A4
:10D9700009E0002A04DD064B19401205114330BDB1
:10D980000120C0070140002030BDC046FE07000056
:08D99000FFFF0F800000F07F93
:10D9980010B54B005B0D084CA34201D0002B02D1FF
:10D9A8000023136010BD054C1B191360044A114075
:10D9B800044A891810BDC046FF07000002FCFFFF9B
:08D9C800FFFF0F800000E03FAB
:10D9D000F0B589B01E460025EF436A4C7B1C0794C6
:10D9E00023466B4103937B1C0493674B1C460895AD
:10D9F0006C41069474000294640D644D00D1A8E05B
:10DA0000C40F4D0001952D19440005973C1B079C40
:10DA1000AC4100D2ACE0D40F029D2D195700049CFC
:10DA2000E71B039CAC41089C584D00D28DE0069C3E
:10DA30000C4006940C461C4033400746059D2F4081
:10DA4000154005950297ED1B1D46A54100D382E0C8
:10DA500001252F050797019F7F0D039508D000240E
:10DA600008946D42079DA5412940079C214311E080
:10DA7000079884420CD2E80408900298C10F650010
:10DA8000691840007F1E089DAC420C46F6D301E0A9
:10DA900002982146340D3E4D2C4009D000230893B6
:10DAA000039D6D42079D9D412E40079B1E4312E042
:10DAB000079A93420DD2039AD2040892059AD60F80
:10DAC0005D00AE195200641E089DAB423346F6D38A
:10DAD00001E0059A1E46A74212DD831A0D46B541A4
:10DAE00004D450407140014302D112E003460D4678
:10DAF000D80F6900091858007F1EA742EDDC2746A1
:10DB0000841A0B46B341039D06D450407140014333
:10DB100004D1049C069D18E004460B460798034276
:10DB200009D1E804E10F5A00511864007F1E034236
:10DB30000B46F7D000E01946002F1CDD781E049A32
:10DB4000A418069A514100050D182046294609B02F
:10DB5000F0BD089CF9E7059A3D4655405C402C43D2
:10DB6000069D00D00D46002C00D00490049CECE7EC
:10DB7000089C064DE9E7EA1B204600F079FF0446C1
:10DB80000020DCE7FFFFDFFFFFFFFF7F0000F87FE3
:04DB9000FF0700008B
:10DB9400F0B583B00E46044627494A1C300D1040A8
:10DBA400421E8A423DD22649884205D20024002ED4
:10DBB400254632DA254D30E03331884201D93546E5
:10DBC4002BE01E494518204631462A4600F03EFF08
:10DBD4001C4A114001434F424F4100201A49019011
:10DBE40002952A4600F052FF0D463540019A01D5B0
:10DBF400114600E001210F4320400446D043401C5D
:10DC040010495141029A00F031FF20186941002F58
:10DC140000D10D46002F00D104462046294603B00A
:10DC2400F0BD002802D10121C9070E403546002865
:10DC3400F3D10024F1E7C046FE07000001FCFFFF1A
:10DC4400FF030000FFFF0F000000F0FF0000F0BF23
:10DC5400F0B587B00A0D521E494B9A4215D206AA56
:10DC6400FFF798FE06460F46069C49484949711A33
:10DC7400394681413046394618DA0022474B00F0D4
:10DC840007FB06460F46641E14E0C30F4A00D31870
:10DC9400440064423B4C9C416AD3520D6CD0002931
:10DCA4000A4600DA394A002963DA66E000223A4B70
:10DCB40000F0EEFA019404900D460024E24305942A
:10DCC40030463946FFF742FE354B002200F0E0FAB9
:10DCD40002460B460498294600F06CFC04900F465B
:10DCE40002460B4602F0DFFF04460D462D4E02218C
:10DCF400304622462B4603F006FD2B4A2B4B00F000
:10DD0400C7FA0390029110360321304622462B466F
:10DD140003F021FD02460B460398029900F04AFCE9
:10DD240022462B4602F0BFFF049C22463B4602F0EB
:10DD3400BAFF22463B4600F0ABFA06460F4601986E
:10DD440000F0CAFD04460D46194A1A4B02F0ABFF17
:10DD540032463B4600F09CFA06460F46164B2046D8
:10DD64002946059A02F09FFF32463B4600F090FA9E
:10DD74000A46114607B0F0BD034A0020F9E7C04641
:10DD8400FE0700000000E0FF0000F0FF0000F87F45
:10DD94009EA0E63FCE3B7F660000F0BF0000E0BFE0
:10DDA4000000E03FC03000089AB5B312FF0750C02E
:0CDDB400A80C615C10D02BBF0030E63FD3
:10DDC000F0B585B00D4607465A48411C2A0D0A4059
:10DDD000511E814200D390E059485A49C91BA841BD
:10DDE00000DAA4E000205849584AD21BA941014654
:10DDF00000D280E00120C007294681435548564A99
:10DE0000BA1A814175D3554A554B3846294602F016
:10DE10004CFF00240494E243524B521C63412B40BC
:10DE2000514C234300F036FA00F0A2FC039000F0BE
:10DE300055FD04460E464D4B049A02F036FF3A4615
:10DE40002B4600F027FA05460F46494A494B204623
:10DE5000314602F02AFF2A463B4600F01BFA0646EE
:10DE60000D4602460B4602F020FF0F46424A434B46
:10DE70000446029002F019FF414A424B00F00AFAB0
:10DE800022463B4602F011FF3F4B049C224600F025
:10DE900001FA32462B4602F008FF05460E462046A0
:10DEA00031492A46334600F0D9FA01900091374AA9
:10DEB000374B029C2046394602F0F7FE354A364B76
:10DEC00000F0E8F922463B4602F0EFFE019A009B83
:10DED00000F0E0F902460B462846314600F06CFBA4
:10DEE000049A214B00F0D6F9039A521CFFF730FD3B
:10DEF00001E01749002005B0F0BDF80F69000818CF
:10DF0000790049420C49814129460ED30120C007BE
:10DF100081430A484840384300D074E7002D294621
:10DF200000DA0021002D00DA00273846E3E7034934
:10DF3000E0E7C046FE0700000000E0FF0000F07FC1
:10DF4000422E8640EF39FAFE2B2386C0D2BC7ADD02
:10DF50000000F03FA19CC73B2342920C3CF92F9E4E
:10DF60002C15F73FFFFFFF7F0000E03F0030E6BFCA
:10DF7000A80C615C10D02B3F1CDC586FA452F13E02
:10DF8000E0F6B36FE4707C3F0000D03F0938DE6FED
:0CDF9000993F403FB35142718E71AC3F8D
:10DF9C00F0B587B01D460027FC43864B641C7B41C3
:10DFAC0006914B40029003436FD06E00700D824976
:10DFBC007DD00592824B5A1C06990C0D1440641EA0
:10DFCC009C4277D22B0D13407E4A9B18521C9342D5
:10DFDC0070D3059C2046294600F0C4FB074600F090
:10DFEC0077FC60406940014332D101200490C007A6
:10DFFC0087422DD0002F019749D0F81747403D1A82
:10E00C006D4F002403940298069E012D039A00D0B4
:10E01C0002460694012D684B00D033460446314627
:10E02C0002F03DFE3246064605912846049908400A
:10E03C00614B00D01346424222400698394602F00A
:10E04C002EFE04460F466D083046059EDDD120E0BD
:10E05C000027029C2046069E31463A463B4600F07D
:10E06C0061FB002801D05C4921E00120C10700229E
:10E07C00404291410E4020463146FFF7E5FD059A9E
:10E08C002B4602F00CFEFFF795FE07460FE04A4FB9
:10E09C0000240020484922463B4600F087FA019AAA
:10E0AC00002A00D43946002A074600D427463846B1
:10E0BC0007B0F0BD029CE20F4B009A1863005B1E88
:10E0CC00424B53410598F1D23F4A0124C30FF1183A
:10E0DC0043001B1B914114D204943849069A1346F1
:10E0EC000B4011D03A4914464C400298044326D0B8
:10E0FC001446324A544004433BD1002D56DA39467B
:10E10C00D5E707462946D2E7294600F02BFB074600
:10E11C0000F0DEFB2A46059C4A402346434013434D
:10E12C0000D05EE7069E0021002D00DA2349F80797
:10E13C0003D00498C007064071180027B7E70020E9
:10E14C000690002D00DB1D480390059F384629469C
:10E15C0000F008FB044600F0BBFB69407840084324
:10E16C0017D10498044014D0C00703990918069FCE
:10E17C009DE74D40059828430ED11649069D4D400C
:10E18C00029828430C4992D000210A4898428ED319
:10E19C000CE0069F03998AE706489842394686D2D6
:10E1AC000C48069D45400298284301D011467EE755
:10E1BC0001497CE7FFFFEF3F0000F03F0000F07FDC
:10E1CC00FE07000001F8FFFF0000E0FFFFFF1F004B
:0CE1DC000000F0FF0000F0BF0000F87F22
:10E1E80003490868002800D0704702480860704753
:08E1F800D80B00208400002078
:10E200007F2805D8034A125C0348405C10407047E1
:0CE21000002070472B190108F0180108CD
:10E21C007F2805D8034A125C0348405C10407047C5
:0CE22C00002070472B190108F0180108B1
:10E23800F0B581B000280090124D13D00146C017E8
:10E2480041400F1A0026104CF80707D00CCC304676
:10E258002946083C02F025FD06460D4608347F088D
:10E26800F2D100E000260020064932462B4600F095
:10E278009FF9009A002A00D43046002A00D4294683
:0CE2880001B0F0BD0000F03FE8300008DD
:10E29400F0B40125ED070F005F405AD48B4200D142
:10E2A400824205D950404240504059404B40594069
:10E2B4004E18760DDF187F0D3BD0741C640529D0F1
:10E2C400F41B352C26D80E0DDB022B43DB0AC902C6
:10E2D4002943C9121700202C1ED2E741E2405740BF
:10E2E400E3415A40A340E3405A4000248018594176
:10E2F4000AD3B21C520521D0C207012F6241170074
:10E304004008CB0718434908013636054208AF4197
:10E3140060417141F0BC7047203C06D01F00E741CA
:10E32400E3405F400024012A6741C0186141EBD3F8
:10E33400DFE7002EEED129400020EBE7013631055E
:10E344000020E7E7E742E5D10020C143090DC904F5
:10E35400E0E76B400E00871A9E4104D26E40C01B5A
:10E36400B141D21973414E18DF18AC0AE642E9D222
:10E37400760D7F0D31D0F41B362CCBD8B4460E0D60
:10E38400DB022B43DB0AC9022943C90A012C32D818
:10E3940004D1D4075208DF073A435B08EF0A64420A
:10E3A400904199411ED0002239424DD12419404157
:10E3B40049410124394204D1013400184941394208
:10E3C400FAD06246A24204D9361B013E36058919A9
:10E3D400A0E7F10AC90700209CE736429AD1002041
:10E3E400002197E70200224394D0B842DED2010014
:10E3F40020002024E3D1202C13DD203CE24117002F
:10E40400A240E2405740E3415A40A340E3405A400F
:10E41400012FBF410137174300227C4298419141AB
:10E424000CE01700E741E2405740E3415A40A34063
:10E43400E3405A407C429041994100220F0303D2A9
:10E44400013E241940414941013E36054708AC418B
:08E4540050417141F0BC70471A
:10E45C00F0B40125ED076B40004C20479BE200080F
:10E46C0030B405004D400124E407254042004B0028
:10E47C00120E32D01B0E3CD0FF2A33D0FF2B3FD0D4
:10E48C00D21800022043000A09022143090AC4B22F
:10E49C004C43000AC3B24B43000A4843210A5B18A1
:10E4AC00190A091801D44900013A080A7F3A2ADBF3
:10E4BC00FE2A0FD2D2051C43240601D0012421438D
:10E4CC00C9B280295041802901D14008400028431D
:10E4DC0030BC7047FF20C005F9E71B0EFF2B0AD09C
:10E4EC002800F5E7400206D1FF2BF3D1490202D1F7
:10E4FC00F0E7FF2AF4D17F2000010C300005E7E79C
:10E50C004902F8D1E6E743020132E9D15B1202334A
:08E51C00E6D9D805E4E7C0468A
:10E5240030B405004D400124E407254042004B006F
:10E53400120E26D01B0E34D0FF2A2DD0FF2B35D03F
:10E54400D21A000220430902214343084908A00DBE
:10E554005B1A02D2013A5B005B185B008B4200D36A
:10E564005B1A4041F9D37F3222DDFF2A06D2D2055D
:10E57400C91A8B425041284330BC7047FF20C00564
:10E58400F9E71B0E03D0FF2B12D1490210D07F20D4
:10E5940000010C300005EFE74002F8D1FF2BEDD16C
:10E5A400F5E7FF2AEAD14002F1D1E7E74902EED1CB
:04E5B4002800E1E773
:10E5B800F0B40125ED070C005C402C40A446AE0ADF
:10E5C8004C18DF18F4423DD2F74245D2640D4CD0C6
:10E5D8007F0D3CD0E41BC9022943CF0ADB022B4341
:10E5E800DB0A0600B61A9F4104D2013CB6197F41E6
:10E5F800B6185F416812800D241838DD001884426F
:10E6080025D8E80C0021B6197F41B61A9F4103D3DB
:10E6180040414941F7D304E0B6185F410018494129
:10E62800F1D32405B6197F41B61A9F4105D3374364
:10E63800C20717430022012F50416141624611432E
:10E64800F0BC70470CD100280AD1F74208D200204C
:10E65800C143490D0905F1E7002A01D1F74206D067
:10E668000020C143090DC904EAE77F0DF8D0002056
:04E678006146E5E72B
:10E67C0070B4012676054C005D00E6420CD8EE42E3
:10E68C000AD825430543154303D0994204D190423F
:10E69C0002D1012070BC7047002070BC7047C0468E
:10E6AC0030B401256D054C00E54215D85C00E542FF
:10E6BC0012D80C001C436400044314430FD005D241
:10E6CC00904299418041013030BC704782428B416D
:10E6DC008041013030BC7047002030BC70470120B5
:04E6EC0030BC704787
:10E6F00030B401256D054C00E54215D85C00E542BB
:10E7000012D80C001C436400044314430CD005D2FF
:10E7100082428B418041404230BC704790429941D7
:10E720008041404230BC7047002030BC7047C0463A
:10E7300030B401256D054C00E54215D85C00E5427A
:10E7400012D80C001C436400044314430CD005D2BF
:10E75000904299418041404230BC704782428B4197
:10E760008041404230BC7047002030BC7047C046FA
:10E77000F4464A1805D200F063F801D5C0174008E6
:10E78000604701235B05D34206D200F059F801D55A
:10E790000120C0074042604701D10042F5D0D017A8
:04E7A0004008704776
:10E7A4004A00520D01239B02D21A01321DD4524257
:10E7B4003F321DDD8C46C902430D1943C0020123BB
:10E7C400DB071943202A02D308000021203AD14153
:10E7D400D04048409140D140484063461B4203D555
:10E7E400002340428B4119007047002000217047EC
:10E7F400002801D0012211434B0001225205D342CB
:10E8040000D959080020C90FC90701D4C0434108E1
:04E814007047C04643
:10E8180041000DD2090E7F390AD449421F3105D46F
:10E8280000020122D2071043C8407047C81770473A
:04E838000020704705
:10E83C004A0010D2520D03231B02FF33D21A0AD402
:10E84C0052421F3209D4400DC90208430123DB0791
:10E85C001843D040704700207047D0177047C0460F
:10E86C004B001BD25A0D01239B02D21A013215D434
:10E87C0052423F3215DBC902430D1943C00201233A
:10E88C00DB071943202A02D308000021203AD1418A
:10E89C00D04048409140D140484070470020002172
:08E8AC007047D017010070470E
:10E8B400C20F12029D3201000CD001D5494202D48C
:10E8C400013A4900FCD5D205080A0906494100D39A
:08E8D400012950417047C046C4
:10E8DC00054B004206D5404200B5984708BC0122C2
:0CE8EC00D20711431847000075E900082E
:10E8F8000B00034329D0CA0FD200043212023D3262
:10E90800094203D5002349424042994102D10100FE
:10E918000020203A0B0C04D1103A0904030C1943C7
:10E928000004094203D4013A00184941FBD5844642
:10E93800C00A4B051843C90A120563465B055B41CB
:0CE9480002D3012B0023584151417047BD
:10E954009D2201000AD002D4013A4900FCD5D20517
:10E96400080A0906494100D3012950417047C046AD
:10E9740042221201033A010007D002D4013A0018DE
:0CE98400FCD51205C30A40059918704725
:10E990000B00034305D0042212023D320942014B11
:08E9A0001847704715E9000853
:10E9A80041008C46012212068A420BD809093823F5
:10E9B8001B06C918C30FDB07194340076346DA4231
:10E9C80004D27047C10FC9070020704703D138230C
:10E9D8001B06C918704738231B06C9180122D20420
:04E9E8001143704720
:10E9EC004B1801225205DA4217D25B0D0722D201D5
:10E9FC009B1A0FD9FF2B13D2DB05CA0FD207134377
:10EA0C000903020D1143490AC200524100D90131D8
:10EA1C00C8187047C80FC007704706D1002804D12A
:10EA2C00C80F0002FF30C00570470123DB070A0046
:10EA3C00C900400F084398431A4010435B0A18431F
:04EA4C007047C04609
:10EA5000202A07D203009040914052422032D340F6
:10EA600019437047203A0100914000207047C0468A
:10EA7000202A07D2D0400B00D1405242203293408E
:10EA800018437047203A0800D04000217047C04624
:10EA9000202A07D2D0400B0011415242203293402D
:10EAA00018437047203A08001041C9177047C04604
:10EAB00030B5514343435C18010C130C0D005D430A
:10EAC000641992B2514380B242430D0C09045218AA
:10EAD00065415843010C00048018694130BDC046AF
:10EAE000CA1751408B1A17D0C1174A409446484064
:10EAF000411A48081A0000E052008242FCD9002066
:10EB000000E05208914200D3891A40419A42F8D15C
:10EB100062465040801A704710B500F095F810BD5D
:10EB200007B5FFF7DDFF0EBC4243891A00BDC046A2
:10EB30000A0015D00300400800E052008242FCD9D0
:10EB4000002000E052089B1A06D340418A42F9D1C6
:10EB5000704752089B18F8D200188A42F9D17047C2
:08EB600010B500F071F810BDC2
:10EB680038B504004D42FFF7DFFF4543611938BD52
:10EB780070B5CC1760406140001BA141DD176A40A9
:10EB88006B40521BAB4100F00BF862406340121B14
:10EB9800A3416C4060406140001BA14170BDC0466C
:10EBA800002B09D1002907D110B51100FFF7D8FFB4
:10EBB8000A000021002310BD70B400240125ED07D0
:10EBC800002B07D1002905D0834203D2130000226D
:10EBD8002C0000250026A419994200D1904212D990
:10EBE80092185B4103D2EE076D086408F3E7DE076D
:10EBF8005B08520892190126F6079B1903E0DE0705
:10EC08005B0852089219801A994103D364416D41F7
:10EC1800F5D30FE024196D410AD2DE075B085208CC
:10EC2800921980185941F5D364416D41E7D301E049
:10EC38008018594102000B002000290070BC704761
:08EC4800002000217047C046C6
:10EC5000F0B503AF93B06E46F51D2135F41D393480
:10EC600074613362F261F160306102F0D8FDB0602E
:10EC7000C21D07218A436946B1616946881A7060DE
:10EC80008546F41D1D3400212422204600F0BEFFDD
:10EC90000B487169F2680A6048600A482860306968
:10ECA0002862B06868617068E8602046F169326A7D
:10ECB00000F01EF8B1698D46FC1F053CA546F0BD6D
:08ECC0000F180108FFFFFF7FA0
:10ECC80083B010B581B0044603A80EC0054800689B
:10ECD80003AA0092214602F0EAF801B010BC02BC77
:08ECE80003B00847A000002062
:10ECF000F0B59FB013920B4604460020206001211E
:10ED00000A020F924A020B928A020492CA020392EA
:10ED100003220C92920206920A0309924A03079276
:10ED20008A0305920191C90317910890C04302908C
:10ED300016941978252909D0002901D100F032FE56
:10ED40005C1C169802F05AF82346F2E7DB1C089F79
:10ED50000B9C099D981E00780246203A102A2DD857
:10ED6000802192003E461F4602A39A583B463746F2
:10ED70009746C046B9ED0008D9ED0008D9ED000866
:10ED8000D3ED0008D9ED0008D9ED0008D9ED000851
:10ED9000C5ED0008D9ED0008D9ED0008FDED00082B
:10EDA000C9ED0008D9ED0008CDED0008D9ED000847
:10EDB000D9ED0008D1ED000840210AE05E2829467F
:10EDC00007D009E0179904E0202102E0102100E0BB
:10EDD00021460F435B1CBDE75B1E01463039002412
:10EDE000092917D80A2161434418303C591C187866
:10EDF0000246303A0A2A0B46F4D30BE0139901C9B4
:10EE00001391002801D510210F43C1174840441A1F
:10EE1000581E007800252E281CD118782A2805D1E4
:10EE200058789B1C139920C913910FE05B1C014675
:10EE3000303909290CD80A2169434518303D591C3D
:10EE400018780246303A0A2A0B46F4D3002D01D432
:10EE50000F990F43E1176B2808DC4C2803D0682872
:10EE600036D06A280AD10220074305E06C2834D046
:10EE70007A2801D0742801D118785B1C8C4346286D
:10EE800011930D9419DD01466339152935D8C04613
:10EE90007944097949008F44540B4919D10A0B0A66
:10EEA0000A0A0A65737F0A0A8D0A920A0A3840E73D
:10EEB000059B1F430024394689E0442815DD452879
:10EEC00032D0462800D034E70798074303982EE055
:10EED000187868282ED1082003E018786C282CD1E7
:10EEE0000220074358789B1CC8E7252800D07BE206
:10EEF0002521169801F082FF74E2472800D19BE09B
:10EF0000582800D015E707990F43D14A782800D137
:10EF100020323906CC170F990F4201D0CD490F404E
:10EF20003946059B144052E007980743049807436D
:10EF3000069A85E05B1C042201E05B1C012217435A
:10EF40009CE7139D20462C78421E169E304639467B
:10EF5000159201F0A5FF3046214601F04FFF2D1D0F
:10EF60001395D7E013980068390700D540E2B90738
:10EF700016990968016000D43DE2002141603AE23F
:10EF80000F990F42394601D0B24A11403A06D217C2
:10EF900030241440059B1AE038060F990F430E9752
:10EFA000C017232101400A91139840C813900024F0
:10EFB0000825B0E11295139901C9139186E00F99C4
:10EFC0000F4201D0A3490F403946059B002402227D
:10EFD0000A4019420A9405D1002A139A08D1131D38
:10EFE00000240BE0002A139B13D104CBD41715E0A7
:10EFF000D21D07239A4354681346083313931668A7
:10F000004A0713D408220A4000D0F6B2002A0ED1D3
:10F0100002E1DB1D0722934314CB003313934B070C
:10F0200007D40B0700D5E3E01646E4E0B6B20024AF
:10F03000F2E016B21204DDE007980743069A174380
:10F040000F98074201D0284600E0062039461140BB
:10F05000891A4A424A41002800D002461292139C63
:10F06000E41D072084432668656830462946FEF77C
:10F070004FFC083413940028304629460DD0002256
:10F080001346FFF755FB3A4607990A4000280ED071
:10F09000002A714818D0714816E0FEF72BFC0028B2
:10F0A0003ED0079807426E480ED06E480CE0002A0A
:10F0B0006D4900D06D49002A01D06C4800E06A48D3
:10F0C000401CBA0600D5084669490F400028694E21
:10F0D00000D006463D465F4805400F98074230463F
:10F0E00002D100F00FFD02E0129900F043FD04464A
:10F0F000169F0D98021B38462946159201F0D0FE46
:10F10000002C06D03178384601F078FE761C641E5B
:10F11000F8D12F46119BF80600D40AE6159A5DE156
:10F1200030462946FEF700FC002800D1064600289C
:10F1300000D1002514963046294602F0E4FA044630
:10F140000120002C0A9001D0C00745401EAA30467D
:10F1500010952946FEF720FC1E980C9948430A2179
:10F16000FFF7BEFC1E900646002C01D0602007432E
:10F170000022149C2046294615921346FFF77EFA7A
:10F18000002818D1701CFFF757F822462B46FFF7CE
:10F19000CFFA00281E9806D0411C1E91801CF2E771
:10F1A0001E98401E1E90FFF747F822462B46FFF799
:10F1B0009FFA0028F4D13B4606990B400A9880023A
:10F1C0008342109D149C00D119E10E908B42129A3B
:10F1D00008D11E98824200DC12E10421C943884212
:10F1E00000DC0DE10498074200D015E11592FAE128
:10F1F00056B21206D417002C05D48A060AD44A0641
:10F200000AD5202207E000227642A2412D230A934C
:10F21000144601E02B220A920F9A114201D00D4AA6
:10F2200011400A460F990A420E9200D1012500278B
:10F230006E2838DD6F38092800D98BE078440079D2
:10F240004000874419688787878736878768C04664
:10F2500058300000FFFDFFFF02190108FD180108EA
:10F26000CF190108CB1901080C1901080719010869
:10F27000FFFEFFFF98180108304620436AD0F008CF
:10F2800061074018014607203040303018AAD05599
:10F29000C808E408620780180A4622437F1C002A37
:10F2A0000E46EFD156E0582835D0642801D06928A1
:10F2B00050D1304620434DD011461798014010914F
:10F2C000129532461098002808D038460C9908400C
:10F2D000032803D118A82C21C1557F1C00251046F6
:10F2E0001594214614920A222B46FFF75DFC0C462A
:10F2F0000A2206462B46FFF7DBFB149A101A302130
:10F30000014318A8C1557F1C0920801A1598854112
:10F31000129DD6D31EE0304620431AD007980E998E
:10F320000142FB4800D0FB48310922078918002719
:10F330000A460F213140415C18ABD9551109240907
:10F340002307C918134623437F1C002B1646EFD111
:10F3500000E000270D98C01B0A99FF2900D9401E24
:10F36000002900D0401EED1BE9178D43421B0B986E
:10F370000E99014205D1169801F092FD00201590DA
:10F3800000E015920A9C210A169E03D0304601F037
:10F3900035FD01E0002C03D03046214601F02EFD62
:10F3A00030460E99159C224601F07AFD30213046F8
:10F3B0002A4602F01EFA012F0ADB7D1C18A840190C
:10F3C000801E0178304601F019FD6D1E012DF5D823
:10F3D0000E98C006119B00D4ABE42246202116985B
:10F3E00002F007FA119BA4E4002800D0A1E4E9E2AE
:10F3F0001699096801701398001D139099E41E98DE
:10F4000015930F993431884233D120462946CA4A90
:10F41000CA4BFFF7D1F833E01E980E2800DDE2E07A
:10F42000C0431418102C00DB1024380600D5D9E096
:10F43000002C159400D1D6E02046FEF7FDFE149A6C
:10F440002B4601F032FC00263246BD4BFEF722FF70
:10F45000FEF7A0FB3246BB4BFEF7BAFA32461596D2
:10F460000023FFF70BF9002800D1BBE0641EE3D1B5
:10F47000B9E04042FEF7E0FE22462B4601F015FCC3
:10F4800004460E4600221346FFF7F8F8002839D14B
:10F4900020463146FEF73CFA00282046314600D08F
:10F4A000EDE50E970022A74BFFF700F91E9F0028FD
:10F4B0000FD0002220463146A24BFFF77DF80446CC
:10F4C0000E4600229F4BFFF7F1F87F1C0028F0D179
:10F4D0001E970022204631469B4BFFF729F9002852
:10F4E00011D0002220463146964B01F0DEFB044647
:10F4F0000E460022944BFFF71BF97F1E0028F0D127
:10F500001E9700E00E97069815998142129801D037
:10F51000014600E0411E029D0028159100D1002106
:10F5200014914842FEF788FE2A46FEF711FA224659
:10F530003346FEF7AFFE06460D4600221092814C80
:10F540002346FFF7B3F800280AD01E98401C1E90EF
:10F550000022304629462346FFF72EF806460D4680
:10F56000149812960095002839D003990B468033E1
:10F570000E9A13408B4200D0A9E0102800DB102027
:10F580000546FEF759FE3246009B01F08EFBFFF761
:10F590006DF9074608431098159000D197E00C4686
:10F5A0000A2200233846FFF7FFFA002D00D18DE034
:10F5B0001A4300D08AE015950A22002338462146D6
:10F5C000FFF7F2FA0C4607460A220023FFF7ECFA8F
:10F5D0001598401E15907AD01A43EDD077E0109818
:10F5E000159074E015941E98103815994942884278
:10F5F00000DC0846FEF720FE029AFEF7A9F9149AED
:10F600002B46FEF747FE05460C461E98401CFEF7AB
:10F6100013FE2A462346FFF78BF81E99002800D0D8
:10F62000491C002914D4112918D3084610381E90FB
:10F630001020401AFEF700FE2A46234601F035FB53
:10F64000FFF714F906460C46002012900A9018E0C5
:10F650000A95129400261E96344612E000201E9051
:10F6600028462146FFF702F9129406460C46FFF79A
:10F670008FF902460B4628461299FEF7EFFE0A90D4
:10F68000129138460E998843D349083100250A461D
:10F6900008326D1C0B684968F31A23468B411146EA
:10F6A000F6D21495159B002B019901D1F9B2C90925
:10F6B0007A06920F01D1494200E0C9431E9A891A85
:10F6C0000D9AD21A5118491B074677E01595159DDA
:10F6D000002D019802D10E98C0B2C0090D99491BA6
:10F6E000081A0E9F421F1E9C09983E46074202D1EF
:10F6F0000A990F463EE01092032720463946FFF74D
:10F700000FFA881C04282ED803A1085C4000874407
:10F71000BB190108AB190108061D2C061D00641E4B
:10F720001E94002212980099A94B01F0BEFA109A7B
:10F73000521E022714E0C046A0C8EB85F3CCE17F3F
:10F740000000E03F000024400000F03FA41E1E9493
:10F750000022129800999F4B01F0A7FA109A921E6E
:10F760001290009103E0002700E00127109A0A9907
:10F77000E81785437006800F159500D0521E109231
:10F78000CD02204602F011F86328149702DD10988C
:10F79000401E10903746AF431298009D2946FFF750
:10F7A00065F806460C46FFF7F3F802460B4612983A
:10F7B0002946FEF753FE0A9012911099C8170D467C
:10F7C00085430B9810300E9707420AD1012908DBB8
:10F7D000169F2021384601F011FB6D1EF9D10E99BC
:10F7E00000E03946402008408906149F03D40028D1
:10F7F00009D0202104E0002801D02D2100E02B2198
:10F80000169801F0FBFA0E98C00609D4002D07D017
:10F81000169F3021384601F0F1FA6D1EF9D1149F80
:10F820007F1EF8006C4A111849681258B01A204619
:10F83000884101D2302007E03020B61A8C41401CAC
:10F84000B31A23468B41F8D2C1B2169801F0D6FA0A
:10F85000002FE5D10E9E344603980440169F0BD02E
:10F860001E98012808DB401E1E903021384601F00A
:10F87000C5FA1E980028F6DC80203040159E3043E3
:10F8800046D02E21384601F0B9FA102E00DB1026A2
:10F89000F01737468743002C01D1384601E01E9807
:10F8A000381AFEF7C9FC159A1497D21B1092012E34
:10F8B00021DB0A9A129B01F0F8F9FEF7D7FF044604
:10F8C0000E467F1EF800444A111849681258A01AC3
:10F8D0003046884101D2302007E03020A41A8E4102
:10F8E000401CA31A33468B41F8D2C1B2169801F0DE
:10F8F00085FA002FE5D110980028169F159807D09B
:10F9000014990C1A3021384601F078FA641CF9D3A6
:10F9100004980E99014238D00798014201D0452140
:10F9200000E06521169E304601F068FA1E98002816
:10F93000304604D42B2101F061FA1E9805E02D21F8
:10F9400001F05CFA1E9840421E9064280DDB642191
:10F95000FFF7EEF801463031304601F04FFA1E98BD
:10F960006421FFF7DDF808461E910A21FFF7B8F879
:10F9700001463031304601F041FA1E980A21FFF766
:10F98000CFF83031304601F039FA002D119B01D10A
:10F99000FFF7CFF9169C2021204601F02FFA6D1EAB
:10F9A000F9D11FE5169CE068002805D006CC083C7C
:10F9B000914201D2089A4254204601F064FA20682C
:10F9C0001FB0F0BD169801F05EFA0298F8E7C04645
:0CF9D000000024400000594030310008C5
:10F9DC0009490968091A4A1E9141084A1268121A03
:10F9EC00531E9A410A4006490968081A411E88416B
:10F9FC00104040427047C046A0000020A4000020E8
:04FA0C00A80000202E
:10FA10000F480321016141610E4A82610E49C161B3
:10FA2000012189020162002181624162C162026694
:10FA30000A4A4266102282660167C1664167084A27
:10FA400013784354521E491C1029F9D17047C046FF
:10FA50007C07002022190108340C002034100020FB
:04FA60002019010860
:10FA6400F0B581B00D461821414316484618F06A96
:10FA74001836022811D01446012814D00027002873
:10FA84001DD1304601F027FAA04218D3304629464A
:10FA9400224601F02BFA274611E03046294601F0B0
:10FAA400BEFE07460BE0304601F015FA0746A042B9
:10FAB40000D32746304629463A4601F017FA38461D
:08FAC40001B0F0BD7C07002039
:10FACC00F0B581B014460D4606460A480078002869
:10FADC0001D1FFF797FFEFF31087012181F3108815
:10FAEC00304629462246FFF7B7FF87F3108801B04E
:08FAFC00F0BDC0467C070020AC
:10FB0400F0B581B00178002925D003220146009286
:10FB140091430D680023DC438607F60EB440E443AA
:10FB24002C43114D6719A743104A174206D14C685C
:10FB340067191646A643091D3E42F8D022060FD087
:10FB44002204120E09D02202120E08D0220E009BAB
:10FB540006D0042304E0002004E0012300E0022393
:10FB6400C918081A01B0F0BDFFFEFEFE8080808037
:10FB7400F0B581B00022002933D00378002B30D0B7
:10FB8400032302469A4316680024E5438707FF0EC1
:10FB9400BD40ED43354306461E40711804290093C9
:10FBA4000AD3124EAF19104BAB433B4204D1091F89
:10FBB4005568121D0329F5D82B060DD02B041B0EF6
:10FBC40007D02B021B0E06D02B0E009C04D004245D
:10FBD40002E0012400E002248C4200D30C46101AF7
:10FBE4000219104601B0F0BD80808080FFFEFEFE49
:10FBF400002A03D0013A8B5C8354FBD17047C04682
:10FC040000220B0011001A00002A02D0013A81548C
:04FC1400FCD1704768
:10FC180046A5000856A5000866A5000876A50008B0
:04FC280086A50008A5
:10FC2C00C2BF000800BF00080CBF000816BF0008C8
:10FC3C0020BF0008C2BF00087CBF000882BF0008BC
:10FC4C008CBF000896BF00089CBF0008A6BF000828
:10FC5C000000000000000000000000000000000098
:10FC6C000000000000000000000000000000000088
:10FC7C00010000000200000003000000040000006E
:10FC8C00060000000700000008000000090000004A
:10FC9C000000000000000000000000000000000058
:10FCAC00010000000200000003000000040000003E
:0CFCBC009F180108E8FC0008C8FC0008C4
:10FCC80001E20008C3170108CF1701081DE2000868
:10FCD800DB170108E7170108B3170108450C0108ED
:10FCE800A1180108DD180108DD180108DD18010850
:10FCF800DD180108DD180108DD180108DD18010804
:10FD0800DD180108DD180108FFFFFFFFFFFFFFFFF7
:10FD1800FFFFFFFFFFFF0000A3180108FF00010815
:10FD2800250201089304010882180108DE18010859
:08FD3800E71801088918010811
:10FD4000034C206804348047FBE7FBF717FFFEE70E
:04FD5000D4190108B9
:10FD540004480549884385460448804704480549C2
:10FD64000160EBE7008000200700000055D0000888
:08FD740008ED00E0003000087A
:10FD7C00FEE7FEE7FEE7FEE7FEE7FEE7FEE7FEE74F
:10FD8C00FEE7FEE7FEE7FEE7FEE7FEE7FEE7FEE73F
:10FD9C00FEE7FEE7FEE7FEE7FEE7FEE7FEE7FEE72F
:10FDAC00FEE7FEE7FEE7FEE7FEE7FEE7FEE7FEE71F
:0CFDBC00FEE7FEE7FEE7FEE7FEE7FEE7DD
:10FDC8004552524F52204144535F313236305F53CF
:10FDD8006574436F6E76657273696F6E4D6F646597
:10FDE800000000004552524F52204144535F3132C7
:10FDF80036305F53657443686F704D6F64650000FB
:10FE08004552524F52204144535F313236305F538E
:10FE18006574446174615261746500004552524FC3
:10FE280052204144535F313236305F536574446920
:10FE3800676974616C46696C746572004552524F0B
:10FE480052204144535F313236305F496E707574C9
:10FE58004D757853656C6563740000004552524FC8
:10FE680052204144535F313236305F536574496ED6
:10FE78007465726E616C5265666572656E63650065
:10FE880046100000460A00002D2D2D204761696E9E
:10FE9800202043414C202D2D2D0000004144535F6C
:10FEA800313236305F4261747465727943757272AB
:10FEB800656E744761696E43616C696272617469E9
:10FEC8006F6E53746172743A204552524F522049F2
:10FED8004E2043414C4942524154494F4E2C204EEA
:10FEE8004F205245464552454E43452043555252B0
:10FEF800454E542100000000492028776974686F36
:10FF0800757420636F6D70656E736174696F6E29A7
:10FF18003D25660A00000000492052656665726545
:10FF28006E7A3D25660A0000547368756E743D2527
:10FF3800660A000054736869703D25660A0000006F
:10FF48004B6F7272656B74757266616B746F723D1C
:10FF580025660A002D2D2D204761696E202043411A
:10FF68004C20454E44452D2D2D0000002D2D2D20D3
:10FF78004761696E2044726966742043414C202DA4
:10FF88002D2D000041637475616C20543D25662059
:10FF9800430A000064656C746120543D2566204363
:10FFA8000A00000041637574616C20493D25662094
:10FFB8004128776974686F7574206761696E207469
:10FFC800656D7020647269667420636F7272656310
:10FFD80074696F6E290A000052656620493D2566DE
:10FFE8000A0000004B6F7272656B74757266616B04
:08FFF800746F723D2566205B69
:020000040801F1
:100000002031202F2043656C736975735D0A0000F1
:100010002D2D2D204761696E20447269667420433E
:0C002000414C20454E4445202D2D2D0064
:10002C0046697273742073746172742064657465AC
:10003C006374656421000000436F6D7061727469B4
:10004C00626C65207374617274206F7220757064B9
:10005C0061746520646574656374656400000000F8
:10006C00496E636F6D7061727469626C6520737434
:10007C006172742F75706461746520646574656356
:10008C0074656400454550524F4D2046554C4C20EC
:10009C00524553544F5245210000000045455052E3
:1000AC004F4D20464143544F525920524553544FC3
:1000BC0052452100454550524F4D2053544F524507
:1000CC0020434F4E46494721000000005772697487
:0800DC00696E6720534E2100FC
:0400E40069D00008D7
:1000E8004552524F52205452494D4D494E47205681
:0700F800414C5545530A007D
:1000FF0053756E004D6F6E00547565005765640043
:0D010F005468750046726900536174000069
:10011C0063616C696C62726174696F6E2076616C7C
:10012C007565203A202564003A202020667265719E
:10013C0075656E6379203A2025640A0056616C75EA
:10014C0065206E6F742076616C696400467265710F
:10015C0075656E6379204D65617375726564203DBC
:10016C002025640A000000006869676865737420C4
:10017C006672657175656E63792025640A000000EE
:10018C006C6F7765737420206672657175656E632C
:06019C00792025640A0031
:1001A20084B0039002910192039B9B6A029A1F21E1
:1001B2000A400F2191400A00D2431A40019B9B0E34
:1001C2000F211940029B1F20034099400B001A4344
:0A01D200039B9A62C04604B0704718
:0E01DC0075617274206572726F72200A0D00D8
:1001EA0082B001900091019B9B6A009A5203520BC4
:0E01FA00D2431A40019B9A62C04602B0704781
:100208002D2D2D2064693D25642C2064753D2564C1
:0D0218002C20723D2564202D2D2D0D0A0097
:100225004A616E75617279004665627275617279AF
:10023500004D6172636800417072696C004D6179AF
:10024500004A756E65004A756C790041756775736E
:10025500740053657074656D626572004F63746FE9
:10026500626572004E6F76656D6265720044656306
:07027500656D626572000077
:10027C004953454E534F525F3530303A20496E69E1
:10028C00740000007265616420636F6E6669672E8E
:10029C002E2E0000666163746F7279207265737420
:1002AC006F72652E2E2E00004144533132363020B1
:1002BC00496E697400000000554E4B4E4F574E204E
:1002CC00434F4D4D414E4400537461727420656E22
:1002DC0061626C6520726561646F75742070726FF9
:1002EC0074656374696F6E00466C61736820756E1B
:1002FC006C6F636B206572726F720000466C617379
:10030C0068206F6220756E6C6F636B206572726F04
:10031C00720000002E2E2E466C61736820756E6C78
:10032C006F636B002E2E2E456E61626C65206C6FB8
:10033C00636B206572726F7200000000466C617313
:10034C0068204F7074696F6E62797465206C6F638E
:10035C006B656400466C61736820206C6F636B6521
:10036C00640000002E2E2E456E61626C65206C6F51
:10037C00636B2070726F636573732066696E69734B
:10038C00686564002E2E2E466C617368206C6F635A
:10039C006B20616C72656164792061637469766548
:1003AC00000000002E2E2E466C61736820756E6C5A
:1003BC006F636B65640000002E2E2E466C617368B3
:1003CC00206F6220756E6C6F636B656400000000BB
:1003DC00466C617368204F7074696F6E62797465D6
:1003EC002070726F6772616D6D206661696C6564F7
:1003FC0000000000466C617368204F7074696F6E6A
:10040C00627974652070726F6772616D6D656400DE
:10041C002E2E2E44697361626C65206C6F636B20A9
:10042C0070726F636573732066696E697368656457
:10043C000000000050524F54454354494F4E3A204F
:10044C004F425F5244505F4C4556454C5F30000064
:10045C0050524F54454354494F4E3A204F425F52ED
:10046C0044505F4C4556454C5F31000050524F5440
:10047C00454354494F4E3A204F425F5244505F4CD3
:07048C004556454C5F3200AC
:100493004A616E00466562004D61720041707200F0
:1004A3004D6179004A756E004A756C0041756700AD
:1004B300536570004F6374004E6F760044656300AC
:0104C3000038
:1004C4004F5554505554535F4C56505F4241545409
:1004D4004552595F554E444552564F4C5441474539
:1004E400000000004F5554505554535F4C56505F14
:1004F4004F56455243555252454E54004F55545051
:100504005554535F4C56505F5348554E545F4F56A5
:10051400455254454D5045524154555245000000F2
:100524004F5554505554535F4C56505F43484950AF
:100534005F4F56455254454D5045524154555245CE
:10054400000000004F5554505554535F4C56505FB3
:100554005348554E545F554E44455254454D5045AD
:1005640052415455524500004F5554505554204C57
:100574005650204F4B0000004F5554505554535F74
:100584004F56505F424154544552595F4F5645525D
:10059400564F4C54414745004F5554505554535FA2
:1005A4004F56505F4F56455243555252454E540094
:1005B4004F5554505554535F4F56505F5348554E02
:1005C400545F4F56455254454D504552415455522F
:1005D400450000004F5554505554535F4F56505FDB
:1005E400434849505F4F56455254454D504552413A
:1005F40054555245000000004F5554505554535F14
:100604004F56505F5348554E545F554E44455254CF
:10061400454D504552415455524500004F55545094
:100624005554535F4F56505F434849505F554E44AD
:100634004554454D50455241545552450000000023
:0E0644004F5554505554204F5650204F4B00E8
:1006520082B00190019B9A6880235B051A40802337
:100662005B059A4201D1012300E00023180002B089
:020672007047CF
:0A06740082B00190C04602B070474A
:0A067E0082B00190C04602B0704740
:1006880000B585B00190019B9B6A0393039B1800FA
:0A069800FFF7ECFFC04605B000BDFF
:1006A20000B585B00190019B9B6A0393039B9B6DF0
:1006B20040221A43039B9A65039BDB6D04221A4373
:1006C200039BDA65039B1800FFF7D8FFC04605B00D
:0206D20000BD69
:1006D40000B583B00190019B1800F3F787FC030079
:0606E400180003B000BD88
:1006EA0000B587B0039002910192009317236B44DF
:1006FA0000221A70039B24229B5C012B01D1022346
:10070A0070E0039B242201219954039B25229B5CC0
:10071A00DBB2012B57D1039B252202219954039B5B
:10072A000022DA63039B1B681A68039B1B6801217A
:10073A008A431A60009B019A02990398F3F7ADFD68
:10074A00039B1B6B002B08D0039B1B681A68039B37
:10075A001B680E210A431A600FE0039B1B681A6884
:10076A00039B1B6804218A431A60039B1B681A684F
:10077A00039B1B680A210A431A60039B5B6C1A6875
:10078A0080235B02134008D0039B5B6C1A68039BAF
:10079A005B6C802149000A431A60039B1B6D002B86
:1007AA0008D0039B1B6D1A68039B1B6D80214900AF
:1007BA000A431A60039B1B681A68039B1B68012182
:1007CA000A431A6007E0039B242200219954172345
:1007DA006B4402221A70039B242200219954172386
:0A07EA006B441B78180007B000BD37
:1007F40082B00190080011006B460233021C1A807B
:100804006B4601330A1C1A706B4601331B78002BAC
:1008140005D06B4602331A88019B9A6104E06B464B
:0E08240002331A88019B9A62C04602B07047E8
:1008320082B001900A006B4602331A80019B5B6909
:100842006A4602321288134005D06B4602331A8878
:10085200019B9A6204E06B4602331A88019B9A61FB
:06086200C04602B0704721
:1008680000B585B00190019B1B68DA68019B1B6885
:10087800A0218A43DA60F2F71FFD030003930AE020
:10088800F2F71AFD0200039BD21AFA239B009A4240
:1008980001D9032306E0019B1B68DB682022134073
:0A08A800EED00023180005B000BDDB
:1008B20084B002006B4607331A70002303930B23A4
:1008C2006B446A46073212781A7009E0039B0133BF
:1008D20003930B236B440B226A4412780A3A1A7070
:1008E2000B236B441B78092BF0D8039BDBB21B0153
:1008F200DAB20B236B441B781343DBB2180004B04B
:0209020070473C
:0A09040082B00190C04602B07047B7
:0A090E0082B00190C04602B07047AD
:1009180084B00190009100230393009B0C2B1ED000
:10092800009B0C2B20D8009B082B13D0009B082B76
:100938001AD8009B002B03D0009B042B05D013E092
:10094800019B1B685B6B03930FE0019B1B689B6B10
:1009580003930AE0019B1B68DB6B039305E0019B93
:100968001B681B6C039300E0C046039B180004B08F
:020978007047C6
:0A097A0082B00190C04602B0704741
:0A09840082B00190C04602B0704737
:0A098E0082B00190C04602B070472D
:0A09980082B00190C04602B0704723
:0A09A20082B00190C04602B0704719
:0A09AC0082B00190C04602B070470F
:0A09B60082B00190C04602B0704705
:0A09C00082B00190C04602B07047FB
:0A09CA0082B00190C04602B07047F1
:1009D40082B00190019B80229B58212B2AD1019B3C
:1009E40056229B5A9BB2002B10D1019B1B681A689C
:1009F400019B1B6880218A431A60019B1B681A684B
:100A0400019B1B6840210A431A6013E0019B1B6D84
:100A14001A78019B1B689A62019B1B6D5A1C019BEF
:100A24001A65019B56229B5A9BB2013B99B2019BCA
:0A0A340056229952C04602B07047E6
:100A3E0030B589B00590049103921A000A236B44D5
:100A4E001A800A236B441B88002B04D00A236B44A4
:100A5E001B88022B03D90A236B4401221A800A2316
:100A6E006B441B8809330793039B002B02D0039B17
:100A7E00012B02D1079B013307930A236B441B887A
:100A8E00039D049C0C990598079A019200932B00E4
:100A9E002200F7F7C6FD059B00225A77059B002220
:100AAE009A84059B00221A84059B262200219954C4
:100ABE00059B00221A77059B0022DA83059B2222D2
:0A0ACE0000219954C04609B030BD64
:100AD80000B583B00190019B1B681A68019B1B68D5
:100AE80040218A431A60019B802220219950019B52
:100AF80000221A67019B1800FFF75EFFC04603B08B
:020B080000BD2E
:100B0A0010B584B001900091009B023B1A000A24A0
:100B1A006C44019B11001800F8F727F803002380A2
:100B2A00009B013B019AD3181B781BB21B021AB215
:100B3A00009B023B0199CB181B781BB213431AB2D4
:100B4A0002AB1A800A226A4402AB12881B889A42B4
:100B5A0002D1009B039302E001235B420393039BB0
:060B6A00180004B010BDEC
:100B700082B00190019A8A239B000021D150019BF1
:0A0B800000221A75C04602B070474B
:100B8A0000B585B0019000230393019B273302939C
:100B9A00019B180000F062FC029B1978019A282335
:100BAA00FF33D154039B01330393019B2833FF3353
:100BBA001800029B1B78039A029900F093FC030029
:100BCA000393019B2833FF33039A1100180000F0A6
:100BDA004FFC03000393019A8B239B000399D15086
:100BEA00019B180000F022FC019B1800FFF7BBFFD5
:060BFA00C04605B000BD7D
:100C000010B580235901A023DB0501221800FFF74E
:060C1000F1FDC04610BD1D
:0A0C160010B5F9F722F9C04610BD31
:020C2000FEE7ED
:100C220010B582B00B4601AC2070012120460A4665
:100C320000F04EFD002801D0207800E0C04302B051
:020C420010BDE3
:100C440010B50446002000290DD0002A0BD00978E5
:100C540048B2002808D4002C00D02160002119607B
:0E0C64005960411E884110BD0120C04310BDE3
:100C720008D1002806D1F54204D801D3002A01D1B7
:100C82006D0D09D10020C143090DC904F0BDF9D190
:100C92001242F7D1640DF5D00020C143490549083D
:100CA200A6E000206146F0BDF0B50127FF070E0067
:100CB2005E403E40B446BE0A4C18DD18F442D7D21C
:100CC200F542E4D2640DECD06D0DEAD06419C9028C
:100CD2003943460DC0023143DB023B43DB0A10B409
:100CE2008E4685B297B26F43140C6C433E0CA41926
:100CF200260C2404BFB227439CB26C43A419190CDE
:100D02006943250CA4B249190D04090C6419000C9D
:100D120095B245433E0C76193743BFB2360C150CDB
:100D22004543AD19A6B2240CAD192E0437432E0C3F
:100D320036199DB24543AD19ACB22E0C89191D0C62
:100D420045436D182E04290C3443704680B295B287
:100D520045433E0C76193743BFB2360C150C45435A
:100D6200AD19A6B2AD19240C2E0437432E0C361938
:100D72009DB24543AD19ACB22E0C89191D0C4543E9
:100D82006D182E043443290C75462D0C90B268431D
:100D92003E0C80190604BFB23E43070CA0B23F18B6
:100DA200120C6A43D019020C80B2240CA4189AB215
:100DB2006A43121914042043120C89181B0C6B434A
:100DC200C91810BC01273D05294203D1B61940417B
:100DD2004941013CFF077D0D013D641B0BDB6D00AA
:100DE200AC4209DA240500254208BE41684161414E
:0A0DF20066463143F0BD54E74EE7BA
:100DFC0030B581B0044668460170206900280FD0D8
:100E0C000CCC083C9A4233D26269531C6361815406
:100E1C00A069616981422BD1204600F02EF827E0B1
:100E2C00E068002809D00CCC083C9A4220D2551C12
:100E3C009D4200D1002181541AE0A068002808D0FE
:100E4C000CCC083C9A4213D2551C9D420DD0C9B211
:100E5C000CE0236A002B0BD003CC083C884207D251
:100E6C00694601222046984702E0002192008150F9
:0A0E7C002068401C206001B030BD6A
:100E860010B54269002A07D00446036A002B01D038
:0A0E9600216998470020606110BD3B
:100EA00080B5CB0606D4890501D5302100E020218C
:060EB00000F09FFC80BD74
:100EB60070B514460D460646FDF793F901463046D1
:0A0EC6002A462346FDF7C1FE70BD69
:0A0ED00080B50068FEF7FAFD80BD52
:100EDA00C2680169914201D9D04302E0D24389181C
:060EEA0080680818704743
:100EF000F0B581B0154604464068A268E6688019DE
:100F0000971BAF4204D92A46FEF774FE751909E013
:100F10000E463A46FEF76EFEF119ED1B60682A4652
:0A0F2000FEF768FEE56001B0F0BDC9
:100F2A0082B00190019B1A68E0235B041340180009
:040F3A0002B070474A
:100F3E0084B0039002910192039B5B69029A042193
:100F4E000A40072191400A00D2431A40029B042115
:100F5E000B40019999400B001A43039B5A61C046FE
:040F6E0004B0704714
:100F720082B00190019BDA68C0231B01134001D1AA
:0C0F8200012300E00023180002B07047BB
:100F8E0082B001900091019B9A6A009B5B035B0B00
:0C0F9E001A43019B9A62C04602B07047E3
:100FAA0082B00190019B9B6801221340012B01D161
:0C0FBA00012300E00023180002B0704783
:100FC60082B00190019B9B6802221340022B01D143
:0C0FD600012300E00023180002B0704767
:100FE20082B00190019B9B6804221340042B01D123
:0C0FF200012300E00023180002B070474B
:100FFE0000B585B00190019B1B681800FFF7DCFF60
:10100E0003000393019B1B681800FFF7C7FF031E25
:10101E0040D0039B002B3DD1019B1B689B68052292
:10102E001340012B0DD1019B1B681800F2F7AFF98D
:10103E00019B1B6803221A60F2F73BF9030002932F
:10104E0022E0019B9B6D10221A43019B9A65019B26
:10105E00DB6D01221A43019BDA6501231BE0F2F7D7
:10106E0028F90200029BD31A022B0DD9019B9B6D0E
:10107E0010221A43019B9A65019BDB6D01221A43D4
:10108E00019BDA65012306E0019B1B689B68012228
:0C109E001340E4D10023180005B000BD91
:1010AA0082B00190019B9B6801221340012B01D160
:0C10BA00012300E00023180002B0704782
:1010C60082B00190019B9B68DB0FDA0780231B0629
:1010D6009A4201D1012300E00023180002B07047B4
:1010E60000B585B0029101920F236B44021C1A7061
:1010F600029A0F236B441B785BB211001800F2F7BB
:08110600FEFEC04605B000BD6D
:10110E0000B583B002006B4607331A706B46073387
:10111E001B785BB21800F2F7C2FEC04603B000BDEA
:10112E0000B583B002006B4607331A706B46073367
:10113E001B785BB21800F2F7C8FEC04603B000BDC4
:10114E0084B001900A006B4602331A80019B1B6922
:10115E006A4602321288134004D00F236B440122D8
:10116E001A7003E00F236B4400221A700F236B4496
:08117E001B78180004B0704753
:1011860082B002006B4606331A80C04602B0704732
:1011960000B585B001900F236B4400221A70019BA5
:1011A6001B68DB68402213402ED1019B1B68DA685E
:1011B600019B1B6880210A43DA60F2F77EF8030080
:1011C600029316E0F2F779F80200029BD21A0F2377
:1011D6006B440F21694409781970FA239B009A42DF
:1011E60007D90F236B4403221A70019B292203217E
:1011F6009954019B1B68DB684022134004D10F23DE
:101206006B441B78032BDDD10F236B441B7818002E
:0412160005B000BD62
:10121A0000B587B0059004910392049AC02359013E
:10122A000598039B009313000022F5F708F9031EA3
:10123A0007D0059B1B6E20221A43059B1A660323BF
:10124A0027E0049A0598039B00931300002280214B
:10125A00F5F785F8031E07D0059B1B6E20221A435B
:10126A00059B1A66032314E0049AC023D900059843
:10127A00039B009313000022F5F7E1F8031E07D041
:10128A00059B1B6E20221A43059B1A66032300E066
:08129A000023180007B000BD9D
:1012A20000B583B00190019B002B01D101231EE008
:1012B200019B3D229B5CDBB2002B07D1019B3C22B0
:1012C20000219954019B1800FFF71BFB019B3D2253
:1012D20002219954019B1A68019B043319001000E2
:1012E200F5F7DFFB019B3D220121995400231800F1
:0412F20003B000BD88
:1012F60086B0039002910192029B1F2213400122A5
:101306009A4013000593039B1B6A059AD2431A4021
:10131600039B1A62039B1A6A029B1F210B400199C9
:1013260099400B001A43039B1A62C04606B07047E9
:1013360084B00190019B80229B58212B2FD1019BC9
:1013460056229B5A9BB2002B10D1019B1B681A6830
:10135600019B1B6880218A431A60019B1B681A68DF
:10136600019B1B6840210A431A6018E0019B1B6D14
:101376000393039B1B881A00019B1B68D205D20DA1
:101386009A62019B1B6D9A1C019B1A65019B562252
:101396009B5A9BB2013B99B2019B56229952C04679
:0413A60004B07047D8
:1013AA0082B00190019B80229B58212B2BD1019B5B
:1013BA0056229B5A9BB2002B10D1019B1B681A68BC
:1013CA00019B1B6880218A431A60019B1B681A686B
:1013DA00019B1B6840210A431A6024E0019B1B6D94
:1013EA001A78019B1B689A62019B1B6D5A1C019B10
:1013FA001A65019B56229B5A9BB2013B99B2019BEB
:10140A00562299520FE0019B1B681A68019B1B68C0
:10141A0080218A431A60019B1B681A68019B1B681A
:0C142A0040210A431A60C04602B070471F
:1014360000B583B00190019B26220C219954019B93
:101446001868019B2833FF331900019A8B239B00F0
:10145600D3589BB21A00F5F7ECFCC04603B000BDAA
:1014660082B00190019A8B239B000021D150C04687
:0414760002B0704709
:10147A0010B584B0019000910E246C44009A019B2F
:10148A0011001800F7F771FB030023800D236B444A
:10149A000E226A4412881A700E236B441B881B0A98
:1014AA009AB203AB1A70019A009BD3180D226A44B0
:1014BA0012781A70009B01330093019A009BD3188B
:1014CA0003AA12781A70009B01330093009B18003C
:0414DA0004B010BD8D
:1014DE0082B00190019B1B7DDBB2180002B07047F9
:1014EE0000B587B00390029101921A006B46033348
:1014FE001A70029B01331B780493049B102B1FD090
:10150E00049B102B27D8049B032B03D0049B062B84
:10151E000BD020E06B4603331B78019A0299039897
:10152E00F7F7ABFB030005931EE06B4603331B7806
:10153E00019A02990398F7F7CEFC0300059313E086
:10154E006B4603331B78019A02990398F7F723FC35
:10155E000300059308E0019B04990398012200F013
:10156E0007F803000593C046059B180007B000BDA1
:10157E0084B00390029101920093029B80330293F8
:10158E00039A009BD318029AD2B21A70009B0133B1
:10159E000093039A009BD318019AD2B21A70009B43
:0C15AE0001330093009B180004B070474C
:1015BA0030B58BB005000C00100019006B460633DD
:1015CA002A1C1A8001AB221C1A806B460233021CA9
:1015DA001A806B460A1C1A806B4606336A46023228
:1015EA0010881B8819B202B2914200DD031C1BB29B
:1015FA00099301AB6A4610881B8819B202B291425C
:10160A0000DD031C1BB208936B4606336A4602329E
:10161A0010881B8819B202B2914200DA031C1BB26D
:10162A00079301AB6A4610881B8819B202B291422D
:10163A0000DA031C1BB206930EAB00229B5E0593D5
:10164A00079A099BD31A0493049B002B01D1002308
:10165A0015E0069A089BD31A0599099A8A1A5A43D9
:10166A000799099BCB1A08994B43D31803930499FA
:10167A000398FDF730FA03000293029B1BB218008D
:04168A000BB030BDB4
:10168E0000B583B002006B4606331A806B460633F4
:10169E001A8880239B009A4201D1FFF7B5FAC04603
:0416AE0003B000BDC8
:0416B200C046704777
:0416B600C046704773
:0416BA00C04670476F
:0416BE00C04670476B
:1016C20010B580239B001800F3F7E9FAC04610BD5D
:1016D200F0B581B01E4615460C4607461846FEF781
:1016E2007CF90146002000290AD46543A54207D3AC
:1016F200304639462A46FFF7EAFB2146FDF717FA3C
:0417020001B0F0BD85
:04170600C80F704751
:10170A00F0B581B01C4615460091CA0017183E462E
:10171A00103EB068F1682A46FFF7C2FA0CCEFCF711
:10172A00B4FD009A032A0DDB183F561E2A462346AB
:10173A00FFF7B6FA0CCF083FFCF7A7FD761E083F65
:10174A00012EF3D82A462346FFF7AAFA01B0F0BDC4
:10175A00F0B581B01D4616460346C800022916DBBD
:10176A0000931F18083F4C1C304629460CCF083FEF
:10177A00FCF78BFD32462B46FFF792FA641E083FB0
:10178A00022CF3D8009B083306460D4600E01B18CE
:10179A00083B0CCB30462946FCF777FD01B0F0BD7B
:0817AA00C1174840401A7047C6
:1017B200024601207F2901D9C0437047117070474A
:0C17C200014661391A2900D22038704716
:0C17CE00014641391A2900D22030704732
:0C17DA00014661391A2900D220387047FE
:0C17E600014641391A2900D2203070471A
:1017F20070B5012A09DB0C460546561C28462146CF
:0C180200FFF7FBFA761E012EF8D870BD2F
:10180E0010B50C46436A01212046FFF75BFF10BD61
:04181E0040207047AF
:10182200F0B583B016460D46C768002101900269E3
:10183200BA42029103D9F9435418826803E0F9438A
:10184200511882688C184168D21B944200D3144606
:10185200C819B44200D3344629462246FEF7C9F9D4
:10186200E719019881688F4200D100270299C76069
:10187200361B2D196118002ED9D1084603B0F0BDD0
:07188200414D00504D000034
:0F18890025612025622025652025542025590042
:07189800286E756C6C29003D
:02189F00430004
:0218A1002E0017
:1018A30053756E646179004D6F6E64617900547590
:1018B3006573646179005765646E6573646179006B
:1018C3005468757273646179004672696461790062
:0A18D30053617475726461790000BE
:0118DD00000A
:0918DE00256D2F25642F257900EA
:0918E70025483A254D3A2553002D
:0D18F0000007032004170201085710408074
:0518FD002D494E4600DC
:051902002D696E660076
:051907002B494E4600D3
:05190C002B696E66006E
:1019110000000000000054545220524547474553EF
:0119210000C5
:091922005465726D696E616C0080
:10192B002020202020202020206828282828202044
:10193B00202020202020202020202020202020209C
:10194B004810101010101010101010101010101054
:10195B0084848484848484848484101010101010F4
:10196B00108181818181810101010101010101014D
:10197B000101010101010101010101101010101001
:10198B00108282828282820202020202020202021E
:10199B0002020202020202020202021010101020C6
:1019AB00303132333435363738394142434445468A
:1019BB0030313233343536373839616263646566BA
:0419CB004E414E003B
:0419CF006E616E00D7
:0119D300FF14
:1019D400A51A0108B0000020960F0000B71A0108EC
:1019E40000000020F4190108B00000004BFD0008BD
:1019F40088B0019000911F236B4400221A70019B50
:101A04000693009B05931A4B5A69194B8021C9020E
:101A14000A435A61EFF310830393039B049372B652
:101A2400C04610E0059A069B12681A60059B0433B1
:101A34000593069B043306931F236B441A781F23D4
:101A44006B4401321A701F236B441B783F2BE9D976
:101A5400C046074B1A6980235B021340F9D1049BEB
:101A64000293029B83F31088C046C04608B07047B7
:101A740000200240BCFC0008BCFC0008BCFC0008C0
:101A8400BCFC0008BCFC00080400000001000000CD
:101A9400CC0B0020D00B0020D40B00200024F40039
:101AA400206861680834002200E042540139FCD502
:021AB400704779
:101AB60020686168A2680C3401E08B5C8354013AAB
:041AC600FBD5704795
:101ACA00FFFFFFFFFFFFFFFFFFFFFFFFFFFFFFFF1C
:101ADA00FFFFFFFFFFFFFFFFFFFFFFFFFFFFFFFF0C
:101AEA00FFFFFFFFFFFFFFFFFFFFFFFFFFFFFFFFFC
:101AFA00FFFFFFFFFFFFFFFFFFFFFFFFFFFFFFFFEC
:02F7FA00FFFF0F
:04F7FC005C59EE2B3B
:040000050800FD559D
:00000001FF
